:020000040800F2
:1000000000200010C1A502081D940108ADFD0008E4
:1000100019940108159401081194010800000000CA
:100020000000000000000000000000000D94010826
:10003000099401080000000005940108CDEB0008B8
:1000400029A6020829A6020829A6020829A602084C
:1000500029A6020829A6020855AD000819AD000816
:100060006DF8000831F80008F5F7000845BE0008F3
:1000700035BE000825BE000815BE000805BE0008F4
:10008000F1BD0008DDBD000829A6020829A6020866
:10009000AD94010829A6020829A60208B9F70008AC
:1000A00029A60208F9070108C90701082108010863
:1000B000E9070108D907010829A6020829A60208AC
:1000C00029A6020829A6020829A6020829A60208CC
:1000D00029A60208F9EC00087DEC000801EC0008F4
:1000E0007DF7000829A60208F593010829A6020851
:1000F00029A6020829A6020829A6020829A602089C
:1001000000000000000000000000000029A6020816
:1001100029A6020829A6020829A6020829A602087B
:10012000C9BD0008B5BD0008A1BD00088DBD00080F
:1001300079BD000829A602080000000000000000A8
:1001400029A6020829A6020829A602080000000024
:10015000000000000000000000000000000000009F
:10016000000000000000000029A6020829A60208DD
:1001700029A60208000000000000000000000000A6
:080180000000000029A602089E
:100188002DE9F04FB0F908502DED048B0D81EDB23B
:10019800382D8FB00C4600F08E82804691462ED9BD
:1001A800802D00F0928079D8522D00F0E98040F23D
:1001B8003682542D00F0D8826E2D40F013817E4B8C
:1001C8000A681B887D4DFF2BA8BFFF23511C2160A7
:1001D8001370A96881F3100189B220460BF07EF9EB
:1001E800774B204619880BF079F9296801F30F013C
:1001F80089B2204601250BF071F92B4647E0042D02
:1002080000F0A68240F2F381202D00F09D8040F29C
:100218001182242D00F09482282D40F0E3800B6891
:10022800DFF8BC81674E591C022221601A702368CE
:1002380006275A1C22601F7023680A22591C216055
:100248001A70236801255A1922601D70B8F8001029
:1002580020460BF043F9B8F8021020460BF03EF99F
:1002680023685A1922601F70236850225919216087
:100278001A7023680022591921601A7031882046A3
:100288000BF02CF9718820460BF028F92B462846EC
:1002980063810FB0BDEC048BBDE8F08F822D26D0B2
:1002A800C0F07A82A02D00F06B82FE2D40F09A807B
:1002B800454D05F1080635F8021B20460BF00EF9EE
:1002C800B542F8D101252B46E1E70B683F4A581C97
:1002D8000A211288206019702168FF2A01F10103A0
:1002E800A8BFFF22012523602B460A70CFE70B68C1
:1002F800374A324D1178374A581C20601970D18816
:1003080020460BF0EBF82C4B22681B88FF2B02F1E0
:100318000101A8BFFF2321601370A96881F31001B0
:1003280089B220460BF0DAF8296801F30F0189B287
:1003380020460BF0D3F8284B22681978531C012566
:1003480023602B461170A2E70B68224D591C6A786E
:1003580021601A7023682A78591C21601A70236852
:10036800AA78591C21601A70E98820460BF0B6F863
:1003780023682A79591C21601A7022686979DDE797
:100388000A68164E531C0321236006F10C071170EE
:100398003346062001212268551C25601170226809
:1003A8009F4202F101012160107000F0AA81997941
:1003B800D8790633EFE700BF844F0020884F00202C
:1003C80050690020EC2F002024380020FC2F00204A
:1003D800CD4F00205869002053690020D4ED020851
:1003E800083A0020A5F10A03E72B00F2EA80DFE8CB
:1003F80013F0A507E800E800E800E800E800E800D6
:10040800E800E800E800E800E800E800E800E800A4
:10041800E800E800E800E800E800E800E800E80094
:10042800E8007507E800E800E8006407E800E8006D
:10043800E8005F07E8001E07E8000507E800DE0699
:10044800E800C606E800A006E800CB06E800E800D9
:10045800E800C7029706E8009006E800E80087066B
:10046800E800E800E800E800E800BA02E800E80070
:10047800E800E8006B06E8004906E80037061F06B2
:10048800E800E800E800E800E800E800E800B00557
:10049800E8008505E8002405E800DA04E800C90456
:1004A800E800E800E800E8006D04960464043C04F1
:1004B8002A04E800E80011040504E8008103640345
:1004C800E800E800E800E8005903E800E80038031D
:1004D800E800E800E800F403DB032803EA02E80088
:1004E800E800E800DA02E800E800E800E800E800D0
:1004F800E800E800E800E800E800E800E800E800B4
:10050800E800E800E800E800E8006D04E800E8001A
:10051800E800E800E800E800E800E800E800E80093
:10052800E800E800E800E800E800E800E800E80083
:10053800E800E800E800E800E800E800E800E80073
:10054800E800E800E800E800E800E800E800E80063
:10055800E800E800E800E800E800E800E800E80053
:10056800E800E800E800E800E800E800E800E80043
:10057800E800E800E800E800E800E800E800E80033
:10058800E800E800E800E800E800E800E800E80023
:10059800E800E800E800E800E800E800E800E80013
:1005A800E800E800E800E800E800E800E800E80003
:1005B800E800E800E800E800E800E800E800CE020B
:1005C800F405742D00F03F81772D48D1D8F800301C
:1005D800D8F804209A421EBF5A1CC8F8002019787F
:1005E800A14A08BF002120460FF06EFB6AE6022DE3
:1005F80000F0218100F20E81012D7FF4F3AE0B682B
:100608000022591C21601A7023685A1C22601D7030
:1006180022682421531C23602B46117037E6442D91
:100628007FF4E0AE002A3FF44DAE904B13600125F5
:100638002B462CE6052D7FF4D5AE0B228C4920469F
:100648000AF01EFF08228B4920460AF019FF0125EF
:100658000722894920460AF013FF2B4617E6F52D95
:1006680000F0248198E84800292DA6EB030600F045
:10067800C08640F29586392D01F00286532D40F050
:10068800E5865A1CC8F800201978721E0329D2B2D0
:100698000DD84B1EDBB2794D794803EB430305EBCC
:1006A800430301705B7811B19A4201F06A874FF0F9
:1006B800FF352B46EBE50B68724901255A1C226071
:1006C8001D7023680522581920601A7023680A22B1
:1006D800581920601A7023680022581920601A706F
:1006E80023680A78581920601A7023684A785819BC
:1006F80020601A7022688978531923602B4611707C
:10070800C5E55F4B21681A78481C20600A70002AEA
:100718003FF4D8AD013AD2B202EB420206EB4202F4
:100728005278002A3FF4CEAD0132D5180133226841
:1007380013F8011F501C9D4220601170F7D1C1E5CC
:10074800514B1968204601250AF0B1FE2B469EE55B
:100758002A464E4920460AF093FE002120460AF018
:10076800BDFE22680021E9E50B6800215A1C2260C1
:10077800197022680125531923602B46117086E5EC
:10078800434B084619680AF092FE424B2046196806
:100798000AF08DFE404BD4E7404A414E93681168F9
:1007A80003EB83034FF6FF725B009342A8BF134627
:1007B8009142A8BF114623EAE37321EAE1719DB291
:1007C80089B24FF00A0E002714E0B368316803EBD2
:1007D80083034FF6FF725B009342A8BF1346914212
:1007E800A8BF114623EAE37321EAE1719DB289B2F9
:1007F8004FF0500E23685A1C2260204683F800E010
:100808000AF06CFE0137294620460AF067FE022FDF
:10081800DBD157E50B680222591C21601A70236846
:1008280001255A1922601D7022680021531923607E
:100838002B4611702BE504221A49204601250AF09F
:100848001FFE2B4623E5D8F80030D8F804209A423A
:100858001EBF5A1CC8F800201978134A08BF002187
:1008680020460FF031FA2DE5A9F8000879FB0008B9
:100878007CF1020888F1020894F10208D4ED02081C
:10088800D06A00209F280020FC29002074F102086B
:10089800ACF7FF1FB0F7FF1FB4F7FF1FB02F002002
:1008A800F02F00206CF1020851FB0008D8F8003046
:1008B800D8F804209A4241F0D485AB4BFF221A7233
:1008C8004FF00008A94D16F079FC41463022A8489F
:1008D80085F800802CF0E5F98DF814809DF8143027
:1008E8000B2B01F26E86A34FA14E42469DF81430A1
:1008F80003EB430307EBC3035B7CE3B19DF81430C0
:1009080003EB430307EBC3035B69A3B19DF8143002
:1009180003EB430307EBC3032021586946F8220081
:100928000EF008FD2B7856F823000EF0C5FE2A7845
:100938000132D2B22A709DF814300133DBB28DF83F
:1009480014309DF814300B2BD0D92368591C216022
:100958001A70B9F1000F3FF4B5AC874BC9F80030F5
:1009680001252B4693E4236800255A1C226029465A
:1009780020461D700AF09BFD294620460AF097FD87
:100988000021204601250AF092FD2B467FE47B4D8D
:100998002046A9890AF0A2FD6989204601250AF0A6
:1009A8009DFD2B4673E4764D2046A98A0AF096FDF4
:1009B800E98A20460AF092FD298B204601250AF093
:1009C8008DFD2B4663E4DFF8DCE10027FEB27146BB
:1009D80000232268501C206016702268501C20607A
:1009E8001370226811F8010F0133551C062B25607E
:1009F8001070EED10137062F0EF1060EE6D16149CF
:100A080000232268501C206017702268501C206048
:100A18001370226811F8010F0133551C0B2B256048
:100A28001070EED123685849581C072220601A70AC
:100A380023680022581C20601A70226891F8F01070
:100A48007CE42368514A524910784C4A5D1C256061
:100A5800187023689278581C20601A702268897868
:100A68006CE44C4D05F16006A98820460AF036FD75
:100A7800E98820460AF032FD298920460AF02EFD31
:100A88002368AA7A591C21601A702368EA7A591CCB
:100A980021601A7055F80C1B20460AF008FDB54273
:100AA800E2D10FE43C4952232268501C20601370A5
:100AB80011F8013F002BF7D104E4384D00232268D8
:100AC800286803EB4301561C405C266010702A68B6
:100AD80020680A44461C5278266002702A682068FA
:100AE8000A4401339278411C0A2B21600270E6D136
:100AF800FFF7E8BB2A4D23682A68591C1278216041
:100B08001A702B6822689978531C2360002311708F
:100B18002A6821681A4401335279481C032B206043
:100B28000A70F5D123682A68591C127A21601A7054
:100B380023682A68591CD27821601A7023682A68A9
:100B4800591C127921601A702B68204659890AF0BD
:100B5800C5FC23682A68591C527A21601A702B68D0
:100B680022685978FFF7EABB641C00202F65002033
:100B78009C270020A460002001370208183A0020B2
:100B88001C440020C3510020E0500020D053002016
:100B9800303A00205068002014CE0208A82800200F
:100BA800406E00209F5100202268BB4BBB4918783B
:100BB800551C2560107022685878551C25601070E7
:100BC80022689B78501C20601370C9882046012534
:100BD8000AF084FC2B46FFF75ABBB04D2046298803
:100BE8000AF07CFC698820460AF078FCA98820462F
:100BF80001250AF073FC2B46FFF749BB002120466C
:100C08000AF055FC0125002120460AF067FC2B4616
:100C1800FFF73DBBA24D204629880AF05FFC698892
:100C280020460AF05BFCB5F904309E49DA1781FBCF
:100C38000313C2EBA30399B2204601250AF04EFC28
:100C48002B46FFF724BB984E3378002B3FF43AAB82
:100C5800964F002537F8021F20460AF03FFC3378EC
:100C680001359D42F6DBFFF72DBB914D914EDFF824
:100C78008082DFF88092DFED908ADFED909A9FED19
:100C8800909A05F1200708E0204604350AF026FC72
:100C9800AF4206F118063FF415AB717C0029F3D07A
:100CA80095ED008AB0EE480A29F0EEFE98F800307B
:100CB800002B41F0A48381B2E6E710228149204647
:100CC80001250AF0DDFB2B46FFF7E1BA0DF1140907
:100CD80000220592DFF820A27B4B03920492C9F808
:100CE8000420904601214FF6FF7B07E008F1010838
:100CF800B8F10B0F01F0DD821AF9011F4E1CF5D077
:100D08004BFA08F2D007F1D51A8842FA08F2D2074E
:100D1800ECD5484601930AF005FE019BE6E76B4EC9
:100D2800338AB3F5007F06F1340594BF0127042701
:100D3800403655F8041B91FBF7F1204689B20AF0BA
:100D4800CDFBAE42F5D1624D624F05F10C06B5EC14
:100D5800010AD7ED087A80EE270A29F095FE81B2BC
:100D680020460AF0BBFBAE42F1D15B4D05F10C0603
:100D780055F8041B204689B20AF0B0FBB542F7D1FA
:100D8800FFF7A0BA2368554A5549D078554A5D1CE3
:100D98002560187023681278581C20601A70226821
:100DA800C978FFF7CBBA002120460AF097FB00214B
:100DB80020460AF093FB002120460AF08FFB2268A8
:100DC800494D0023511C2160137022682968501C6A
:100DD80091F82F102060117022682968501C91F832
:100DE8003A102060117022682968501C91F83B1055
:100DF800206011702268511C216013702268511CF8
:100E0800216013702268511C216013702B682046E2
:100E1800D98F0AF063FB2B682046998F0AF05EFB96
:100E280023682A68591C92F8312021601A702B68AF
:100E3800226893F83210FFF781BA2C4D23686A793B
:100E4800294E591C21601A7033682046198C0AF003
:100E580045FB33682046598C0AF040FB69892046D7
:100E68000AF03CFBA98920460AF038FB3368204683
:100E7800998C0AF033FB33682046D98C0AF02EFB94
:100E8800E98920460AF02AFB298A204601250AF02A
:100E980025FB2B46FFF7FBB9103A0020D84100206C
:100EA800D03B002067666666F8630020B2690020C0
:100EB80040380020A46000200000404200407444F4
:100EC80000E0824430380020DC690020E037002050
:100ED8000C5C0020E45300200C420020183A00204B
:100EE800303A0020283A0020A8280020D0530020BB
:100EF800444400204C49002044CE0208B24EF37806
:100F0800002B01F06F8223680822591C21601A7097
:100F180023680122991821601A702368AB4D591C67
:100F28002A7921601A702368AA78591C21601A70DE
:100F3800298820460AF0D2FA698A20460AF0CEFAB1
:100F48002368F279591C21601A702268E978FFF742
:100F5800F5B924F0B3FFFF28064601F07A820EA9FE
:100F6800002501F82E5D0DF109008DF8095024F0D7
:100F7800A9FE0EA800F82D5D24F098FE0EA800F832
:100F88002C5D24F087FE0EA820F8245D24F076FE60
:100F980023685A1C22601E7023689DF80920591C7A
:100FA80021601A7023689DF80A20591C21601A7064
:100FB80023689DF80B20591C21601A7023689DF83E
:100FC8000C20591C21601A70BDF814102046012508
:100FD8000AF084FA2B46FFF75AB97D4B03F17005E6
:100FE80022681978501C2060117022685978501CAA
:100FF8002060117022689978501C20601170226856
:10100800D978501C2060117022681979501C206012
:10101800117022685979501C2060117022689979E2
:101028000733501C9D4220601170D9D1FFF74AB98F
:101038002268684B0125511C216015702268997837
:1010480050192060117022681978501920601170A9
:1010580022685978531923602B461170FFF717B986
:10106800236800255A1C22601D7023685A1C2260C0
:101078001D7023685A1C226029461D7020460AF0FC
:1010880016FA7DE4544E3378002B3FF41BA9534FD6
:101098000025B846236817F81520591C21601A70D6
:1010A80098F8011001EB810101EB810101F2EE21B9
:1010B80089B220460AF012FA337801359D4208F1C8
:1010C8000208E7DBFFF7FEB82368454D591C2A786C
:1010D80021601A7023686A78591C21601A7069881F
:1010E80020460AF0FBF923682A79591C21601A70F6
:1010F800E98820460AF0F2F92268297AFFF71EB932
:1011080008223849204601250AF0BAF92B46FFF78C
:10111800BEB82268344B501C9978206011701FE5C6
:1011280022680121531823600D460B461170FFF702
:10113800AEB82E4B03F15A0522685979501C20602D
:10114800117022681978501C206011702268597833
:10115800501C2060117022689978501C2060117012
:101168002268D978501C20601170226819790633DA
:10117800501C9D4220601170DED1FFF7A3B8194BB7
:101188002268597DFFF7DAB8194D1A4E05F1300774
:1011980095F902100023F2568A4200F0E4800C33DD
:1011A800482BF8D10835AF42F2D1FFF78BB8124D72
:1011B80005F1800655F8041F20460AF078F9AE427A
:1011C800F8D1FFF77FB800BFD05300201C4400209F
:1011D800906600200D2F0020F8630020782800205A
:1011E800EC4100201C4900203C3A00204425002006
:1011F800CC6D0020B0480020DC500020894D05F15E
:101208004006B5F8801020460AF068F9236895F87A
:101218008220591C21601A70236895F883200435B0
:10122800591CB54221601A70EBD1FFF74BB87E4DBF
:1012380023682A7A591C21601A70A98B20460AF063
:101248004DF9298B20460AF049F9698B20460AF0A6
:1012580045F92368EA7C591C21601A70E98C2046FC
:101268000AF03CF9298D20460AF038F92368AA7F4C
:10127800591C21601A70236895F82020591C216098
:101288001A70A98C20460AF029F92368EA7A591CB1
:1012980021601A70E96820460AF009F923682A7C57
:1012A800591C21601A70226895F82110FFF746B87A
:1012B8005E4B22681978FFF741B85D4D20462988B2
:1012C8000AF00CF9A98820460AF008F9298920466D
:1012D80001250AF003F92B46FEF7D9BF554D564FA5
:1012E80005F1500600212878544A0B4606E00133E0
:1012F800242B02F10C0233D012F80C1C8842F6D1D0
:1013080003EB4303226807EB8303511C93F8443033
:101318002160137023686A78591C21601A70236849
:10132800AA78591C21601A702368EA780435591C78
:10133800B54221601A70D5D1FEF7C4BF404828F0E5
:101348007DFC00287EF7BEAF3D4B1D18226813F8C0
:10135800011B501CAB4220601170F7D1FEF7B2BFE1
:1013680000231B7AFFDE23685A1C22601970298823
:1013780020460AF0B3F82368EA78591C21601A70ED
:1013880023682A79591C21601A702368AA79591C84
:1013980021601A7023686A79591C21601A7001E764
:1013A800212D53D11A46591CC8F80010254D12F8A2
:1013B800021B6970C8F800205A782A70DA1CC8F82D
:1013C80000209B78AB7040460AF04FF8D8F8003000
:1013D800E880591C1A46C8F8001012F8021B297137
:1013E800C8F800205B786B714FF0FF352B46FEF78D
:1013F8004EBF5A1CC8F800201B780A2B01F05D80EC
:10140800502B7FF454A940460AF02FF80E4E308036
:1014180040460AF02AF84FF0FF3570802B46FEF759
:1014280036BF00BFE05000201C490020603A002071
:1014380074370020643A002014CE02085CCE0208FB
:10144800902E002058690020EC2F00200B3DEF2D36
:101458003FF62DA901A252F825F000BF132200087B
:10146800B7060008B7060008B7060008B706000860
:10147800B7060008B7060008B7060008B706000850
:10148800B7060008B7060008B7060008B706000840
:10149800B7060008B7060008B7060008B706000830
:1014A800B7060008B7060008B7060008B706000820
:1014B800B7060008B7060008B7060008A521000807
:1014C800B70600088B210008B70600086921000844
:1014D800B7060008B7060008B70600085521000837
:1014E800B70600089F200008B70600086720000814
:1014F800B70600083F200008B70600082B200008A0
:10150800B7060008C91F0008B7060008811F0008B1
:10151800B7060008B7060008B7060008B7060008AF
:10152800CD020008B7060008611F0008B7060008CA
:10153800B7060008451F0008B7060008B7060008E8
:10154800B7060008B7060008B7060008B70600087F
:10155800B7060008B7060008B7060008B70600086F
:10156800F91E0008B7060008711E0008B706000833
:10157800B70600083D1E0008B7060008B7060008B1
:10158800B7060008B7060008B7060008B70600083F
:10159800B7060008E11C0008B7060008B71D0008D8
:1015A800B70600089B1C0008B70600083B1C00088B
:1015B800B70600080D1C0008B7060008B7060008A3
:1015C800B7060008B7060008B7060008B7060008FF
:1015D800B7060008B7060008B7060008B7060008EF
:1015E800B7060008B7060008B7060008B7060008DF
:1015F800B7060008B7060008B7060008B7060008CF
:10160800B7060008B7060008B7060008B7060008BE
:10161800B7060008B7060008B7060008B7060008AE
:10162800B7060008B7060008B7060008B70600089E
:10163800B7060008B7060008B7060008B70600088E
:10164800B7060008B7060008B7060008B70600087E
:10165800B7060008B7060008B7060008B70600086E
:10166800B7060008B7060008B7060008B70600085E
:10167800B7060008B7060008B7060008B70600084E
:10168800B7060008B7060008B7060008B70600083E
:10169800B7060008B7060008B7060008B70600082E
:1016A800B7060008B7060008B7060008B70600081E
:1016B800B7060008B7060008B7060008B70600080E
:1016C800B7060008B7060008B7060008B7060008FE
:1016D800B7060008B7060008B7060008B7060008EE
:1016E800B7060008B7060008B7060008B7060008DE
:1016F800B7060008B7060008B7060008B7060008CE
:10170800B7060008B7060008B7060008B7060008BD
:10171800B7060008B7060008B7060008B7060008AD
:10172800B7060008B7060008B7060008B70600089D
:10173800B7060008B7060008B7060008B70600088D
:10174800B7060008B7060008B7060008B70600087D
:10175800B31B0008B7060008751B0008B706000889
:101768008B1A0008711A0008191B0008B706000830
:10177800571A0008B70600082D1A0008B70600080F
:10178800CD190008B7060008A5190008B706000813
:10179800B7060008831900084F1900083B1900080C
:1017A8000D190008E5180008C3180008B706000856
:1017B800B7060008B7060008B7060008B70600080D
:1017C800B7060008B7060008B7060008B7060008FD
:1017D800B7060008B7060008B7060008B7060008ED
:1017E800B7060008B7060008B7060008A9180008D9
:1017F800B7060008B70600083F180008B706000833
:10180800B7060008B7060008B7060008B7060008BC
:10181800B7060008B706000825180008C34B1B7850
:10182800DB073EF544AF01250EF01AFB0EF0B4FBC2
:101838002B46FEF72CBD5A1CC8F800201A780F2A30
:101848003EF635AF991CC8F80010C2EBC202B84981
:1018580058788854D81CC8F800000A449978517000
:10186800191DC8F80010D9789170591DC8F80010D2
:101878001979D170991DC8F8001059791171D91DBD
:10188800C8F800109979517103F10801C8F80010DF
:10189800DB799371012522F099FA2B46FEF7F7BC04
:1018A800404609F0E2FDA34EB081404609F0DDFD57
:1018B800012570812B46FEF7EABC404609F0D5FDAC
:1018C8009D4EB082404609F0D0FDF082404609F0B6
:1018D800CCFD012530832B46FEF7D9BC1A46591C8E
:1018E800C8F8001012F8020BC8F80020DA1C597862
:1018F800C8F800209A781DF0A9FE00287EF4E2AC12
:10190800FEF7D5BE1A46591CC8F800108B4912F8C4
:10191800020B0870C8F8002086495A788A70DA1CC9
:10192800C8F80020864A9B78937001252B46FEF75D
:10193800AEBC844B844918684A22012528F030FF40
:101948002B46FEF7A4BC19465A1CC8F800207F4A4B
:1019580011F8020B1070C8F8001059785170D91C92
:10196800C8F800109B789370404609F07EFD784BCC
:101978000125D8802B46FEF78ABC404609F075FD44
:10198800734E3080404609F070FD7080404609F083
:101998006CFD0125B0802B46FEF779BC6D4F3B7876
:1019A800002B3EF48FAC6C4E0025404609F05DFDDF
:1019B80018F072FE3B78A6EC010A01359D42F4DB73
:1019C800FEF780BC0F2E7EF472AE5A1CC8F80020B9
:1019D8001D78072D3EF66BAE604F40460C2609F089
:1019E80044FD06FB05F6BD19A880404609F03DFDFB
:1019F800E880404609F039FDD8F8003028811A46B9
:101A0800591CC8F8001012F8021BA972C8F8002067
:101A18005B78EB72404609F011FD0125B8512B4661
:101A2800FEF735BC5A1CC8F800201878060600F1E5
:101A3800CB853E4B1B78DD073EF544AC032828BF19
:101A4800002001250EF0F0F92B46FEF720BC374B9D
:101A58001B78D8073EF536AC01250EF07FFC0EF05A
:101A68009BFA2B46FEF713BC304B1B78D9073EF583
:101A780029AC3B4B4FF4C87201251A802B46FEF760
:101A880006BC092E7EF613AE364F1A46591C3D6821
:101A9800C8F8001012F8021B2970C8F800205A78FC
:101AA800AA70DA1CC8F800209A78642A03F10401A5
:101AB800A8BF64226A71C8F80010DA78642A03F1B2
:101AC8000501A8BF6422AA71C8F800101A79EA7142
:101AD8009A1DC8F800205A79642A28BF6422D91DA3
:101AE8002A72C8F800109A79EA7003F10802C8F857
:101AF8000020DB792B71404609F0B7FC0A2E68817B
:101B080040F08C85012525F081FD2B46FEF7BFBBF3
:101B1800064B1B78DA073EF5D5AB134A1378012537
:101B280043F0040313702B46FEF7B1BB3569002060
:101B380090660020183A00201C440020D053002052
:101B4800303A0020A828002088DA0208103A00203D
:101B5800D84100202C380020E040002050680020A8
:101B68005C6E0020406E0020F0640020D24A1068AD
:101B7800DA1C01462133951EC8F8005012F8035CA0
:101B88000D70551EC8F8005012F8025C4D70C8F868
:101B9800002012F8015C8D700332934201F10301B9
:101BA800E9D122F0EDFAFEF78DBBC6F34706122EF7
:101BB8003EF67DADB6B10EAB0DF1120703EB46054F
:101BC800B946263D404609F050FC29F8020F4D451C
:101BD800F8D1BA4B37F8022F23F8022F4F45F9D125
:101BE800112E09D8B64A7300023B13440021223251
:101BF80023F8021F9A42FBD1B24A01231D461370F3
:101C0800FEF745BB1A46591CC8F80010AE4912F831
:101C1800020BC870C8F80020AC495A780A70DA1C60
:101C2800C8F80020AA4A9B78D37001252B46FEF7F6
:101C38002EBB404609F019FC404609F016FC404608
:101C480009F013FCD8F800309B4D9A1C2F68C8F88F
:101C580000205A7887F82F20DA1CC8F800209A78D4
:101C680087F83A201A1DC8F80020DA7887F83B2050
:101C78000733C8F80030404609F0F7FBF8874046BC
:101C88002F6809F0F2FB112EB88700F2F18428685A
:101C980087E75A1CC8F80020874D8E4F1B78D5F867
:101CA80000907B71404609F0E0FBA9F8200040460F
:101CB800D5F8009009F0D9FB052EA9F8220000F20A
:101CC800E9840EF0D7F81FF06FF92868012518F09D
:101CD80019FB2B46FEF7DBBA404609F0C6FB054662
:101CE80024F0ECF8FF283EF4EDAAB5F57A7F80F0F1
:101CF800A7840DF13809002309F8243DEE08494668
:101D080003A88DF80C30013623F0DCFF9DF80C3069
:101D1800F6B205F00705B34205F1010503D19DF8B8
:101D28001430AB4203D02946304624F0B3F8D8F833
:101D38000030D8F80420D21A012A7EF7C3AA5A1C08
:101D48000EA8C8F8002000221D7800F82C2D23F0DA
:101D5800ADFF9DF80C30AB420AD05F4B1B683BB11E
:101D68009A79AA4204D31B681B690BB12846984785
:101D7800D8F800305A1CC8F80020484600221D78C0
:101D88008DF8142023F086FF9DF81430AB423EF402
:101D980099AA514B1B68002B3EF494AA1B685B69F7
:101DA800002B3EF48FAA28469847FEF78BBA1A46AE
:101DB800591CC8F80010474E12F8021BB170C8F839
:101DC800002046495A780A70DA1CC8F80020444DA9
:101DD8009A782A711A1DC8F80020DB78092BA8BF49
:101DE80009234046AB7009F040FBD8F80030D8F81A
:101DF80004202880D11A012907DD404609F035FB67
:101E0800D8F80030D8F8042068829A4240F06584F7
:101E18000EF030F8D8F80030D8F804209A423EF492
:101E280051AA5A1CC8F800201B78EB7001252B46D4
:101E3800FEF72DBA2B4A1278012A3EF643AA194614
:101E48005A1CC8F80020284A11F8020B9070C8F8EC
:101E5800001059781170D91CC8F800109B7853707D
:101E680001252B46FEF713BA5A1CC8F800201E7825
:101E7800112E3EF61CAC9A1CC8F800201B4D5B784E
:101E880005F81630404609F0F0FA40F6CA039842C1
:101E9800A8BF184640F2EE23984205EB4601B8BFAA
:101EA80018460125A0F2EE222B46192092FBF0F2EB
:101EB8004A70FEF7ECB900BFA82800209E26002033
:101EC800A0260020C4260020183A0020283A002026
:101ED800303A0020D0530020E06900200C3A00205E
:101EE8001C4400200C2F00200D2F002078280020F3
:101EF8001A46591CD34DC8F8001012F8021B297055
:101F0800C8F800205B786B70404609F0AEFAD8F844
:101F1800003068805A1CC8F800201B782B71404696
:101F280009F0A3FAD8F80030E8805A1CC8F8002055
:101F38001B782B7201252B46FEF7A9B9C24A03F17B
:101F480008010133C8F8003013F8010C02F8010F3A
:101F58009942F6D1FEF7B6B9591C1A46C8F80010CE
:101F6800BA4912F8020B8870C8F800205B784B70E9
:101F780001252B46FEF78BB90722B6FBF2F2C2EB1E
:101F8800C201761A7EF493ABD2B2571EFFB2002A72
:101F98003EF498A9DFF8B8A201375A1CC8F8002007
:101FA80093F90010AA4B002593F902208A4200F009
:101FB8009A820135062D03F10803F5D1FEF777BBA8
:101FC8005A1CC8F800201A780E2A3EF670AB991CE5
:101FD800C8F800105D78032D3EF669AB9D480621D0
:101FE80001FB02F14218DE1C5571C8F800609D78AB
:101FF8004554191DC8F80010D9785170591DC8F8F2
:10200800001019799170991DC8F800105979D1708C
:10201800D91DC8F800109B79137101252B46FEF7CE
:1020280036B95A1CC8F800208B4A1B78537501250D
:102038002B46FEF72CB95A1CC8F800201D781F2D16
:102048003EF635AB052E7EF432AB404609F0F6F984
:10205800824B43F8250023F087FDFEF733B97F4D07
:1020680005F14006404609F000FAD8F80030A5F816
:102078008000591C1A46C8F8001012F8021B85F88F
:102088008210C8F800205B7885F883300435AE42AA
:10209800E8D1FEF717B95A1CC8F800206E4D1B7816
:1020A8002B72404609F0E1F9A883404609F0DDF9B2
:1020B8002883404609F0D9F9D8F8003068835A1CBB
:1020C800C8F800201B78EB74082E7EF6FBA8404663
:1020D80009F0CBF9E884404609F0C7F90C2E2885A9
:1020E8007EF6F0A8D8F800301A46591CC8F8001037
:1020F80012F8021BA977C8F800205B7885F8203011
:10210800404609F0B2F9102EA8847EF6DBA8D8F86C
:1021180000305A1CC8F800201B78EB72404609F0C2
:102128008DF9D8F80030E8605A1CC8F800201A78F1
:102138002A74162E7EF6C6A89A1CC8F800205B786A
:1021480085F8213001252B46FEF7A1B85A1CC8F89E
:102158000020434A1B78137001252B46FEF797B8D9
:10216800404609F082F93F4E3060404609F07DF95B
:102178007060404609F079F90125B0602B46FEF7FA
:1021880086B8394E00233360404609F057F9336862
:102198000125034333602B46FEF779B85A1CC8F86B
:1021A8000020187813283EF682AA9A1CC8F8002046
:1021B8005D782E4A002105E00131242902F10C0244
:1021C8003EF475AA167AAE42F6D1294D294A0C2654
:1021D80006FB0151DD1C91F83C1002F82010C8F8EC
:1021E800005002EB800299785170191DC8F8001050
:1021F800D8789070581DC8F800001F491B790868E6
:10220800D37025F091F9FEF75DB81C4B102E4FF0F6
:10221800000228BF10261A605A609A60DA601A74A1
:10222800002E3EF44FA8D8F8002016440132C8F812
:10223800002012F8011C03F8011BB242F6D1FEF788
:1022480041B800BFEC4100201B4900203C3A002067
:10225800CC6D0020442500201C490020E0500020BF
:10226800603A002074370020FC29002050CE020874
:1022780014CE0208643A0020A8280020902E0020DE
:102288005A1CC8F800201A780A2A7EF410AA9A1C48
:10229800C8F80020D24A59781170D91CC8F8001023
:1022A80099785170191DC8F80010DB789370FEF703
:1022B800FEB9DFF864B34FF000084FF0080A08F1E0
:1022C8000108B8F1240F1BD0C8F120020AFA02F263
:1022D8002BFA08F6A8F1200316432AFA03F31E4343
:1022E80006F0010200231343E9D05FFA88F025F0D5
:1022F80015F90028E3D04146484609F013FBDEE70C
:10230800B84B1B78DF0700F1DE800026B64FB046D9
:1023180002E00136242E0ED03146384609F011FB72
:102328000028F6D03146484609F00BFB002854D166
:1023380008F10108EDE7AD4BAD4EB3F8501020465B
:1023480009F0CCF80021204609F0C8F8A94B1A6812
:10235800530103F02001C2F340030B43C2F3800191
:1023680043EA4103C2F3C00143EA8103C2F34011C7
:1023780043EAC10102F010021143204609F0AEF809
:1023880003A90422204609F07BF8236831789A4A89
:10239800581C2060197011886429A8BF6421204640
:1023A80009F09CF8962D00F093800021204609F052
:1023B80095F82168B8F1190348BFA8F11203A3F3EF
:1023C800C4034A1C226020460B701A4604A9012542
:1023D80009F056F82B46FDF75ABF414603A809F005
:1023E800A1FAA5E72368B178844A581C20601970BF
:1023F80023681278591C21601A70FEF78EBDD9F82F
:10240800003013F48053B4EEE88A00F0B380F1EEA4
:1024180010FA12DBB4EEC98AF1EE10FA00F28D80E0
:10242800DFED777A9FED777A77EEC87AB4EEC78AD0
:10243800F1EE10FAB0EE678A7FD94FF47A71B5EEF3
:10244800408AF1EE10FA40F2DC5308BF1946FEF755
:102458001BBC22680125531923602B461070FDF719
:1024680016BF5A1C1946C8F800205F4811F8022BFD
:102478000272C8F800105B784372042A06D9FF2A52
:102488003EF41EAA22680021FDF758BF5E4909786C
:10249800994203D8022AF5D1FF2BF3D123680125ED
:1024A8005A1922601D70B9F1000F3DF40BAF574B5C
:1024B800C9F800302B46FDF7EABE404608F0D5FFC4
:1024C800534EFEF7A4BF059B43F0010305931CE799
:1024D80023680322591C21601A7023687278591CDA
:1024E80021601A7065E70AEBC509404689F80210B1
:1024F80008F0BBFFD8F800202AF835001346511C15
:10250800C8F8001013F8021B89F80310C8F8003047
:10251800537889F80430D31CC8F80030937889F8C8
:102528000630131DC8F800300136D27889F8052026
:10253800B7427FF432ADFDF7C5BEF7EE007A78EE0C
:10254800677AB6EE007AF0EE696AE7EE876A40F2DB
:10255800E932FDEEE67A17EE901AB1F5FA6FA8BFE8
:102568004FF4FA619142B8BF114689B2002B3EF48C
:102578008BAB64E7F1EE10FADFDA4FF47A71FEF70D
:1025880083BB831C00211960596019726AB1511C00
:10259800D8F800200144013B0132C8F8002012F8A5
:1025A800010C03F8010F9942F6D11A4B1B78002B46
:1025B8003EF47DA84FF0FF3524F040FB2B46FDF795
:1025C80066BE4246FEF7C1B900F07F00032828BF67
:1025D8000020012514F032FE2B46FDF758BE00BF3F
:1025E8009F28002035690020641C00206C150020FD
:1025F8008C2E0020185C0020162400200C3A0020A5
:1026080000C0884400C082442C38002091FB000898
:10261800083A00209037002090E33FF4D8F80030C3
:102628003A68591CC8F80010197851720B2E3FF4FB
:1026380069AA991CC8F800105B785370FFF762BA52
:102648000DF11409484623F019FBBDF81430AB42CC
:102658003FF46DAB264B1B68002B3FF468AB1B683F
:102668009B69002B3FF463AB28469847FFF75FBB95
:10267800D8F800302968581C1A46C8F8000012F823
:10268800020B81F83100C8F800205B7881F83230FD
:10269800FFF7FDBA404608F0E8FE7881404608F0AA
:1026A800E4FEB8814046D5F8009008F0DEFEA9F8AF
:1026B80024004046D5F8009008F0D7FE0D2EA9F862
:1026C80026007FF6FEAA404608F0CFFEF881404675
:1026D80008F0CBFE3882FFF7F4BA5A1CC8F800207D
:1026E8001B78003318BF0123F371FFF791BB00BFBC
:1026F800E06900202DE9F04FDFF808A12DED0C8BE3
:102708009AF800309FB0012B099002F0D784DFF8C7
:10271800F8B09BF80021002A41F05384072B354C70
:1027280002F051844FF00009636832489847002846
:102738006ED0B4F8A870002284F84920002F40F029
:102748009382B4F92450E16AB4F92600226BB4F9F3
:102758002830691AA16328490491821A606BE263E0
:102768000D461B1A94F84A102448236420F0F6FCFE
:102778002B6813F0005302F04384D4ED0F5AD4EDC4
:102788000E7A1F4A9BED656ADBED666A9BED677AF8
:10279800DBF8A0311268B8EEE58AD4ED105AF8EEED
:1027A800E77AF8EEE58A013377EE867A38EE268AFC
:1027B80078EE878A9342CBED657A8BED668ACBED0E
:1027C800678ACBF8A03101F06D879AF80070142F52
:1027D80003F030840023DBF8A8510593062D02F29C
:1027E800EC84DFE815F05B1927198A140F1B781B96
:1027F800861A1F1AE45300204C4900201C5400205C
:102808001C5C00205C3A0020701C0020DDF814904D
:102818009AF80080B8F1070F00F0DD829BF8B83114
:102828000B93002B40F0E382CD4B5B79002B40F0FB
:10283800168201239AF800208BF8B831072A02F093
:102848007B8500230D93C74BDBED709A93ED007ADF
:10285800C54AC64B12680692F7EE007A37EEE98A47
:10286800C34A079228EE078AC24AC34FDBED6F8A34
:10287800DFF87893DFEDC1AA9FEDC19A9FEDC1BA49
:10288800DFEDC1CA9FEDC1AADFEDC1BADFF86083F1
:10289800C04E0A93B4EEE78A0024F1EE10FA0892CB
:1028A80088BFB0EE678A059325460497BA4B234440
:1028B800D3ED007AB94BF5EE407A2344F1EE10FAE5
:1028C80093ED00CA17D0B64B234493ED007A7CEE03
:1028D800476AB0EEE66AF4EEC67AF1EE10FA08D569
:1028E800F5EEC06AF1EE10FACCBF37EE87CA37EEC4
:1028F80067CA83ED00CA079B1F88BB0700F07F8269
:10290800022D05F0E9830699A64B91F8322007EECF
:10291800102A91F831202344D3ED006A5342B8EECF
:10292800C77A07EE903A27EE267AF8EEE77AB4EE01
:10293800E77AF1EE10FA0AD407EE902AF8EE677AF1
:10294800F4EEC77AF1EE10FA88BFF0EE477A964BAC
:102958000C93964A03EB450332F91510B3F90A3084
:10296800C81A07EE100AB8EEC77AFF07E7EE497AE9
:1029780040F1B8828E4F97ED00CA27EE8CCA9BF8BB
:10298800D071E7B18A4FDBF8D40197ED00CA894FBF
:102998005B1A07EE903A099B39682CEE09CAF8EEE3
:1029A800E77A1F1A8F422CEE27CA01F3DD82F7EE71
:1029B800007AF4EEE79AF1EE10FA01F1A1827E4B6B
:1029C8002344D3ED007A059BD3ED01DA049B68EE2E
:1029D800A77A3CEE6DDA67EE8D7AC3ED007A089B34
:1029E800D9ED006A93ED007A744BD6ED007A26EEA5
:1029F800877A234467EE086A93ED007A26EE877A91
:102A0800F0EE676AE7EE0D6AB0EE667A9BED706AE3
:102A1800F7EE006AB4EEE66AF1EE10FAACBF0123F5
:102A2800002343B1F0EEE77AF0EEC76AF4EEE76A06
:102A3800F1EE10FA01D586ED007A022D05F000833B
:102A48005F4A604B52F825001B68B0EE6D0A984744
:102A58005D4A5E4B52F825001B689847069B93F821
:102A68003A30632B04D8079B1B88002B01F08E8219
:102A7800F0EE6C7A564B99ED007A37EEC00A234493
:102A8800D3ED007A83ED000A069B30EE670A93F8CF
:102A9800482080EE07CADAB1F7EE007AF4EEE79A3A
:102AA800F1EE10FA14DB4B4BD3ED007AB0EECC7A92
:102AB800B4EEE77AF1EE10FA0ADD474BD3ED007A6F
:102AC800B0EECDDAB4EEE7DAF1EE10FA01F377837F
:102AD800424B9BF8E0212344D3ED007A68EEA77AB5
:102AE80027EE8CCA88ED00CA32B9049BC6ED00CA2D
:102AF800C3ED00CAC8ED00CA049B04330493059BC8
:102B0800043404330C2C05F1010508F1040806F11E
:102B1800040605937FF4CAAE9AF80030072B02F03A
:102B28006083012B02F0F883002309932C4B049354
:102B38001A460D4B12681B680692114693F82F200F
:102B480011F480530A9300F04F82264B08931B78A8
:102B5800DFF8A08013F0010F234B05934CE000BF72
:102B6800D0530020D0670020A8280020085C00204F
:102B7800DC69002000000020BC37002000009642DD
:102B8800CDCCCC3DAE47813F000000000000C842DC
:102B980000003443C8370020C4670020741D00209B
:102BA800341E0020DC1D0020183A0020D03B0020F5
:102BB800AC670020D4670020806700208C67002065
:102BC800003C0020FC3B0020643C0020603C0020CE
:102BD800481E0020E4670020E06700209867002076
:102BE8004C490020356900201C4900207C670020E2
:102BF800D4370020D04F0020198BA94B98ED037AC9
:102C0800DB8808BFABF8E811C81A07EE900AF8EE9F
:102C1800E77AB4EEE77AF1EE10FA42F2FD82CC18C8
:102C280006EE904AF8EEE66AB4EEE67AF1EE10FAAD
:102C380081F20D85BBF8E831984284F20380994B04
:102C48009949D3ED003A91ED004A984B8BED7B4AB8
:102C5800CBED7C3AD3ED006ADFED957AE0E1954B58
:102C68001B78013BDBB2E5E59349944B49780A931D
:102C780004911B68924E9AF80080B6F906004FF44A
:102C88007A71B1FBF3F3C3EB431503EB8503DD0066
:102C9800ADB2AF4203F0B482E16FB4F924E0236E21
:102CA8004A1C07EE90EA7344012AE2672366F8EEAD
:102CB800E77A03F0AF82D4ED1B5AD4ED1D6A07EE14
:102CC800102A37EEE56AB8EEC75A012F86EE057A64
:102CD80037EE257A77EEC77A84ED1C7AE6EE276A16
:102CE80084ED1B7AF0EE667AC4ED1E6AC4ED1D6AA7
:102CF80004F00780D4F89010B4F926E0636E4A1CFB
:102D080007EE90EA7344012AC4F890206366F8EE4F
:102D1800E77A03F09782D4ED205AD4ED226A07EEC1
:102D2800102A37EEE56AB8EEC75A012F86EE057A03
:102D380037EE257A77EEC77A84ED217AE6EE276AB0
:102D480084ED207AF0EE667AC4ED236AC4ED226A37
:102D580004F00780D4F8A410B4F928E0A36E4A1C44
:102D680007EE90EA7344012AC4F8A420A366F8EE9B
:102D7800E77A03F08082D4ED255AD4ED276A07EE6E
:102D8800102A37EEE56AB8EEC75A012F86EE057AA3
:102D980037EE257A77EEC77A84ED267AE6EE276A4B
:102DA80084ED257AF0EE667AC4ED286AC4ED276AC8
:102DB80003F0CA87F080B4F8A8309AF80080013B85
:102DC800A4F8A8300A990023B8F1070F4B608B606C
:102DD800CB607FF423AD0BF0B1FD394E9BF8B831D1
:102DE8000B93A0EB09003080002B3FF41DAD013B95
:102DF8008BF8B8311FB0BDEC0C8BBDE8F08F9BF899
:102E0800D03163B1022D05F056812E4B0C932E4A1A
:102E180003EB450332F91510B3F90A30B2E52B4B31
:102E2800234493ED000A059BD3ED01DA049B28EEB9
:102E3800800A3CEE6DDA022D20EE0D0A83ED000AC1
:102E48007FF4CDAD224A234B10681B689847089B36
:102E580099ED007AD3ED006A1F4BD6ED007A1A7807
:102E68001E4B83ED020A1E4B26EE877A234427EE7B
:102E7800087A93ED006A27EE067AF0EE676AE7EEC5
:102E88000D6A012AB0EE667A02D0192A7FF4BEAD27
:102E9800B4EEEADAF1EE10FACCBF01230023C0E564
:102EA800D8410020D0410020FC390020E841002012
:102EB800000000000C3A0020D0530020085C0020DD
:102EC80024380020183A0020D03B002080670020DA
:102ED800C4400020D840002078670020BC3700207C
:102EE8008C670020DBED5E6A9BED5F7AB2F900E04B
:102EF800B2F90270B4EEE67AF1EE10FA8EEAEE70EC
:102F080087EAE77C4CBFB7EE007AF7EE006AA0EBE1
:102F1800EE70ACEBE77C4CBF77EE665A76EEC75A9C
:102F2800604541F30E81BEF1000FD6BFCEF100001F
:102F380007EE10EA07EE100A274FB8EEC77A3F7877
:102F480027EE097A002F01F00C81244F97ED005AE3
:102F5800B5EEC05AF1EE10FA42F3C380204FD7ED18
:102F6800004AF5EEC04AF1EE10FA42F3BA8034EEA8
:102F7800C77AB7EE006AC7EE246A75EEC65AF4EE51
:102F8800C66A65EE8A5AF1EE10FA85EE857A88BF30
:102F9800F0EE466AF5EEC06AF1EE10FA37EE067A00
:102FA800B8BFF0EE6C6A66EE876AF4EEC66AF1EEB8
:102FB80010FA88BFF0EE466AF5EEC06AF1EE10FA34
:102FC800B8BFF0EE6C6A074F97ED007A67EE877A24
:102FD800A7EEA6CAD3E400BFB8670020B4670020F4
:102FE800BC670020B0670020E24B05935B8BDFF8DD
:102FF800C083E14998ED037A91ED004A07EE903AD3
:10300800DE4B8BED7B4AD3ED003ADD4BCBED7C3AC2
:10301800F8EEE77AD3ED006ADA4B089377EE677A31
:10302800C7EEA62AD849D94B91ED008AD849DFEDD9
:10303800D96A91ED005AD8499FEDD86AD1ED005A66
:1030480093ED007AF7EE007AF4EEE72A38EE058A77
:10305800F1EE10FA88BFF0EE672A38EE258AF4EE12
:10306800E62AF1EE10FA28EE066AB8BFF0EE662AF4
:10307800F1EE476A34EE635AB4EEE66AF1EE10FAFE
:10308800CBED7D2A8BED7F5A00F16B85B4EEC76AD4
:10309800F1EE10FA88BFB0EE476ABB4BDFEDBF7A9E
:1030A800D3ED018ABA4BD3ED014ABB4B78EEA48A23
:1030B800D3ED015A78EEA58A68EEA77AF4EEE76AAE
:1030C800F1EE10FA08DCB4EEE77AF1EE10FA8CBFF4
:1030D800F0EE676AF0EE476AAB4BDFEDB07A93ED3E
:1030E800029AAB4BD3ED025AAD4B39EE259A93EDCC
:1030F800007A69EE277AF1EE475AF4EEE57AF1EEB6
:1031080010FA08D4F4EEC77AF1EE10FA8CBFF0EE9C
:10311800475AF0EE675A002A41F04F83F7EE007ADB
:10312800A04B5A789BF80032002A9F4ABFEE003A1B
:10313800B7EE007A127814BFB0EE472AB0EE432AF1
:10314800002B14BFF0EE434AF0EE474A002A03F082
:103158000381F4EEC77AF1EE10FA65EE825A934BCA
:1031680041F3E68393ED027A93ED011AD3ED031A46
:103178009FED882A26EE877A27EEA43AA1EE067AF2
:10318800A1EEA57A27EE037AB4EEC27AF1EE10FA30
:10319800B4BFF0EE427AF0EE477A8DED127A88BF2E
:1031A800B0EE427A012A00F0BE81D3ED064AD3ED93
:1031B800051A93ED072A66EEA44AE1EE864AE2EE86
:1031C800254A64EE834AF4EEC74AF1EE10FAF4EEAB
:1031D800E74A8CBFB0EE472AB0EE642AF1EE10FA47
:1031E80098BFB0EE427AA8BFF0EE647A022ACDED1D
:1031F800134A00F09881D3ED0A4AD3ED091A93EDEA
:103208000B2A66EEA44AE1EE864AE2EE254A64EE0F
:10321800834AF4EEC74AF1EE10FAF4EEE74A8CBF9F
:10322800B0EE472AB0EE642AF1EE10FA98BFB0EE7D
:10323800427AA8BFF0EE647A032ACDED144A00F072
:103248007281D3ED0E4AD3ED0D1A93ED0F2A66EE77
:10325800A44AE1EE864AE2EE254A64EE834AF4EE99
:10326800C74AF1EE10FAF4EEE74A8CBFB0EE472AEF
:10327800B0EE642AF1EE10FA98BFB0EE427AA8BF19
:10328800F0EE647A042ACDED154A00F04C81D3EDB6
:10329800124AD3ED111A93ED132A66EEA44AE1EE11
:1032A800864AE2EE254A64EE834AB4EEE47AF1EE09
:1032B80010FAF4EEE47A8CBFB0EE642AB0EE472A36
:1032C800F1EE10FA58BFB0EE427AB8BFF0EE647A69
:1032D800052ACDED164A00F02681D3ED164AD3ED26
:1032E800151A93ED172A66EEA44AE6EE214AE5EE92
:1032F800824A64EE834AF4EEC74AF1EE10FAF4EE1D
:10330800E74A8CBFB0EE472AB0EE642AF1EE10FA15
:1033180098BFB0EE427AA8BFF0EE647A062ACDEDE7
:10332800174A00F00081D3ED1A4AD3ED191A93ED2C
:103338001B2A66EEA44AE6EE214AE5EE824A64EECE
:10334800834AF4EEC74AF1EE10FAF4EEE74A8CBF6E
:10335800B0EE472AB0EE642AF1EE10FA98BFB0EE4C
:10336800427AA8BFF0EE647A072ACDED184A00F039
:10337800DA801FE01C490020FC390020803800203A
:10338800E041002035690020BC370020E8670020B4
:10339800C837002000000000D43700206F12833A9D
:1033A800EC670020603A00202C38002010410020F3
:1033B800D04F0020D3ED1E4AD3ED1D1A93ED1F2ADE
:1033C80066EEA44AE6EE214AE5EE824A64EE834AB6
:1033D800F4EEC74AF1EE10FAF4EEE74A8CBFB0EE0D
:1033E800472AB0EE642AF1EE10FA98BFB0EE427A9E
:1033F800A8BFF0EE647A082ACDED194A00F0938050
:10340800D3ED224AD3ED211A93ED232A66EEA44A7E
:10341800E1EE864AE2EE254A64EE834AF4EEC74AB4
:10342800F1EE10FAF4EEE74A8CBFB0EE472AB0EEA0
:10343800642AF1EE10FAD8BFB0EE427AA8BFF0EED7
:10344800647A092ACDED1A4A6DD0D3ED264AD3ED18
:10345800251A93ED272A66EEA44AE1EE864AE2EEA3
:10346800254A64EE834AB4EEE47AF1EE10FAF4EEFB
:10347800E74A8CBFB0EE642AB0EE472AF1EE10FAA4
:1034880098BFB0EE427AA8BFF0EE647A0A2ACDED72
:103498001B4A48D0D3ED2A4AD3ED291A93ED2B2A9B
:1034A80066EEA44AE6EE214AE5EE824A64EE834AD5
:1034B800B4EEE47AF1EE10FAF4EEE47A8CBFB0EEF2
:1034C800642AB0EE472AF1EE10FACDED1C4A58BF37
:1034D800B0EE427AA8BFF0EE674A0B2A03F0AE833B
:1034E800D3ED2E7AD3ED2D1A93ED2F2A66EEA77A17
:1034F800E1EE867AE2EE257A67EE837AB4EEE77A31
:10350800F1EE10FAF4EEE74A8CBFF0EE676AF0EEDF
:10351800476AF1EE10FACDED1D7AA8BFB0EE667AD3
:10352800A8BFF0EE647A77EEC77AF7EE006AF4EE99
:10353800E67AF1EE10FACBED707A43F3698386EE02
:10354800A77A012ADDED127A67EE877ACDED127A35
:1035580055D0DDED137A67EE877A022ACDED137A1E
:103568004DD0DDED147A67EE877A032ACDED147A13
:1035780045D0DDED157A67EE877A042ACDED157A08
:103588003DD0DDED167A67EE877A052ACDED167AFD
:1035980035D0DDED177A67EE877A062ACDED177AF2
:1035A8002DD0DDED187A67EE877A072ACDED187AE7
:1035B80025D0DDED197A67EE877A082ACDED197ADC
:1035C8001DD0DDED1A7A67EE877A092ACDED1A7AD1
:1035D80015D0DDED1B7A67EE877A0A2ACDED1B7AC6
:1035E8000DD0DDED1C7A67EE877A0B2ACDED1C7ABB
:1035F80005D0DDED1D7A27EE877A8DED1D7AE14B3A
:10360800196811F0805100F096854FF07C53CBF883
:10361800F431002A02F09A86089BDB4E1F78DB4CB7
:10362800DB48DC4D96ED006A9BF8F831059EE4789E
:103638000078B5F90650DBED7D6A768B07F0010C52
:10364800069F07F0100E07F48007002B40F09C82BD
:10365800BEF1000F00F01686BCF1000F43F0308277
:10366800002C43F01783CC4BDDED127A93ED007AF2
:10367800CA48E7EE267ABDEEC47A17EE101AB0EE05
:10368800637AA5EE277A0D46F0EE477AFDEEE77AE3
:10369800BDEEE37A17EE906A17EE104AB142A8BF62
:1036A8003546B442C8BF254607EE905AF8EEE77A89
:1036B800012AC0ED007A00F04D8193ED047ADDED2A
:1036C800137AE7EE267AB0EE637AA5EE277AFDEE56
:1036D800C77A17EE906A17EE905A8E42A8BF0D4629
:1036E800A642B8BF254607EE905AF8EEE77A022AB6
:1036F800C0ED017A00F02E8193ED087ADDED147AA1
:10370800E7EE267AB0EE637AA5EE277AFDEEC77A61
:1037180017EE906A17EE905A8E42A8BF0D46A64241
:10372800B8BF254607EE905AF8EEE77A032AC0EDAF
:10373800027A00F00F8193ED0C7ADDED157AE7EE51
:10374800267AB0EE637AA5EE277AFDEEC77A17EEF1
:10375800906A17EE905A8E42A8BF0D46A642B8BF8F
:10376800254607EE905AF8EEE77A042AC0ED037A68
:1037780000F0F08093ED107ADDED167AE7EE267A08
:10378800B0EE637AA5EE277AFDEEC77A17EE906A57
:1037980017EE905A8E42A8BF0D46A642B8BF2546DE
:1037A80007EE905AF8EEE77A052AC0ED047A00F0A1
:1037B800D18093ED147ADDED177AE7EE267AB0EE34
:1037C800637AA5EE277AFDEEC77A17EE906A17EEB0
:1037D800905A8E42A8BF0D46A642B8BF254607EEAE
:1037E800905AF8EEE77A062AC0ED057A00F0B28022
:1037F80093ED187ADDED187AE7EE267AB0EE637A63
:10380800A5EE277AFDEEC77A17EE906A17EE905A62
:103818008E42A8BF0D46A642B8BF254607EE905A6D
:10382800F8EEE77A072AC0ED067A00F0938093ED68
:103838001C7ADDED197AE7EE267AB0EE637AA5EE0A
:10384800277AFDEEC77A17EE906A17EE905A8E42E5
:10385800A8BF0D46A642B8BF254607EE905AF8EE17
:10386800E77A082AC0ED077A74D093ED207ADDED67
:103878001A7AE7EE267AB0EE637AA5EE277AFDEE9D
:10388800C77A17EE906A17EE905A8E42A8BF0D4677
:10389800A642B8BF254607EE905AF8EEE77A092AFD
:1038A800C0ED087A56D093ED247ADDED1B7AE7EE69
:1038B800267AB0EE637AA5EE277AFDEEC77A17EE80
:1038C800906A17EE905A8E42A8BF0D46A642B8BF1E
:1038D800254607EE905AF8EEE77A0A2AC0ED097AEB
:1038E80038D093ED287ADDED1C7AE7EE267AB0EE33
:1038F800637AA5EE277AFDEEC77A17EE906A17EE7F
:10390800905A8E42A8BF0D46A642B8BF254607EE7C
:10391800905AF8EEE77A0B2AC0ED0A7A1AD093ED9E
:103928002C7ADDED1D7AE6EE877AE5EE273AFDEE94
:10393800E37A17EE903A9942A8BF19469C42D8BF3D
:103948000C4607EE904AF8EEE77AC0ED0B7A002AAB
:1039580000F09F8292001249104826F021FF114B77
:103968001B68002B00F09A820F4B1B78192B22D86A
:1039780001220E4902FA03F31940002943F0148288
:1039880016E000BFF0390020DC4000206469002008
:1039980044440020B4690020104100204038002031
:1039A800E04000207467002078670020324130032F
:1039B800190302F131836D4D6D4E069B9B061BD595
:1039C800F37AFF2B04D06B4A12789A4202F21F83D3
:1039D800B6F90870F37D2F80FF2B04D0654A127862
:1039E8009A4202F20F83B6F914406C80082023F043
:1039F80095FD002841F0F887B6F90600B5F900E012
:103A0800B5F90270B6F91210B6F91E20B5F90440DE
:103A1800B6F90430B5F906C07045A8BF7046B9427A
:103A2800A8BF3946A242A8BF22469E45A8BF034662
:103A38002B80B6F91030B5F90800BB42C8BF19464B
:103A4800B6F92A306980B6F91C10B6F934706345A6
:103A5800A8BF6346A142CCBF0C461446B6F936202F
:103A6800AC80B6F92840B5F90A108242A8BF0246D0
:103A7800A445ACBF9C46A446B6F94230B5F90C4003
:103A8800A5F806C08B42A8BF0B468742CCBF384674
:103A98001046B6F94E202881B6F94000B5F90E70E7
:103AA800A242A8BF22468842C8BF0346B6F95A00B8
:103AB800B6F94C106B81B842B6F958302E4EA8BFF3
:103AC80038469F42A8BF0346A142D8BF1146A981E4
:103AD800EB81B38923B3294FDFF8A890DFF89080F2
:103AE80007F11004B7F9023000EE103A4846B8EE74
:103AF800C00A06F033FE26F0C7FFB8F90430B8F95B
:103B0800062000B2984209F12C0908F10C0803DBE1
:103B180082421346A8BF034627F8023FA742E1D1D5
:103B2800174B1B78013B182B00F28A86DFE813F04D
:103B3800760688068806480F880688068806B11221
:103B480088068806880688068806A21288068806D7
:103B5800880688069112480FBE1288068806A212A7
:103B68007606B0EE666AFFF798BA00BF30380020D4
:103B780050680020F86300201C4200202E380020E6
:103B88007867002030650020BEF1000F40F0FA840D
:103B9800D44BDDED127A93ED007A002841F0FE83D4
:103BA800E7EE267AD048B1EE455AB0EE447AA5EE53
:103BB800277AF0EE477ABDEEC47A002C43F01283E0
:103BC800FDEEE77A17EE104A17EE906AFDEEE37AFB
:103BD800B44217EE901A17EE105AA8BF3546B142F4
:103BE800C8BF0D4607EE905AF8EEE77A012AC0EDF5
:103BF800007A00F04A8193ED047ADDED137AE7EE5E
:103C0800267AB0EE447AA5EE277AFDEEC77A17EE4B
:103C1800906A17EE905AA642A8BF25468E42B8BFB2
:103C28000D4607EE905AF8EEE77A022AC0ED017ABF
:103C380000F02B8193ED087ADDED147AE7EE267A11
:103C4800B0EE447AA5EE277AFDEEC77A17EE906AB1
:103C580017EE905AA642A8BF25468E42B8BF0D4619
:103C680007EE905AF8EEE77A032AC0ED027A00F0E0
:103C78000C8193ED0C7ADDED157AE7EE267AB0EE3D
:103C8800447AA5EE277AFDEEC77A17EE906A17EE0A
:103C9800905AA642A8BF25468E42B8BF0D4607EEE9
:103CA800905AF8EEE77A042AC0ED037A00F0ED8026
:103CB80093ED107ADDED167AE7EE267AB0EE447AC7
:103CC800A5EE277AFDEEC77A17EE906A17EE905A9E
:103CD800A642A8BF25468E42B8BF0D4607EE905AA9
:103CE800F8EEE77A052AC0ED047A00F0CE8093ED6D
:103CF800147ADDED177AE7EE267AB0EE447AA5EE6F
:103D0800277AFDEEC77A17EE906A17EE905AA64208
:103D1800A8BF25468E42B8BF0D4607EE905AF8EE6A
:103D2800E77A062AC0ED057A00F0AF8093ED187A9D
:103D3800DDED187AE7EE267AB0EE447AA5EE277A1A
:103D4800FDEEC77A17EE906A17EE905AA642A8BF02
:103D580025468E42B8BF0D4607EE905AF8EEE77A30
:103D6800072AC0ED067A00F0908093ED1C7ADDED0D
:103D7800197AE7EE267AB0EE447AA5EE277AFDEEB8
:103D8800C77A17EE906A17EE905AA642A8BF254642
:103D98008E42B8BF0D4607EE905AF8EEE77A082A29
:103DA800C0ED077A71D093ED207ADDED1A7AE7EE4F
:103DB800267AB0EE447AA5EE277AFDEEC77A17EE9A
:103DC800906A17EE905AA642A8BF25468E42B8BF01
:103DD8000D4607EE905AF8EEE77A092AC0ED087A00
:103DE80053D093ED247ADDED1B7AE7EE267AB0EE18
:103DF800447AA5EE277AFDEEC77A17EE906A17EE99
:103E0800905AA642A8BF25468E42B8BF0D4607EE77
:103E1800905AF8EEE77A0A2AC0ED097A35D093ED80
:103E2800287ADDED1C7AE7EE267AB0EE447AA5EE24
:103E3800277AFDEEC77A17EE906A17EE905AA642D7
:103E4800A8BF25468E42B8BF0D4607EE905AF8EE39
:103E5800E77A0B2AC0ED0A7A17D093ED2C7ADDEDBC
:103E68001D7AE6EE877AA5EE274AFDEEC47A17EEAC
:103E7800903A9C42A8BF1C469942D8BF214607EEFB
:103E8800901AF8EEE77AC0ED0B7ABCF1000F3FF418
:103E98005EAD164B1B68002B7FF466AD144B1B7888
:103EA80093B1144B187860B10F4D134E0024E0B253
:103EB8003368B5EC010A98470E4B187801348442F0
:103EC800F5DB0E4B1B6898479AF80030072B01F07A
:103ED8000C8101238BF800311FB0BDEC0C8BBDE8C1
:103EE800F08F00BF10410020403800207467002088
:103EF800AC4800202C3800203844002040440020E2
:103F08000C9BB2F90070B3F90A30C849F81A09686D
:103F180080EAE073A3EBE0738B42BEF650ADB2F9D2
:103F280002300C9AB2F90C209A1A82EAE273A3EBD7
:103F3800E27399427EF743AD0A99BD4BD1ED017A00
:103F480093ED007AF0EEE77AF4EEC77AF1EE10FA24
:103F58007EF535ADD1ED027AF0EEE77AB4EEE77A88
:103F6800F1EE10FA7EF72BADB24B1A8800238BF8CE
:103F7800D031002A40F08C83AF4AB04B11781868D2
:103F880081F001010BF09EFBFEF719BDAC4BAD4A69
:103F98002344D3ED006A92ED007AAB4B26EE877A84
:103FA800F7EE006AB4EEE67AD3ED007AF1EE10FA95
:103FB80088BFB0EE667A27EE277A67EE0C7AFEF7AE
:103FC80059BD072B02F01F860025A04B04931B68E0
:103FD8009F4C5B0501F196819E4B1B78002B40F0AE
:103FE80004819D4B05939BF8126126B19B4B1B885E
:103FF8009F0742F09683059A9BF81831D27F002BD1
:1040080041F0218105998F7F002F00F05386022F00
:1040180002F09581032F01F0C98491494988023241
:10402800D2B2002B02F07E81002902F07B818D48FC
:104038000768B1FBF7F10FB2ABF84871002A03F03B
:10404800038607EE907AF8EEE77AF7EE006A86EED6
:10405800A77ADFF82C82012ADBED576AD8ED007ABF
:1040680077EEE67A67EE877ACBED537A21D0D8EDF2
:10407800017ADBED586A77EEE67A022A67EE877AEC
:10408800CBED547A15D0D8ED027ADBED596A77EE8C
:10409800E67A032A67EE877ACBED557A09D0D8ED10
:1040A800037ADBED5A6A77EEE67A67EE877ACBED2C
:1040B800567A9AF80010092903F0EF85002F40F38B
:1040C800008692B3DBED577A9BED537A77EE877AC9
:1040D800012ACBED577AC8ED007A21D0DBED587A6A
:1040E8009BED547A77EE877A022ACBED587AC8EDA1
:1040F800017A15D0DBED597A9BED557A77EE877A00
:10410800032ACBED597AC8ED027A09D0DBED5A7A49
:104118009BED567A77EE877ACBED5A7AC8ED037A1B
:10412800013A022AB8BF0222D2B2002B0CBF1346B2
:10413800022300F0C7BD069B58023FF566AAFFF7A9
:1041480068BA002FD6BF784207EE107A07EE100A39
:10415800454FB8EEC77A3F7827EE097A002F7EF4EC
:10416800F4AE424FD7ED006AF4EECB6AF1EE10FAE6
:1041780041F14D80B7EE005A35EE665A9FED3C6A24
:104188003C4F3BEEC77A25EE065A97ED006AE7EEFC
:10419800056A26EE867AB5EEC07AF1EE10FA40F29C
:1041A800A087CAEE076AB7EE006A35EEC67AF0EE67
:1041B800465AE7EE265AF0EE656AFEF7F6BE012388
:1041C8000999CBF8D411022A8BF8D0317EF480AC4F
:1041D800184A1288002A43F04385174A174B11786A
:1041E80018680BF06FFAFEF773BC1B4A224B059256
:1041F8001146B3F906204B8B9A423FF7F4AE1F4B9A
:104208001B78012B02F07F80192B02F07C800E2B8B
:104218003FF4E9AE082B3FF4E6AEDFF864800023F4
:10422800C8F80830CBF80C31DDE600BFD8670020AD
:10423800DC670020985300209A5300209C530020EC
:10424800E81D0020A8670020A46700204C49002032
:10425800E4530020861A00201C490020DC69002055
:10426800F8630020443A0020B8670020C0670020A7
:10427800610BB63BB4670020B4690020603A0020A7
:10428800D04F0020BD4BDDED127A93ED007A002C63
:1042980042F09E82E7EE267AB948BDEEC47A17EE60
:1042A800101AB0EE637AA5EE277A0D46F0EE477A3B
:1042B800FDEEE77ABDEEE37A17EE906A17EE104A44
:1042C800B142A8BF3546B442C8BF254607EE905A4A
:1042D800F8EEE77A012AC0ED007A3FF4D6AD93ED07
:1042E800047ADDED137AE7EE267AB0EE637AA5EE6E
:1042F800277AFDEEC77A17EE906A17EE905A8E422B
:10430800A8BF0D46A642B8BF254607EE905AF8EE5C
:10431800E77A022AC0ED017A3FF4B7AD93ED087A47
:10432800DDED147AE7EE267AB0EE637AA5EE277A09
:10433800FDEEC77A17EE906A17EE905A8E42A8BF24
:104348000D46A642B8BF254607EE905AF8EEE77A22
:10435800032AC0ED027A3FF498AD93ED0C7ADDEDB7
:10436800157AE7EE267AB0EE637AA5EE277AFDEEA7
:10437800C77A17EE906A17EE905A8E42A8BF0D467C
:10438800A642B8BF254607EE905AF8EEE77A042A07
:10439800C0ED037A3FF479AD93ED107ADDED167A2E
:1043A800E7EE267AB0EE637AA5EE277AFDEEC77AB5
:1043B80017EE906A17EE905A8E42A8BF0D46A64295
:1043C800B8BF254607EE905AF8EEE77A052AC0ED01
:1043D800047A3FF45AAD93ED147ADDED177AE7EEDF
:1043E800267AB0EE637AA5EE277AFDEEC77A17EE45
:1043F800906A17EE905A8E42A8BF0D46A642B8BFE3
:10440800254607EE905AF8EEE77A062AC0ED057AB7
:104418003FF43BAD93ED187ADDED187AE7EE267A96
:10442800B0EE637AA5EE277AFDEEC77A17EE906AAA
:1044380017EE905A8E42A8BF0D46A642B8BF254631
:1044480007EE905AF8EEE77A072AC0ED067A3FF4AD
:104458001CAD93ED1C7ADDED197AE7EE267AB0EE05
:10446800637AA5EE277AFDEEC77A17EE906A17EE03
:10447800905A8E42A8BF0D46A642B8BF254607EE01
:10448800905AF8EEE77A082AC0ED077A3FF4FDACB7
:1044980093ED207ADDED1A7AE7EE267AB0EE637AAC
:1044A800A5EE277AFDEEC77A17EE906A17EE905AB6
:1044B8008E42A8BF0D46A642B8BF254607EE905AC1
:1044C800F8EEE77A092AC0ED087A3FF4DEAC93EDFE
:1044D800247ADDED1B7AE7EE267AB0EE637AA5EE54
:1044E800277AFDEEC77A17EE906A17EE905A8E4239
:1044F800A8BF0D46A642B8BF254607EE905AF8EE6B
:10450800E77A0A2AC0ED097A3FF4BFAC93ED287A1E
:10451800DDED1C7AE7EE267AB0EE637AA5EE277A0F
:10452800FDEEC77A17EE906A17EE905A8E42A8BF32
:104538000D46A642B8BF254607EE905AF8EEE77A30
:104548000B2AC0ED0A7A3FF4A0AC93ED2C7ADDED8E
:104558001D7AE6EE877AE5EE273AFDEEE37A17EE66
:10456800903A9942A8BF19469C42D8BF0C4607EE1C
:10457800904AF8EEE77AC0ED0B7A86E41041002005
:1045880040380020BCF1000F42F0E882002841F0DA
:104598009781FDEEE37A0DF1480E17EE906AFDEE75
:1045A800C47A0EEB820317EE907AFDEEC67A84F099
:1045B8000101CE48DFF87093CDF834B017EE905A69
:1045C800CDF83880B1EE455A4FFA84FC0C929846E3
:1045D8008B46034693ED007AFEEC017AE6EE877A85
:1045E8003A461030B0EE447AA5EE277AFDEEC77A47
:1045F80017EE903A9F42A8BF1A469D42CCBF0021B1
:1046080004F00101002914BF114629469E42CCBF7F
:1046180000230BF0010307EE901A002B14BF13467A
:104628003346B8EEE77A07EE903AF8EEE77ABCF14F
:10463800000F18BFF0EE477AC645E9EC017AC8D1F9
:104648000C9ADDF834B0DDF83880FFF780B907EE52
:10465800901AF8EEE77AA648A64CD0ED003A94ED09
:10466800004AA5488BED7B4A06EE903A77EE677ACA
:10467800BCEEC77AF8EEE66A17EE103A77EEE67AFD
:10468800CBED7C3AABF8E831D0ED006AFEF7C8BC58
:104698009A494A69002A3EF492A90A6813604B7441
:1046A800FEF78DB907EE103A9AF80030944ECBF821
:1046B800A071B8EEC77AF7EE006A132B86EE879AD8
:1046C800B6F90400BBF8A45194ED080A01F0FD8482
:1046D8008C4B8D4A93ED001A93ED093A93ED162A07
:1046E80093ED1F6AD3ED0B1A93ED144AD3ED015ADB
:1046F800D3ED0A3A93ED0C7A93ED155AD3ED172AB8
:10470800D3ED206AD3ED044AD3ED030A69EE277A84
:1047180069EE288A29EE088AA7EE813A02EB850716
:104728000021A2EE286ACBF89411CBF89811A8EED4
:10473800214AE7EEA53AA8EE075A93ED1A7AD3ED87
:104748000F5A93ED021AD3ED0E1A87ED003AE2EEF6
:10475800A86A64EEC34A27EE467A93ED0D2AD3ED94
:10476800192A87ED204AE3EE603A65EEC45A93EDC4
:10477800183AC3ED093AE7EE814AF0EE477AA1EE1E
:10478800C45AE8EE025AE2EEC66AE3EE287AC3EDAE
:104798000A4A83ED145AC3ED155A87ED406AC3EDF2
:1047A8001F6AC3ED207ACBF89C116B1C03F01F0322
:1047B800ABF8A431B080FEF708B8544B1A79002A38
:1047C8003EF4ACAC524A1278002A3EF4A7AC1B78EF
:1047D8009FED502A07EE103A4F4B07EE902A1B88A0
:1047E800F8EEE77A04EE903AB8EE477AF8EE644AC3
:1047F80027EE277AB7EE003AC7EE247AF4EEC27AAB
:10480800F1EE10FA88BFF0EE427AF4EEC37AF1EED8
:1048180010FAB8BFF0EE437AFEF782BCB37B002BE8
:1048280043F0A380089B1B7813F0010343F09D809D
:104838003A4A1268002A03F07E83136001230B931F
:10484800049B1B689F0634D4354A1278052A30D059
:10485800DC027FF523ABF57B112D3FF61FAB314B07
:10486800DDF82C801C4633F9153000EE103A40462E
:10487800B8EEC00A6F1C05F10E0612F085FC43461F
:10488800FFB25D1BF6B2A04600E027467C1C7819F3
:10489800122FE4B2C0B23FF401AB38F9173000EE82
:1048A800103AB8EEC00A12F06FFCB442EDD1FFF72F
:1048B800F5BA0B9A13460233541CDBB21046E4B225
:1048C8000B93B5F9003000EE103AB8EEC00A12F0BA
:1048D8005BFCB5F9023000EE103A2046B8EEC00A8B
:1048E80012F052FC049B1B68B2E700BF1041002085
:1048F800D0410020FC390020E8410020A0530020CE
:1049080024380020DC5E0020405C0020586900202C
:10491800CD4F0020713DAA3F844F00202C4200203B
:1049280078670020B46900204038002000000000AB
:1049380093ED027A93ED012AD3ED037A1FED053A40
:1049480026EE877AA6EE027AA7EEA57A27EE247AD3
:10495800B4EEC37AF1EE10FAB4BFF0EE437AF0EE9B
:10496800477A8DED127A88BFB0EE437A012A3EF479
:10497800DAAD93ED063AD3ED051A93ED072A26EE44
:10498800833AA6EE213AA2EE253A23EE243AB4EE73
:10499800C73AF1EE10FAB4EEE73A8CBFB0EE472A08
:1049A800B0EE432AF1EE10FA98BFB0EE427AA8BFF3
:1049B800F0EE437A022A8DED133A3EF4B4AD93ED4E
:1049C8000A3AD3ED091A93ED0B2A26EE833AA6EE9E
:1049D800213AA2EE253A23EE243AB4EEC73AF1EE94
:1049E80010FAB4EEE73A8CBFB0EE472AB0EE432A8D
:1049F800F1EE10FA98BFB0EE427AA8BFF0EE437A13
:104A0800032A8DED143A3EF48EAD93ED0E3AD3EDB4
:104A18000D1A93ED0F2A26EE833AA6EE213AA2EE5E
:104A2800253A23EE243AB4EEC73AF1EE10FAB4EE82
:104A3800E73A8CBFB0EE472AB0EE432AF1EE10FAFF
:104A480098BFB0EE427AA8BFF0EE437A042A8DED03
:104A5800153A3EF468AD93ED123AD3ED111A93ED81
:104A6800132A26EE833AA6EE213AA2EE253A23EE41
:104A7800243AB4EEC73AF1EE10FAB4EEE73A8CBF36
:104A8800B0EE472AB0EE432AF1EE10FA98BFB0EE26
:104A9800427AA8BFF0EE437A052A8DED163A3EF425
:104AA80042AD93ED163AD3ED151A93ED172A26EE7B
:104AB800833AA6EE213AA2EE253A23EE243AB4EE42
:104AC800C73AF1EE10FAB4EEE73A8CBFB0EE472AD7
:104AD800B0EE432AF1EE10FA98BFB0EE427AA8BFC2
:104AE800F0EE437A062A8DED173A3EF41CAD93EDAD
:104AF8001A3AD3ED191A93ED1B2A26EE833AA6EE3D
:104B0800213AA2EE253A23EE243AB4EEC73AF1EE62
:104B180010FAB4EEE73A8CBFB0EE472AB0EE432A5B
:104B2800F1EE10FA98BFB0EE427AA8BFF0EE437AE1
:104B3800072A8DED183A3EF4F6AC93ED1E3AD3ED04
:104B48001D1A93ED1F2A26EE833AA1EE863AA2EEAD
:104B5800253A23EE243AB4EEC73AF1EE10FAB4EE51
:104B6800E73A8CBFB0EE472AB0EE432AF1EE10FACE
:104B780098BFB0EE427AA8BFF0EE437A082A8DEDCE
:104B8800193A3EF4D0AC93ED223AD3ED211A93EDC5
:104B9800232A26EE833AA1EE863AA2EE253A23EEA0
:104BA800243AB4EEC73AF1EE10FAB4EEE73A8CBF05
:104BB800B0EE472AB0EE432AF1EE10FA98BFB0EEF5
:104BC800427AA8BFF0EE437A092A8DED1A3A3EF4EC
:104BD800AAAC93ED262AD3ED251A93ED273A26EEB3
:104BE800822AA1EE862AA3EE252A22EE242AB4EEF2
:104BF800C72AF1EE10FAB4EEE72A8CBFB0EE473AB6
:104C0800B0EE423AF1EE10FA8DED1B2A98BFB0EEE5
:104C1800437AB8BFB0EE672A0A2A02F0D182D3EDF0
:104C28002A7AD3ED291A93ED2B3A66EEA77AE1EEAC
:104C3800867AE3EE257A67EEA47AF4EEC77AF1EE87
:104C480010FAF4EEC27A8CBFB0EE473AB0EE673A8B
:104C5800F1EE10FA98BFB0EE437AA8BFB0EE672A1B
:104C68000B2ACDED1C7A02F0AB82D3ED2E7AD3ED70
:104C78002D1A93ED2F3A66EEA77AE6EE217AE5EE45
:104C8800837A67EEA47AB4EEE77AF1EE10FAB4EE1E
:104C9800E72A8CBFF0EE676AF0EE476AF1EE10FA89
:104CA800CDED1D7A58BFB0EE667AA8BFF0EE427A15
:104CB800FEF739BCABF84871002B00F06E81DFF8C5
:104CC8003C830223C24ADFEDC36A11689AF800E008
:104CD8000A78887807EE902AF8EEE77AB0EE007A3C
:104CE80067EEA67AF4EEC77AF1EE10FA40F38C82FA
:104CF80037EEC77ADFEDB86AB0EE676AA7EE266AC4
:104D0800B0EE467A9FEDB56AD8ED006A66EE866A1F
:104D1800B0EEE66ACBED5B6A8BED5E6A98B105EEA4
:104D2800900AB8EEE55ADFEDAB5A66EEA64A25EED4
:104D3800255AF7EE005A75EEC55A64EE864AE5EE36
:104D4800245A66EEA56ADFEDA65A4A7927EE257A37
:104D580027EE267ACAB1DFED9F6ADFEDA25A26EE6A
:104D6800266A06EE902AF8EEE66A66EE866AF4EEA1
:104D7800E56AF1EE10FA00F39185F7EE005A75EE48
:104D8800E66A85EEA66A27EE067ABEF10C0F9FED5D
:104D9800968ADFED966A00F05585B4EEC87AF1EE92
:104DA80010FA98BFB0EE478AB4EEE68AF1EE10FA30
:104DB800B8BFB0EE668A8BED418A002B00F0E08028
:104DC800B0EE007AF4EEC77AF1EE10FA05DD37EEB0
:104DD800C77ADFED816AE7EE267A98ED017ADFED92
:104DE8007F6A27EE267AB0EEC76A8BED5C7A8BED88
:104DF8005F6A98B106EE900ADFED765AF8EEE66A39
:104E080027EE075A66EEA56AF7EE005A75EEE65ADF
:104E180025EE065AE6EE855A27EE257ADFED706A0A
:104E28008A7967EEA67A67EE877AAAB107EE102A22
:104E3800B8EEC77ADFED675ADFED6A6A27EE067AC1
:104E480027EE257AB4EEE67AF1EE10FA40F32A85D9
:104E5800DFED676A67EEA67ABEF10C0F00F0D38427
:104E6800DFED616A9FED617AF4EEE67AF1EE10FA11
:104E780088BFF0EE667AF4EEC77AF1EE10FAB8BFA2
:104E8800F0EE477A012BCBED427A79DD4B78DFEDF6
:104E9800516A07EE903AF8EEE77AB0EE007A67EEDC
:104EA800A67A4B7AF4EEC77AF1EE10FA05DD37EE02
:104EB800C77ADFED496AE7EE267A98ED027ADFEDE8
:104EC800476A27EE267AB0EEC76A8BED5D7A8BEDDE
:104ED800606A9BB106EE903ADFED3E5AF8EEE66A5C
:104EE80027EE075A66EEA56AF7EE005A75EEE65AFF
:104EF80025EE065AE6EE855A27EE257ADFED386A62
:104F0800CB7967EEA67A67EE877A0BB307EE103A8D
:104F1800B8EEC77ADFED2F5ADFED326A27EE067A50
:104F280027EE257AB4EEE67AF1EE10FA0CDCB5EE4F
:104F3800C07AF1EE10FA01F1ED81B7EE006A36EEB3
:104F4800477AC6EE076A01E0DFED296A67EEA67ABE
:104F5800BEF10C0F00F09184DFED236A9FED237AF8
:104F6800F4EEE67AF1EE10FA88BFF0EE667AF4EE27
:104F7800C77AF1EE10FAB8BFF0EE477ACBED437A74
:104F8800BEF1090F00F03684059B93F82160002ECE
:104F980040F0EA8300238BF81831164B1B7823B9AD
:104FA800154EB378002B41F0F081099822F0A6FD48
:104FB8009AF80030072B00F068840022072B8BF842
:104FC80000217DF4AFAB09F0B9FC8146FDF7ACBB1D
:104FD800406E00200AD7233CD7A368416F12033BD9
:104FE80000004843A4707D3F00C0F94400C0F9C4E4
:104FF8000000C842DE6900200D2F0020D04F00209D
:10500800D04A0A920025CDF81490CF4ECF4FA14632
:105018000A9CA846B6EC018AD9ED087AB8EEC88A87
:1050280028EE278AB8F1000F02F0EF877BBB9AF8C9
:105038000030082B3BD005F5D260B0EE480A484452
:10504800D9F88C36984705F5E360D9F81437484401
:1050580098479AF80030032BB0EE408A22D0D9F84E
:10506800AC30D6F84406B0EE480A984704EB8803FB
:1050780008F10108B8F1030F05F12C0583ED010AC9
:105088003DF4C4AB049B1B6803F00053C2E705F56D
:10509800F460B0EE480A4844D9F89C379847B0EE17
:1050A800408AC4E725F0F0FC27F81800D7E7B0EEEF
:1050B800480A25F0E9FC27F81800BCE7A44BDFF8FC
:1050C800CCB21A68A34BA14E9BF80001D2691B8889
:1050D8003280738000287EF477AF81469E4CFDF7BE
:1050E80023BBDFED9E6AFDF76EBF09F027FC099A26
:1050F800964B801AD880FEF7ECBEDFF89482DBED81
:10510800017A9BED006AB8F80000D8F8143077EE01
:10511800A77AF0EE006AB0EE677AA6EE267A013832
:105128000BEBC002D6EE267A083A1033F6EE003AB8
:1051380027EE237A67EEA37A8BED207ACBED217ADE
:10514800DFF848B25E460BF1800192ED027A92EDEB
:10515800036AD6ED036AD6ED027A53ED014A13EDE0
:10516800025A37EE674A76EEC65A77EE277AE4EEA9
:10517800845A0138A2F10802E5EE047A06F108061D
:1051880003F1080336EE267A01F10801E4EE877A86
:10519800E5EE475A67EEA37A25EEA37AC1ED007AC9
:1051A80081ED017AD1D1142F07D109F0C7FB059BF6
:1051B800664EC01A7080DBF8A851624B0A93684AA1
:1051C800049B013582FB05125119EA17C2EBA102B3
:1051D8001B68C2EBC202AD1ACBF8A85103F000530A
:1051E80010E709F0ABFB9AF800300D9A574E801A79
:1051F800012B708000F09180072B7DF495AC09F0AD
:105208009DFB0990FDF792BCB0EE677A7AE5554FA1
:1052180097ED007AFEF7BFBF53495448544BD1ED80
:10522800003A90ED004A53491B788BED7B4ACBED51
:105238007C3AD1ED006A13B101238BF8F831DBED2C
:105248007D7AFDF7EDBE4C494C48D1F8EC1000686A
:1052580044F62066B142A8BF3146B1F57A7FB8BF9F
:105268004FF47A7110F0100F049889B2ABF81A1144
:10527800006801F0DE84C00440F1D7834048076825
:10528800FE8E7608DFF80C81DFF80CE1DBF81C01F4
:10529800D8ED037AAEFB011E4FEA9E1E642191FBF6
:1052A800FEF11429BDEEE77A0BEB400CA8BF1421E0
:1052B80001308842CBF81C0117EE108AA4BF0020E9
:1052C800CBF81C010BEB4000ACF82081B0F92011A1
:1052D80007EE101AB8EEC77A77EEC77AFDEEE77ACE
:1052E800CDED067ABDF9180080EAE071A1EBE07116
:1052F800B14202F34184234908464FF07E510160D0
:10530800FEF780BEA368002B3EF466AE04F14401AC
:1053180020469847FEF760BE0C4E09F00FFB1A4A6C
:10532800DBF8E43112680990C31A9A1ACBF8E40141
:10533800B380F280FDF7FABB09F000FB0D90FDF792
:1053480082BA00BF085C00201C54002024380020CA
:10535800DC52002016240020E45300200000000046
:1053680093244992B467002080380020D44100205B
:1053780044440020E44100206C150020F03900204E
:10538800A828002000000020443A0020701C0020BB
:10539800285C0020D04F0020D34D6210E7EE267A1B
:1053A800F048B1EE455AB0EE447AA5EE277AF0EE11
:1053B800477ABDEEC47A002C3EF402ACF4EEE37AF0
:1053C800F1EE10FAB8BFF0EE467AFDEEE77A17EE86
:1053D800105A17EE906AFDEEC67AB54217EE901A8B
:1053E80017EE104AA8BF3446B142C8BF0C4607EEB4
:1053F800904AF8EEE77A012AC0ED007A3EF445AD0E
:1054080093ED047ADDED137AE7EE267AB0EE447A6E
:10541800A5EE277AB4EEE37AF1EE10FAF0EE477AC9
:10542800B8BFF0EE467AFDEEE77A17EE906A17EE0F
:10543800904AAE42A8BF2C468E42B8BF0C4607EE33
:10544800904AF8EEE77A022AC0ED017A3EF41DADE3
:1054580093ED087ADDED147AE7EE267AB0EE447A19
:10546800A5EE277AB4EEE37AF1EE10FAF0EE477A79
:10547800B8BFF0EE467AFDEEE77A17EE906A17EEBF
:10548800904AAE42A8BF2C468E42B8BF0C4607EEE3
:10549800904AF8EEE77A032AC0ED027A3EF4F5ACBA
:1054A80093ED0C7ADDED157AE7EE267AB0EE447AC4
:1054B800A5EE277AB4EEE37AF1EE10FAF0EE477A29
:1054C800B8BFF0EE467AFDEEE77A17EE906A17EE6F
:1054D800904AAE42A8BF2C468E42B8BF0C4607EE93
:1054E800904AF8EEE77A042AC0ED037A3EF4CDAC90
:1054F80093ED107ADDED167AE7EE267AB0EE447A6F
:10550800A5EE277AB4EEE37AF1EE10FAF0EE477AD8
:10551800B8BFF0EE467AFDEEE77A17EE906A17EE1E
:10552800904AAE42A8BF2C468E42B8BF0C4607EE42
:10553800904AF8EEE77A052AC0ED047A3EF4A5AC65
:1055480093ED147ADDED177AE7EE267AB0EE447A19
:10555800A5EE277AB4EEE37AF1EE10FAF0EE477A88
:10556800B8BFF0EE467AFDEEE77A17EE906A17EECE
:10557800904AAE42A8BF2C468E42B8BF0C4607EEF2
:10558800904AF8EEE77A062AC0ED057A3EF47DAC3B
:1055980093ED187ADDED187AE7EE267AB0EE447AC4
:1055A800A5EE277AB4EEE37AF1EE10FAF0EE477A38
:1055B800B8BFF0EE467AFDEEE77A17EE906A17EE7E
:1055C800904AAE42A8BF2C468E42B8BF0C4607EEA2
:1055D800904AF8EEE77A072AC0ED067A3EF455AC11
:1055E80093ED1C7ADDED197AE7EE267AB0EE447A6F
:1055F800A5EE277AB4EEE37AF1EE10FAF0EE477AE8
:10560800B8BFF0EE467AFDEEE77A17EE906A17EE2D
:10561800904AAE42A8BF2C468E42B8BF0C4607EE51
:10562800904AF8EEE77A082AC0ED077A3EF42DACE6
:1056380093ED207ADDED1A7AE7EE267AB0EE447A19
:10564800A5EE277AB4EEE37AF1EE10FAF0EE477A97
:10565800B8BFF0EE467AFDEEE77A17EE906A17EEDD
:10566800904AAE42A8BF2C468E42B8BF0C4607EE01
:10567800904AF8EEE77A092AC0ED087A3EF405ACBC
:1056880093ED247ADDED1B7AE7EE267AB0EE447AC4
:10569800A5EE277AB4EEE37AF1EE10FAF0EE477A47
:1056A800B8BFF0EE467AFDEEE77A17EE906A17EE8D
:1056B800904AAE42A8BF2C468E42B8BF0C4607EEB1
:1056C800904AF8EEE77A0A2AC0ED097A3EF4DDAB93
:1056D80093ED287ADDED1C7AE7EE267AB0EE447A6F
:1056E800A5EE277AB4EEE37AF1EE10FAF0EE477AF7
:1056F800B8BFF0EE467AFDEEE77A17EE906A17EE3D
:10570800904AAE42A8BF2C468E42B8BF0C4607EE60
:10571800904AF8EEE77A0B2AC0ED0A7A3EF4B5AB68
:1057280093ED2C7ADDED1D7AE6EE877AA5EE274A11
:10573800F4EEC43AF1EE10FAC8BFB0EE464AFDEEF8
:10574800C47A17EE903A9D42A8BF1D469942D8BF29
:10575800294607EE901AF8EEE77AC0ED0B7AFEF7C5
:1057680094BB00BF403800201E21BD4806F0E9F870
:1057780000283FF40FACBB4B1B8858063FF50AAC1A
:105788009BF88431B34242F0A782B74BDBED627AD3
:1057980093ED010ADBED435A9FEDB46ADFEDB46A7D
:1057A80027EEE57A67EE887AA0EE087AE5EE807A49
:1057B800B4EEC67AF1EE10FA88BFB0EE467AB4EECF
:1057C800E67AF1EE10FAF4EEC67AB8BFB0EE667A71
:1057D800F1EE10FA88BFF0EE467AF4EEE67AF1EED2
:1057E80010FAB8BFF0EE667A8BED417ACBED437ACA
:1057F800FFF7D0BBFDEEC87A9E4E17EE903AB78001
:10580800F380FFF7C1BB9FED997ADFED996A994E56
:10581800F4EEC77AF1EE10FA98BFB0EE677AFDEEB3
:10582800E77AB4EEE67AF1EE10FA17EE902AB8BFEE
:10583800B0EE667A012B8BED427A72803FF726AB89
:10584800FFF7A2BBB4EEC87AF1EE10FA98BFB0EE3B
:10585800478ABDEEC77AB4EEE68A864EF1EE10FAB4
:1058680017EE102AB8BFB0EE668A8BED418A3280F7
:10587800002B7FF4A5AAFFF787BBBDEEE77A7D4E24
:1058880017EE103AB380FFF767BB09F057F8794E67
:105898009AF80030401BB080FFF78FBB9FED766A07
:1058A800FFF771BAB5EEC07AF1EE10FA00F136855D
:1058B800B7EE006A36EE477AC6EE076AFFF7CABA4D
:1058C800FDEEE37A84F0010117EE906AFDEEC47AEA
:1058D8000C9117EE907AFDEEC67A12A800EB8203BF
:1058E800CDF838B0DFF8A891DFF8A8E1DDF830B0DE
:1058F8000D9217EE905AB1EE455A4FFA84FC1946AC
:10590800CDF83C804B4693ED007AF0EC017AE6EE58
:10591800877A04F0010309F11009B0EE447AA5EE84
:10592800277AF4EEC73AF1EE10FAD8BF0023002B1D
:10593800F0EE477A18BFB0EE467ABDEEC77AFDEEB4
:10594800E77A17EE102A17EE908ABA4217EE103A45
:10595800A8BF3B469542CCBF002204F00102002AB2
:1059680008BF2B46474507EE103A3A46A8BF4246BD
:105978004645CCBF00230BF00103002B08BF32467D
:1059880007EE902AB8EEC77AF8EEE77ABCF1000F76
:1059980018BFF0EE477A8842EEEC017AB2D10D9A40
:1059A800DDF838B0DDF83C80FDF7D1BF91F8201064
:1059B800C1EB411001EB8001C90089B2FEF72FBB92
:1059C8002E4BB5F908101A6802B111609B69B5F938
:1059D8000A2003B11A60049B1B689A0601F14A87E2
:1059E80002220B92FEF734BF9BF82432012B01F000
:1059F800C887234B96F916005A8896F90AE01B883F
:105A0800204910FB03F31EFB02F281FB020C81FB11
:105A18000301D217DB17C2EB2C12C3EB21133A4454
:105A28001C442A806C80FDF7E7BF17480768B7F960
:105A3800366027E4DFF860801448D8F80820B8F802
:105A48000C1024F09BF89AF80070142F02F0E481EF
:105A5800DBF8A8510135CBF8A851FFF750BB00BFC0
:105A6800F0390020DC6900200000002000C0F94463
:105A780000C0F9C4243800200000C8422C4200208D
:105A8800D03B00201F85EB51A8280020701C002067
:105A98001041002040380020285C0020DFF8608397
:105AA800B8F80060D8F804E04FEA560C4FEA8C02C8
:105AB8000BEB8607F6080BEB020300F09F80103211
:105AC8000136C44803EB06163A4410330EF11005AC
:105AD80007F1100151ED032A51ED043A10ED043A93
:105AE80010ED032A51ED026A11ED016A10ED020A68
:105AF80010ED018A12ED044A12ED035A53ED044ADF
:105B080053ED035A13ED027A53ED017A52ED020A6E
:105B180012ED011A73EE238A72EE221A40ED048AFE
:105B280040ED031A70EE268A78EE061A40ED028AD6
:105B380040ED011A74EE848A75EE851A43ED048AE5
:105B480043ED031A77EE208A77EE811A43ED028A35
:105B580043ED011A73EE633A75EE655A15ED035A73
:105B680032EE623A74EE644A65EE631A15ED044A41
:105B780023EE052A64EE652AE3EE041A1033B342D5
:105B880024EE843AA3EE842A00F1100005F11005F2
:105B9800A5EE853A01F1100102F11002E4EE852A22
:105BA80041ED071A01ED082A02ED073A42ED082AED
:105BB80055ED055A15ED065A70EE666A38EE466AD6
:105BC80030EEC77A71EE677A26EE253A65EEE63A48
:105BD80025EE674A67EE054AE6EE053AA6EE853AEF
:105BE800A7EE254AE7EEA54A01ED063A41ED053A4A
:105BF80002ED064A42ED054A7FF46CAF1FFA8CF5B8
:105C080072462946744820F031FC2946D8F8042009
:105C1800384620F02BFC9AF80030142B7FF4CBAADE
:105C2800FFF7C3BA6D4BDBF8ACC10A93BBF8A4818C
:105C3800C8F12003D8B26A4B08EB4C1603EB860672
:105C4800830802F0B88001331B016649614A069354
:105C580006EB030E06F1100313ED024A13ED035A87
:105C680013ED016A13ED047A51ED024A51ED035A1E
:105C780051ED016A51ED047A64EE244A65EE255A25
:105C880066EE266A67EE277A1033734542ED024ABC
:105C980042ED035A42ED016A42ED047A01F1100126
:105CA80002F11002D8D1069B4F49A3F11002164405
:105CB80001EB020E5A4410F0030309D0B6EC017A46
:105CC800FEEC017A67EE277A013BE2EC017AF5D126
:105CD800B8F1000F41F0D485142F7FF470AA08F0B2
:105CE8002DFE059B414EDBF8A851C01A7080FFF7C6
:105CF80066BADBF8AC81394A3D4B0A9203EBC8031C
:105D0800126806929DED067A9B88DFED3A7A3A4A48
:105D1800F8EE478A09EE103A643BC82BA8BFC8239F
:105D280068EEA78AF8EE497A782BB8BF782368EE30
:105D3800A78A07EE903A2C26B0EE680A06FB0826DA
:105D4800B8EEE78A24F0ECFEB8EEC99AF0EE409A75
:105D5800B0EE680A24F046FE38EE097A79EE487A01
:105D680028EE098A67EE877AB7EE006A88EE277A06
:105D7800142FF8EE007A77EE076A60EE277A89EE3C
:105D8800A67A77EE065A36EE477AC6EE256A67EEA9
:105D9800A67A27EE267AC6ED006A86ED047AC6ED65
:105DA800026AC6ED017AC6ED037A02F00980134B48
:105DB8009AF8007008F1010883FB083CACEBE87C1A
:105DC8000CEB4C0C0135A8EB0C0CCBF8A851CBF81C
:105DD800ACC12BE7801C0020701C0020085C002050
:105DE800405C0020D05D0020C05D002024380020E9
:105DF800405E002027D4D236845B00205655555586
:105E0800285C0020DFF8AC8398F800205FEA920C49
:105E180002F07680DFF8DCE30CF1010040010EEBC4
:105E280000060EF12003AEF1700113ED076A53ED81
:105E3800056A13ED037A53ED017A53ED025A13ED17
:105E4800084A53ED064A13ED045A26EE066A66EE32
:105E5800A66A27EE077A67EEA77AA4EE046A2033CB
:105E6800B342E4EEA46A01F11001A5EE057AE5EE6D
:105E7800A57AF1EEC65AB1EEE66AF1EEC76AB1EE5E
:105E8800E77A41ED085A01ED076A41ED066A01ED2E
:105E9800057ACAD1203886440BEB0C1112F00303A3
:105EA80018BF0EF1080E0FD05EED017A1EED027AD2
:105EB80067EEA77A013BE7EE077A0EF1080EB1EE1E
:105EC800E77AA1EC017AEFD1142F01F0AF87013501
:105ED800CBF8A85101E0B74B1A78DBF8ACE1B6482B
:105EE8009FEDC67A4FEACE06831983ED007A002A21
:105EF8007AD0B249B0EE476AF0EE476A0023F1EC77
:105F0800017A013367EEA77A05EE903AB4EEE77AA4
:105F1800F1EE10FAF8EEE55AB8BFB0EE677A9A4299
:105F280076EEA76AA7EEA56AE9D1F5EEC06A8319ED
:105F3800F1EE10FA83ED007A56DDC6EE265AA04B34
:105F4800A04A1288F7EE007A75EEE75AD3ED007A88
:105F580065EEA77AFDEEE77A17EE903A812B41F3CA
:105F680036819342A8BF134607EE903AF8EEE77AD7
:105F7800954B2C2101FB0E3393ED097AD3ED003AB2
:105F880093ED0A6A93ED014AD3ED046AD3ED034A0F
:105F980093ED025AA3EEA77AA4EE276A66EEC76AC3
:105FA800A7EE646ABDEEC77AE5EE276A17EE101A07
:105FB800812983ED096AC3ED0A6A41F305818A42A2
:105FC800A8BF0A4607EE902AF8EEE77AFCEEE77AD1
:105FD800CDED067ABDF8183082199380BEF1000F16
:105FE80002D1132F01F04B86152F7FF4DCA8304423
:105FF800764E838826F81E30754BDBF8A8510A9335
:10600800FFF7DDB8734A32F91340FDF7EEBC714A69
:1060180032F91370FDF7DEBC6E4B6F4D1A68596884
:106028002A609A68DB68EB6069606C4EAA60069B20
:10603800FDF7C4BC08F082FC9AF800700590142F94
:1060480005BF624EDBF8A851DBF8A8513580FCF794
:10605800C5BB634F002437F9023F00EE103AE0B2A7
:10606800B8EEC00A013411F08FF8082CF3D10B9464
:10607800FEF7E6BB5B4F002437F9023F00EE103A0B
:10608800E0B2B8EEC00A013411F07EF8062CF3D164
:10609800EDE7554BB5F906101A6802B111609B6916
:1060A800B5F90820002B7FF495AC94E44F4F0024F9
:1060B80037F9023B00EE103AE0B2B8EEC00A0134FC
:1060C80011F062F8042CF3D1D1E7494FDFF82881A9
:1060D80097ED004A97ED097AD7ED014A97ED0A6ADC
:1060E800D7ED046A97ED035AD7ED025A69EE277A7D
:1060F80008EB8503A4EE277AA4EEA76A66EEC76AC2
:10610800A5EE476AE5EEA76A20EE070A87ED096A59
:10611800C7ED0A6A83ED007A29EE088A24F0B4FCF8
:1061280069EE288AD7ED145AD7ED1F6A97ED0B1A36
:10613800D7ED161A97ED155A97ED207A97ED0C2A98
:10614800D7ED172A97ED0F6AD7ED1A7A97ED0E3A21
:10615800D7ED0D3A97ED194AD7ED184AE8EE015AEE
:10616800002208EB8503E8EEA16A00B2CBF894217F
:10617800A8EE025ACBF89821CBF89C21A8EEA27A77
:1061880026EE656A67EEE67AA5EEC35AA8EE236A9C
:10619800A6EEC47AE8EEA47A87ED145AC3ED205A25
:1061A80087ED156AC3ED406A87ED1F7AC7ED207A3F
:1061B800FEF7FBBA225C0020405E0020701C002025
:1061C800245C0020205C0020585E00202438002039
:1061D800085C0020B4690020303800205068002096
:1061E8002E380020323800202C420020363800207B
:1061F800DC5E0020F01C0020405C00200000000055
:10620800B4F92430E26207EE903A0122F8EEE77A18
:106218002366E2670023012FC4ED1C7AC4ED1B7AC4
:10622800636701F01985AF427CF464ADB4F9263098
:10623800636607EE903A00220123F8EEE77A2263BC
:10624800C4F890300023012FC4ED217AC4ED207AE0
:10625800C4F8883001F0FC84AF427CF47BADB4F91B
:106268002830A36607EE903A00220123F8EEE77A79
:106278006263C4F8A4300023012FC4ED267AC4ED6C
:10628800257AC4F89C307CF495AD1FED248AB8F1CA
:10629800030F01F08684049B4BB107EE903AF8EEA9
:1062A800E77AF4EEC87AF1EE10FA01F12486C64ACC
:1062B800A36E12689BF8B011F08003EB550393FBB3
:1062C800F5F50023656393621363D36221B1BF4B75
:1062D8001B88002B7CF46FADBD4B1B6813F4003397
:1062E80004D0BC4B1B79002B41F0FF85BA491A46F4
:1062F800C85C012803F10C0301F0A4820132152ABD
:10630800F6D1FCF758BDB54B9B7B002B3DF485AF10
:10631800FDF769BEF7EE006AFEF718BEF7EE006AF1
:10632800FEF798BDBBF84871013F3FB2002FABF8AC
:1063380048717EF7C1ACDFF8DC82FDF7C2BEBBF85E
:106348001A1101F57A7189B2FDF769BE089B1F78A9
:1063580007F0010CFDF799BDA14BDFEDA27A196892
:10636800CBED707A11F0805100F08584B7EE007A99
:1063780077EE677AF4EEE27AF1EE10FA88BFF0EE83
:10638800627ACBED7D7AFDF744B9974F3A78013AB6
:106398000A2A1CD8DFE812F00A01BA017001550177
:1063A8001B001B004001A701E600D1000B008F4A2B
:1063B8008F4952680968C8328A4203D310F056F9E7
:1063C80028B1B378032B01F0578601233B70F3788B
:1063D800002B3EF4EAAD049B1B68DA0441F19F856B
:1063E800844B9B8807EE903AF8EEE77A824A92ED62
:1063F800012AD2ED022A92ED033AD2ED043A92ED47
:10640800054AD2ED064A92ED075AD2ED085A92EDA6
:10641800096AD2ED0A6A92ED0B7AB4EE672AF1EEB8
:1064280010FAF4EE672A14BF01230023F1EE10FAE4
:10643800B4EE673A18BF43F00103F1EE10FAF4EE38
:10644800673A18BF43F00103F1EE10FAB4EE674A59
:1064580018BF43F00103F1EE10FAF4EE674A18BFD3
:1064680043F00103F1EE10FAB4EE675A18BF43F097
:106478000103F1EE10FAF4EE675A18BF43F0010376
:10648800F1EE10FAB4EE676A18BF43F00103F1EEBB
:1064980010FAF4EE676A18BF43F00103F1EE10FA40
:1064A800B4EE677A18BF43F00103F1EE10FA18BF93
:1064B80043F00103002B41F0948492ED007AB4EE8E
:1064C800677AF1EE10FA41F08C84DFF82481DBF86A
:1064D8009021D8F800309A4201F28A843B78012B47
:1064E8003EF463AD9BF88C21002A3EF45EAD0B2B85
:1064F80018D801229A4040F6030112EA010617D182
:1065080012F4C06F0ED0093B012B0BD8452010F0B8
:10651800CFF8FF2010F0CCF8384810F0B5F8304626
:1065280010F0C6F8314BD8F800205A600B233B70A6
:1065380000238BF88C31FEF738BD314B1B78002BCC
:1065480001F04A841A2020F0E9FF002841F0448431
:106558009BF88C31002B41F03F8409233B7011F0EC
:10656800B7FD34E71A2020F0D9FF0028F7D0254BD3
:106578001B88002BF3D1244B4520D3F8008010F062
:1065880097F80E2010F094F8404611F0D9FADDF88B
:106598002480404611F0D4FA1C4A4FF480510A2353
:1065A800404611803B7011F0DDFAD8E7184B1B7894
:1065B800D9077FF50CAF802022F050FB08B122F0FC
:1065C80051F812F023FB02E7DC5200208869002012
:1065D8003C2500205869002030D602081C420020C3
:1065E800F0390020000000800C2F0020003A002025
:1065F800C0530020D8410020E040002038F30208B2
:10660800B43A00207038002074380020F83900208F
:1066180035690020D04F002010F00AF8604B0021A7
:1066280005208DE80300A3F108020291532012F01F
:1066380023FA00287FF4CBAE5A4A082310603B7037
:10664800C5E60FF0F5FF584A0292A2F10C03252186
:1066580001930091A2F10A035021163A492012F041
:106668000BFA00287FF4B3AE4E4B4FF0FF310722F0
:10667800186059603A70AAE6DFF828810FF0D8FF51
:106688004A4AD8F80430126864339342BFF49FAE84
:1066980040200FF0B3FF00287FF499AED8F80030FF
:1066A80043494FF040090FE0059110F001F80599B2
:1066B800D8F800300A680133013AB9F101090A60D3
:1066C800C8F8003001F0D1843A4AD35C1846002B50
:1066D800EAD100234FF0FF32C8F800300423C8F88D
:1066E80004203B7073E60FF0A3FF11F011FD0028A2
:1066F8003FF46DAE0FF0BAFF00283FF468AE2E4AA3
:106708004FF480510A2311803B7060E6274B254ADD
:106718001B68536026490023136003220B603A70FC
:1067280055E6264BDFED267A93ED080AB4EEE70A24
:10673800F1EE10FA41F2F88024F03CFADBED457AEC
:1067480020EE270A24F0A0F9B0F5617F01F33A8121
:1067580007EE900AF8EEE76ADFED1A7A66EEA76AA6
:1067680007EE906AB8EEE77AFDEEE67A17EE903A11
:106778002033402B41F275839FED130A24F084F9EE
:1067880000B207EE900AB8EEE77ADFF84080D8ED5D
:10679800037A77EE877AC8ED037AFDF72CBC00BF41
:1067A80024D20208003A002076D00208C053002004
:1067B8005C2F002000D00208F8390020903B002010
:1067C8008FC2753CD06D393A00000000D04F0020D0
:1067D800002840F06286E7EE267ADE48BDEEC47AED
:1067E80017EE105AB0EE637AA5EE277A2C46F0EE33
:1067F800477AFDEEE77ABDEEC67A17EE906A17EE95
:10680800101AB542A8BF3446B142C8BF0C4607EEBD
:10681800904AF8EEE77A012AC0ED007A3DF435ABEC
:1068280093ED047ADDED137AE7EE267AB0EE637A1B
:10683800A5EE277AFDEEC77A17EE906A17EE904A12
:10684800AE42A8BF2C468E42B8BF0C4607EE904A0F
:10685800F8EEE77A022AC0ED017A3DF416AB93ED23
:10686800087ADDED147AE7EE267AB0EE637AA5EEC3
:10687800277AFDEEC77A17EE906A17EE904AAE4275
:10688800A8BF2C468E42B8BF0C4607EE904AF8EED9
:10689800E77A032AC0ED027A3DF4F7AA93ED0C7A61
:1068A800DDED157AE7EE267AB0EE637AA5EE277A63
:1068B800FDEEC77A17EE906A17EE904AAE42A8BF6F
:1068C8002C468E42B8BF0C4607EE904AF8EEE77A9F
:1068D800042AC0ED037A3DF4D8AA93ED107ADDEDD1
:1068E800167AE7EE267AB0EE637AA5EE277AFDEE01
:1068F800C77A17EE906A17EE904AAE42A8BF2C46A8
:106908008E42B8BF0C4607EE904AF8EEE77A052AA1
:10691800C0ED047A3DF4B9AA93ED147ADDED177A47
:10692800E7EE267AB0EE637AA5EE277AFDEEC77A0F
:1069380017EE906A17EE904AAE42A8BF2C468E42D8
:10694800B8BF0C4607EE904AF8EEE77A062AC0ED83
:10695800057A3DF49AAA93ED187ADDED187AE7EEF8
:10696800267AB0EE637AA5EE277AFDEEC77A17EE9F
:10697800906A17EE904AAE42A8BF2C468E42B8BF26
:106988000C4607EE904AF8EEE77A072AC0ED067A39
:106998003DF47BAA93ED1C7ADDED197AE7EE267AB1
:1069A800B0EE637AA5EE277AFDEEC77A17EE906A05
:1069B80017EE904AAE42A8BF2C468E42B8BF0C468E
:1069C80007EE904AF8EEE77A082AC0ED077A3DF418
:1069D8005CAA93ED207ADDED1A7AE7EE267AB0EE1E
:1069E800637AA5EE277AFDEEC77A17EE906A17EE5E
:1069F800904AAE42A8BF2C468E42B8BF0C4607EE5E
:106A0800904AF8EEE77A092AC0ED087A3DF43DAAE3
:106A180093ED247ADDED1B7AE7EE267AB0EE637A01
:106A2800A5EE277AFDEEC77A17EE906A17EE904A20
:106A3800AE42A8BF2C468E42B8BF0C4607EE904A1D
:106A4800F8EEE77A0A2AC0ED097A3DF41EAA93ED1A
:106A5800287ADDED1C7AE7EE267AB0EE637AA5EEA9
:106A6800277AFDEEC77A17EE906A17EE904AAE4283
:106A7800A8BF2C468E42B8BF0C4607EE904AF8EEE7
:106A8800E77A0B2AC0ED0A7A3DF4FFA993ED2C7A38
:106A9800DDED1D7AE6EE877AE5EE273AFDEEE37A3C
:106AA80017EE903A9D42A8BF1D468B42A8BF2946C3
:106AB80007EE901AF8EEE77AC0ED0B7AFDF7E5B924
:106AC8000A9B002B00F09887FDEEC67A12A917EEF4
:106AD80090EAFDEEC47A204D1E4E17EE903AFDEE78
:106AE800E37A01EB820217EE907A14E0FDEEC77AA2
:106AF80017EE909A4F4503DC9945CC46A8BF9C46B3
:106B080007EE90CAF8EEE77A9142E6EC017A05F1D1
:106B180010053DF4BEA995ED007AF1EC017AE7EE97
:106B2800267ABC46B0EE637AA5EE277AF0EE477A6D
:106B3800002CDBD030B1F4EE473AF1EE10FAC8BFC2
:106B4800F0EE467AFDEEE77AF44617EE909ACE45D7
:106B5800D2DDD5E740380020104100200A9B002BE9
:106B680000F0AB87FDEEE37A12AB17EE906AFDEE0C
:106B7800C47AD349D34D17EE90EAFDEEC67AB1EE4A
:106B8800455A17EE907A03EB820214E0FDEEC77ABD
:106B980017EE90CAB44503DBF445A8BFF446E146B6
:106BA80007EE909AF8EEE77A9342E5EC017A01F164
:106BB80010013DF46EA991ED007AF3EC017AE7EE4D
:106BC800267AB146B0EE447AA5EE277AF0EE477AF7
:106BD800002CDBD0BC4630B1B4EE637AF1EE10FA8B
:106BE80048BFF0EE467AFDEEE77A17EE909AB9457F
:106BF80004DBF14517EE90CAA8BFF44607EE90CA29
:106C0800F8EEE77AD0E707F099FE0546FDF7DDB91B
:106C1800AD4B196811F080512DD0B6EE007A67EEB1
:106C2800877AF4EEE27AF1EE10FA3FF7AAABFFF7B3
:106C38009DBBC6003EF51FABFDF7E4B9F0EE647AE4
:106C4800FCF771BCA149A248A24BD1ED003A90EDE6
:106C5800004AA1491B78CBED7D7A8BED7B4ACBEDC1
:106C68007C3AD1ED006A002B3CF4DAA901238BF8B9
:106C7800F831FCF7D5B9069B13F4800101D0002147
:106C8800CBE7B6EE007AF4EEC72AF1EE10FAC4DCD0
:106C9800FCF7BFBCFDEEC67A12AB17EE905AFDEEBC
:106CA800C47A8749874C17EE90EA03EB8206D1ED48
:106CB800007AB3EC017AA6EEA77A1031F0EE635AA7
:106CC800E5EE075A07EE905AB0EE657A30B1F4EE69
:106CD800653AF1EE10FAC8BFB0EE467ABDEEC77A53
:106CE80017EE107ABD4204DC7745A8BF774607EE59
:106CF800907AF8EEE77A9E42E4EC017AD7D1FCF775
:106D080026BE012A40F3A88707EE101AB8EEC77A04
:106D1800C7EE876AB1EEE68AB8F1030F00F048873C
:106D2800049B4BB107EE903AF8EEE77AB4EEE78AA7
:106D3800F1EE10FA01F3DF80236E03EB550393FBAA
:106D4800F5F3E362FFF76FBA012A7FF79EAA07EE11
:106D5800101AB8EEC77AC7EE876AB1EEE68AFFF76F
:106D680096BA012A40F3748707EE101AB8EEC77A6C
:106D7800C7EE876AB1EEE68AB8F1030F00F00A871A
:106D8800049B4BB107EE903AF8EEE77AB4EEE78A47
:106D9800F1EE10FA01F3AF80636E03EB550393FB3A
:106DA800F5F32363FFF758BA079B1B88DA0540F110
:106DB800238798ED017A494BD8ED006AD8ED027A1D
:106DC800059A0C93BDEEC77AB3F90660118B17EEDE
:106DD800103AFDEEE66AFDEEE77A16EE902AADF877
:106DE8004A3017EE903AADF84820ADF84C303C4A9E
:106DF8003448B2F90230B2F900203A4CD0ED007AAA
:106E08009FED397A39484FF47A7503F5E16302F555
:106E1800E16205FB02F205FB03F384FB037584FBC7
:106E280002740C9F00780A901D4477EEC77ADB172E
:106E3800C3EBE5233D88B8881444FDEEE77AD21702
:106E48006D1AC2EBE422A3F5FA737C88ADF86030C2
:106E5800ADF8505017EE903A0C9D3F89ADF84E3082
:106E6800641AA2F5FA72401AAB89ADF86220ADF83F
:106E780052406A89EC89ADF854001D4D0A98761A7B
:106E88007F1A521A5B1A641A0021ADF85660ADF8E1
:106E98005870ADF85A20ADF85C30ADF85E40296006
:106EA8006960A960E960002801F0A880114E124FBE
:106EB800DFF84880CDF834B0894605965EE000BF1B
:106EC8001041002040380020F03900208038002090
:106ED800D441002044440020E4410020B46900204B
:106EE800D03B0020C5B3A2910080BB4400670020BE
:106EF800303800205068002004670020741E0020ED
:106F08001EAB03EB440030F9300CA8F80000059BD9
:106F180097F902E00E441EFB00F053F826600123A7
:106F280003FA04F4AC4B83FB003EC017069B3442C3
:106F3800C0EB6E100CBF01244FF0FF3498420EDBFB
:106F4800079B02FB03F2A44B83FB0263D217C2EB3D
:106F58006313A3EB0C031BB28342A8BF034635F8A7
:106F6800112003FB042325F811300A9B09F10109BC
:106F7800994507F1070708F1020850DABB79002B99
:106F880036D1397897F9052007924E00059A97F976
:106F9800043097F803E07C78701802EB8000C28810
:106FA8008088121A92B28C4802FB03F380FB03C05C
:106FB800DB17C3EB60134FEA520CA3EB0C031BB2B5
:106FC8000693BEF1000F9BD01EAB03EB440BB8F940
:106FD80000003BF930BC584513DA8644704503DCA1
:106FE800F3455846A8BF704600B2A8F800008EE7DF
:106FF8001633D8B220F092FA0028C2D1A8F80000BF
:10700800B3E784DDA0EB0E0EDE4503DB7045A8BFB9
:10701800704683460FFA8BF0A8F8000077E7DDF892
:1070280034B0059E96F90A002B886B4A6B4910FB11
:1070380003F3F07A097882FB0342FF284FEAE373EF
:10704800C3EB621200F08D84814240F28A840C9B6B
:1070580033F9100096F916406B88104428805E4A70
:10706800F07D14FB03F382FB0342FF284FEAE3732E
:10707800C3EB621200F07184814240F26E840C9B73
:1070880033F9100096F92240AB8810446880524AC0
:1070980096F8230014FB03F382FB0342FF284FEA10
:1070A800E373C3EB621200F05484814240F25184CE
:1070B8000C9B33F9100096F92E40EB881044A880F9
:1070C800454A96F82F0014FB03F382FB0342FF287E
:1070D8004FEAE373C3EB621200F03784814240F257
:1070E80034840C9B33F9100096F93A402B891044EC
:1070F800E880394A96F83B0014FB03F382FB03420D
:10710800FF284FEAE373C3EB621200F01A8481424E
:1071180040F217840C9B33F9100096F946406B89AE
:10712800104428812C4A96F8470014FB03F382FB8D
:107138000342FF284FEAE373C3EB621200F0FE83B9
:10714800814240F2FB830C9B33F9100096F95240C0
:10715800AB8910446881204A96F8530014FB03F366
:1071680082FB0342FF284FEAE373C3EB621200F08D
:10717800E283814240F2DF830C9B33F9100096F9D9
:107188005E40EB891044A881134A96F85F0014FB0F
:1071980003F382FB0342FF284FEAE373C3EB621356
:1071A80000F0C683884280F0C3830C9A32F910201D
:1071B8000499096806911344EB810B46FCF7FEBB62
:1071C800F0EE427AFCF7AFB98223FEF705BFDFED98
:1071D800047AFEF7CDBE00BF1F85EB51F86300208F
:1071E80000000243FDEEE77A17EE105A17EE906A98
:1071F800FDEEC67AB54217EE901A17EE104AA8BFF0
:107208003446B142C8BF0C4607EE904AF8EEE77A1A
:10721800012AC0ED007A3CF438AE93ED047ADDED36
:10722800137AE7EE267AB0EE447AA5EE277AFDEED9
:10723800C77A17EE906A17EE904AAE42A8BF2C465E
:107248008E42B8BF0C4607EE904AF8EEE77A022A5B
:10725800C0ED017A3CF419AE93ED087ADDED147AAD
:10726800E7EE267AB0EE447AA5EE277AFDEEC77AE5
:1072780017EE906A17EE904AAE42A8BF2C468E428F
:10728800B8BF0C4607EE904AF8EEE77A032AC0ED3D
:10729800027A3CF4FAAD93ED0C7ADDED157AE7EE5F
:1072A800267AB0EE447AA5EE277AFDEEC77A17EE75
:1072B800906A17EE904AAE42A8BF2C468E42B8BFDD
:1072C8000C4607EE904AF8EEE77A042AC0ED037AF6
:1072D8003CF4DBAD93ED107ADDED167AE7EE267A15
:1072E800B0EE447AA5EE277AFDEEC77A17EE906ADB
:1072F80017EE904AAE42A8BF2C468E42B8BF0C4645
:1073080007EE904AF8EEE77A052AC0ED047A3CF4D5
:10731800BCAD93ED147ADDED177AE7EE267AB0EE80
:10732800447AA5EE277AFDEEC77A17EE906A17EE33
:10733800904AAE42A8BF2C468E42B8BF0C4607EE14
:10734800904AF8EEE77A062AC0ED057A3CF49DAD3E
:1073580093ED187ADDED187AE7EE267AB0EE447AE6
:10736800A5EE277AFDEEC77A17EE906A17EE904AD7
:10737800AE42A8BF2C468E42B8BF0C4607EE904AD4
:10738800F8EEE77A072AC0ED067A3CF47EAD93ED75
:107398001C7ADDED197AE7EE267AB0EE447AA5EE8E
:1073A800277AFDEEC77A17EE906A17EE904AAE423A
:1073B800A8BF2C468E42B8BF0C4607EE904AF8EE9E
:1073C800E77A082AC0ED077A3CF45FAD93ED207A9E
:1073D800DDED1A7AE7EE267AB0EE447AA5EE277A42
:1073E800FDEEC77A17EE906A17EE904AAE42A8BF34
:1073F8002C468E42B8BF0C4607EE904AF8EEE77A64
:10740800092AC0ED087A3CF440AD93ED247ADDED0D
:107418001B7AE7EE267AB0EE447AA5EE277AFDEEDF
:10742800C77A17EE906A17EE904AAE42A8BF2C466C
:107438008E42B8BF0C4607EE904AF8EEE77A0A2A61
:10744800C0ED097A3CF421AD93ED287ADDED1C7A84
:10745800E7EE267AB0EE447AA5EE277AFDEEC77AF3
:1074680017EE906A17EE904AAE42A8BF2C468E429D
:10747800B8BF0C4607EE904AF8EEE77A0B2AC0ED43
:107488000A7A3CF402AD93ED2C7ADDED1D7AE6EE36
:10749800877AA5EE274AFEF752B9E7EE267AE8483A
:1074A800BDEEC47A17EE105AB0EE637AA5EE277ACD
:1074B8002C46F0EE477AF4EEE37AF1EE10FAB8BF14
:1074C800F0EE467AFDEEE77ABDEEC67A17EE906AE0
:1074D80017EE101AB542A8BF3446B142C8BF0C46D1
:1074E80007EE904AF8EEE77A012AC0ED007A3CF4FC
:1074F800CCAC93ED047ADDED137AE7EE267AB0EEA4
:10750800637AA5EE277AB4EEE37AF1EE10FAF0EE9C
:10751800477AB8BFF0EE467AFDEEE77A17EE906A42
:1075280017EE904AAE42A8BF2C468E42B8BF0C4612
:1075380007EE904AF8EEE77A022AC0ED017A3CF4A9
:10754800A4AC93ED087ADDED147AE7EE267AB0EE76
:10755800637AA5EE277AB4EEE37AF1EE10FAF0EE4C
:10756800477AB8BFF0EE467AFDEEE77A17EE906AF2
:1075780017EE904AAE42A8BF2C468E42B8BF0C46C2
:1075880007EE904AF8EEE77A032AC0ED027A3CF457
:107598007CAC93ED0C7ADDED157AE7EE267AB0EE49
:1075A800637AA5EE277AB4EEE37AF1EE10FAF0EEFC
:1075B800477AB8BFF0EE467AFDEEE77A17EE906AA2
:1075C80017EE904AAE42A8BF2C468E42B8BF0C4672
:1075D80007EE904AF8EEE77A042AC0ED037A3CF405
:1075E80054AC93ED107ADDED167AE7EE267AB0EE1C
:1075F800637AA5EE277AB4EEE37AF1EE10FAF0EEAC
:10760800477AB8BFF0EE467AFDEEE77A17EE906A51
:1076180017EE904AAE42A8BF2C468E42B8BF0C4621
:1076280007EE904AF8EEE77A052AC0ED047A3CF4B2
:107638002CAC93ED147ADDED177AE7EE267AB0EEEE
:10764800637AA5EE277AB4EEE37AF1EE10FAF0EE5B
:10765800477AB8BFF0EE467AFDEEE77A17EE906A01
:1076680017EE904AAE42A8BF2C468E42B8BF0C46D1
:1076780007EE904AF8EEE77A062AC0ED057A3CF460
:1076880004AC93ED187ADDED187AE7EE267AB0EEC1
:10769800637AA5EE277AB4EEE37AF1EE10FAF0EE0B
:1076A800477AB8BFF0EE467AFDEEE77A17EE906AB1
:1076B80017EE904AAE42A8BF2C468E42B8BF0C4681
:1076C80007EE904AF8EEE77A072AC0ED067A3CF40E
:1076D800DCAB93ED1C7ADDED197AE7EE267AB0EE95
:1076E800637AA5EE277AB4EEE37AF1EE10FAF0EEBB
:1076F800477AB8BFF0EE467AFDEEE77A17EE906A61
:1077080017EE904AAE42A8BF2C468E42B8BF0C4630
:1077180007EE904AF8EEE77A082AC0ED077A3CF4BB
:10772800B4AB93ED207ADDED1A7AE7EE267AB0EE67
:10773800637AA5EE277AB4EEE37AF1EE10FAF0EE6A
:10774800477AB8BFF0EE467AFDEEE77A17EE906A10
:1077580017EE904AAE42A8BF2C468E42B8BF0C46E0
:1077680007EE904AF8EEE77A092AC0ED087A3CF469
:107778008CAB93ED247ADDED1B7AE7EE267AB0EE3A
:10778800637AA5EE277AB4EEE37AF1EE10FAF0EE1A
:10779800477AB8BFF0EE467AFDEEE77A17EE906AC0
:1077A80017EE904AAE42A8BF2C468E42B8BF0C4690
:1077B80007EE904AF8EEE77A0A2AC0ED097A3CF417
:1077C80064AB93ED287ADDED1C7AE7EE267AB0EE0D
:1077D800637AA5EE277AB4EEE37AF1EE10FAF0EECA
:1077E800477AB8BFF0EE467AFDEEE77A17EE906A70
:1077F80017EE904AAE42A8BF2C468E42B8BF0C4640
:1078080007EE904AF8EEE77A0B2AC0ED0A7A3CF4C4
:107818003CAB93ED2C7ADDED1D7AE7EE267AB0EEDF
:10782800637AA7EE857AB4EEE37AF0EE477AF1EE62
:1078380010FAB8BFF0EE467AFDEEE77AFDF781BFA1
:1078480040380020DBF8B45153003DB1981801EBE3
:1078580080006D784078A842BBF4ADAA134401EBD0
:1078680083010023CBF8B411ABF82632CBF82832C9
:10787800FBF7A1BA042303240B930220FDF721B8D8
:107888008300CE180BEB030ECD4B03EBCC1C5FEA49
:10789800980300F0688301331B0106930CEB030087
:1078A80006F110010CF110030EF1100213ED024A5B
:1078B80013ED035A13ED016A13ED047A51ED024AF0
:1078C80051ED035A51ED016A51ED047A64EE244AF0
:1078D80065EE255A66EE266A67EE277A10338342EC
:1078E80042ED024A42ED035A42ED016A42ED047A42
:1078F80001F1100102F11002D8D1069B103B0CEBEC
:107908000302F118734418F003083EF4E5A9B2EC39
:10791800017AF1EC017A67EE277AB8F10108E3EC15
:10792800017AF4D1FEF7D8B99FEDA67AFEF72DBFFC
:10793800B6F95C203CE4B6F9500020E4B6F94400FE
:1079480004E4B6F93800FFF7E8BBB6F92C00FFF7F6
:10795800CBBBB6F92000FFF7AEBBB6F91400FFF7B2
:1079680091BBB6F90800FFF775BB974BB5F90A202C
:107978001B68002B00F0DF821A6001230B93FCF7D1
:107988005FBF924996F916E00B8896F90A20B1F97B
:1079980002008F491EFB03F3524200FB02F081FBF9
:1079A80003E2121181FB00E1DB17C017C0EB2110C5
:1079B800991AD31A01440344791A1C4429806C800B
:1079C800FCF71AB807EE906ADFED826AB8EEE77A3C
:1079D80066EEA65A9FED805A9FED806ADFED807AA9
:1079E800A5EE856A26EEA55AE5EE867AE5EE276AC3
:1079F80026EE870AFEF7C2BEFDEEE37A0DF1480EC9
:107A080017EE909AFDEEC47ACDF840B0CDED0C7A21
:107A1800FDEEC67ACDF84480DFF8D4C1714BDDF8AD
:107A280030B0CDED0D7A17EE908A0EEB82020E95EE
:107A38000F979CED007AFEEC017AE6EE877AB0EEBD
:107A4800637AA5EE277AF0EE477AECB9FDEEC77AAD
:107A58004F4617EE905AA94503DC5D45A8BF5D4621
:107A68002F4607EE907AF8EEE77A002900F0678251
:107A78007245E3EC017A0CF1100CDAD1DDF840B074
:107A8800DDF84480FCF705BA30B1F4EE473AF1EE80
:107A980010FAC8BFF0EE467AFDEEE77A454617EED3
:107AA800907AB84504DC5F4517EE905AA8BF5D464A
:107AB80007EE905AF8EEE77AD7E7FDEEC67A12ABF2
:107AC800CDED0C7AFDEEC47ACDF840B0CDED0D7A4F
:107AD800FDEEE37ACDF84480DFF814E1DFF804C165
:107AE800DDF83080DDF834B00E9517EE909AB1EEDF
:107AF800455A03EB82020F979EED007AF3EC017A68
:107B0800E6EE877AB0EE447AA5EE277AF0EE477A69
:107B1800C4B9FDEEC77A4F4617EE905AA94503DC63
:107B28005D45A8BF5D462F4607EE907AF8EEE77AE6
:107B3800002900F0EA819342ECEC017A0EF1100E74
:107B4800DAD19BE730B1F4EE473AF1EE10FAC8BF4C
:107B5800F0EE467ABDEEE77A07EE908A17EE105AF5
:107B6800A84506DC17EE105A5D45A8BF5D4607EE2E
:107B7800905AF8EEE77ADBE7398F9FED1B7A07EE2C
:107B8800901AF8EEE77A194967EE877AC1ED007A1C
:107B9800FCF738BAB0EE480A22F076FF00B2FFF7D9
:107BA800EFB8B0EE480A22F06FFF00B2FEF773BBE1
:107BB800B0EE480A22F068FF00B2FFF7B1B800BF84
:107BC800405C0020000000002C420020D03B002038
:107BD8001F85EB5184F9223F92E741B99730083C61
:107BE80015A82ABE403800206F12833A00000020F2
:107BF800104100203333333F5FED027A29EE279A94
:107C080028EE278A68EEA77ABDEEC97AFDEEE77AF4
:107C18008DED067A17EE903ABDEEC87AADF84A3087
:107C280017EE101A0A9BBDF91820ADF84C20ADF8D4
:107C38004810002B40F00881CD4B059A0C93118B0E
:107C4800B3F90660FFF7D3B8DFF88883FCF731BAD9
:107C58009FEDC88AFFF790B89FEDC68AFFF75CB81A
:107C6800C54F7A69002A3AF433AFC4493A6808889C
:107C7800C34991FBF0F111607B74FAF729BF9FEDBE
:107C8800C10AC14B0A9325EE800A22F0FDFEBF4EC1
:107C9800DBF8A851F080FDF792BA98ED000A079337
:107CA800069222F0F1FEBA49DFF82CE3D1F8EC1085
:107CB800B64E069A30808EFB013EC917C1EBAE1155
:107CC80007EE901AF8EEE77A079BFDEEE77A17EED3
:107CD800901A7180FCF7F2B907EE906AF8EEE78A1D
:107CE800DFEDAC7A9FEDAC0A8BF8846168EEA78A69
:107CF80038EE800AFDEEC07A17EE903A2033402B1A
:107D080040F22B819FED9B0AA44BFDEEE87A83EDB0
:107D1800010A17EE903A2033402B00F22181DFED63
:107D2800A07AF4EEE78AF1EE10FA40F3BA81DFEDBB
:107D38009D6ADFED9D7A01E0F0EE478AF4EEE78A6E
:107D4800F1EE10FA38EEE67AF6DCDFEDA57AB4EE5D
:107D5800E77AF1EE10FA40F1A1819FED926ADFED2A
:107D6800936A01E0B0EE677AB4EEE67AF1EE10FAC3
:107D780077EE067AF6D49FED887AF4EEC77AF1EEBC
:107D880010FA40F32F819FED867A77EE677A27EE17
:107D9800A76ADFED875ADFED876A9FED877AE6EEFF
:107DA800256A67EE865AA6EE267AE5EE877ACBED47
:107DB800627AFDF7EFBC8149814A8E46FDF77BBFA9
:107DC80006F0BCFD059B714EDBF8AC81DBF8A851D1
:107DD800C01A7080FDF7EBBF09980FF0C3FEFEF7DD
:107DE800BEBB784B1B6803F59C530833CBF8903126
:107DF8003B78012B7DF4D9A89BF88C31002B7DF4BE
:107E0800D4A8B378032B00F04F8110F0FFFE0123B4
:107E18008BF88C31FDF7C9B806F090FD059B5B4ED9
:107E28009AF80070C01A7080FDF712BE06F086FD41
:107E3800059B564E98F80020DBF8A8519AF8007078
:107E4800C01AB080FEF743B8494B0599B3F90660EC
:107E5800098B0C938E42BCBF5242ADF84C20FEF702
:107E6800C6BFDFED4F7AF4EEE76AF1EE10FA40F3A1
:107E7800F180DFED4C5A9FED4C6A01E0F0EE676A45
:107E8800F4EEC66AF1EE10FA76EEE57AF6DCDFED8E
:107E9800546AF4EEE67AF1EE10FA40F1D880DFED9C
:107EA800415A9FED426A01E0F0EE667AF4EEC67A36
:107EB800F1EE10FA77EEA56AF6D4DFED377AF4EE34
:107EC800E76AF1EE10FA04DDDFED357A77EEE66A5F
:107ED8007EE5DFED427AF4EEE76AF1EE10FA44BF90
:107EE800DFED3F7A77EEE66A72E5374B1B7883B3AE
:107EF8000023FEF7FBB9F080A4F8A850FAF762BF98
:107F08002F4901F1800EFDF7C9BF0F9D002D7FF4A9
:107F180012AE0E9DB542B8BFF0EE467A0BE62B4B7B
:107F28001B78002B6DD12A4B1B8B07EE903AF8EE8D
:107F3800E77AFEF75BBA01230B93FCF781BC0F9D30
:107F4800002D7FF495AD0E9DB542B8BFF0EE467A90
:107F58008EE516F055FAFAF72EBF03F0CFFBD3E6FD
:107F6800DFED047A23E7734631466246CBE400BF6F
:107F7800B469002000000000A0530020B85300207E
:107F880020A107000000C842085C00202438002017
:107F98006C15002035FA8E3CDB0FC93F000000202D
:107FA800DB0F4940DB0FC940E4CB1641E4CB16C1D7
:107FB80092E741B99730083C15A82ABEC05D002059
:107FC800701C0020C0530020CD4F002044440020E6
:107FD8001C440020D04F0020D34D6210DB0FC9BFD6
:107FE800DB0F49C01FED037AF4EEC77AF1EE10FA01
:107FF80044BF1FED057A77EE677AC8E6414EFFF772
:1080080011B8DFED417AFEF7F1B99AF800001328AC
:1080180023D04BB105F5F460B0EE480A4844D9F8CE
:108028009C379847B0EE408A9AF80030132B7DF4BD
:1080380000A8B0EE480A22F027FD7880FCF7FBBFC5
:108048009BF8E031002B7AF467ADFAF74EBDF0EEFD
:10805800676A32E7F0EE667A19E7B0EE480A0693E7
:1080680022F012FD069B3880D3E7284AD35C002B08
:108078007EF4ADA9FEF72DBBDFF8A080D8F800008C
:1080880020F0C6FA224B1B780022022BC8F80020E9
:108098007EF49BA920F076F8FEF797B9F0EE477AC0
:1080A80069E6B0EE687A50E6802020F0D7FD002817
:1080B8007CF47BAFA9E60A9BD3ED03DA154B93ED6D
:1080C800020A154B3CEE6DDA28EE800A20EE0D0A06
:1080D80083ED020AFAF7B6BE9BF8D031002BEAD13D
:1080E8000C4B234493ED000A059BD3ED01DA049B66
:1080F80028EE800A3CEE6DDA20EE0D0A83ED000AC8
:10810800FAF7A0BE506800200000000000D0020866
:10811800403A002080670020BC370020602F0020F4
:108128002DE9F04F2DED028B8FB0064616F07EFF3D
:108138009C4B1F7827B10FB0BDEC028BBDE8F08FC8
:10814800DFF8C0B2DBF800305C05F4D5964B974DEC
:108158001B78002B40F05C81954B1B78002B6BD073
:10816800944C954AD4F86431F31A934201F237805B
:1081780094F86C81B8F1000F31D1904F386806F04F
:108188002DFEC0B201280ED9022841F0B3838C4BD2
:108198001A78002A41F0AE85D4F87021B21AB2F5E7
:1081A8007A6F81F0EB86D4F87431002B44D094F8C0
:1081B8006C31BBB9834B1B689B7801211E3B0022A5
:1081C8008B4284F86C1184F8802141F2F485386878
:1081D8000221043016F030FE94F878310FE0D4F81C
:1081E80074314BB3D4F87C3140F6B732F31A93426A
:1081F80022D994F87831002B01F0B1826F4F013BFE
:10820800DBB284F87831002B01F04280D4F8741185
:1082180094F8802111F801EB94F88131C4F87411B5
:1082280072440133386884F88021714684F88131BA
:1082380006F0D8FDC4F87C61634B2F681B7853B1F6
:10824800DFF8C481D8F8000028B1604B1B78013BE7
:10825800012B41F22C805E4B1B7863B15D4F3B686C
:108268004BB1544CD5F80090D4F8B832A9EB0303BD
:10827800632B00F21987584C2378022B01F05082A7
:10828800DFF8888198F80030032B00F0ED87534B16
:108298001B7873B1524F3B685BB1464C06F04EFBFE
:1082A800D4F8C032009044F61F62C31A934200F219
:1082B8007B814C4B1B78002B4BD14B4B1B7843B12C
:1082C8003C4CD4F8103403F5C333A0339E4280F0FD
:1082D8004787464B1B78002B3FF42DAF354E444C57
:1082E800444D06F23147206806F078FD00283FF437
:1082F80022AF206806F06AFD2B7880465A1E33B1FB
:1083080020682A7006F06AFD0028F2D113E70322DC
:108318003946781E24F0ABFC96F8303496F83124B0
:1083280086F8338483F47F4383F0FF039B1A1FFA94
:1083380088F89BB2B8EB132FD5D196F83224DBB26C
:108348009A42D0D1781E16F089FC2B7818442870F0
:10835800C9E7294C2278002A40F0E686154CD4F863
:10836800083403F5C333A0339E42A6D3234A94F8B6
:108378000C34C4F80864D55CE90701F1AE83AA0798
:1083880001F16A836B0701F181821D4A94F80C346C
:108398001178013393FBF1F201FB123384F80C34AA
:1083A8008BE700BFDE6900203C500020C05300204E
:1083B80046500020A41E00203F0D0300E04F00207F
:1083C80008000020E44F00204850002050500020B2
:1083D800585000209C7700209227002060500020F1
:1083E80064500020CC500020DA5000206A50002051
:1083F800705000207450002034500020D4500020C9
:10840800D95000204C490020984F00207D000020C2
:108418005B4C2A68D4F85C31D31A7C2B7FF69CAE6F
:1084280094F86031DFF878919FED568AC4F85C21A2
:10843800013384F860314FF02408404616F0A4FD5B
:10844800514BF9EC016A1B8A07EE103AF8EEE66A1E
:10845800B8EEC77A08F10108C6EE877A5FFA88F89D
:1084680067EE887AFDEEE77ACDED007ABDF900A0D7
:108478005FFA8AF016F064FDCAF3072016F060FD73
:10848800B8F1270FD9D1302016F07EFDDFF814811E
:10849800002016F055FD002016F052FDD8F8000017
:1084A8005E2106F09FFC94F8603113F003092DD18A
:1084B800D4F85C2141F288339A4201F20A851420EB
:1084C80016F062FD314B324AB3F9043082FB0312D5
:1084D8004FEAE379C9EBA2090FFA89F95FFA89F043
:1084E80016F02EFDC9F3072016F02AFD1C2016F001
:1084F8004BFD002016F024FD002016F021FD5E2122
:10850800D8F8000006F06EFC94F86031580701F0C6
:108518005B83282B7FF420AE00271720D5F8009026
:1085280084F8607116F030FD384616F009FD194BD5
:10853800194CA3FB09239B0BA4FB03125209C2EBA2
:108548000212A3EB8203D8B216F0FAFC182016F038
:108558001BFD124BA3FB09239B09A4FB0312520921
:10856800C2EB0212A3EB8203D8B216F0E9FC38463C
:1085780016F0E6FCD8F800005E2106F033FCEBE5C7
:10858800A41E002000007A44E0370020D03B0020E1
:108598006766666673B2E74589888888D34D621036
:1085A80014380020E84F002094F8C632002B41F020
:1085B8004B81E34B1A6802F00803002B48F603418D
:1085C8004AF60B404BF60F4349F6074804BF0346EB
:1085D800884612F0040F4FF0190118BF984692060A
:1085E80084F8C61203D548F4804848F02008D54BD3
:1085F8001A79C8F309010191002A41F0FD845B79D9
:10860800002B41F049869A4664204FF0FF330A4612
:108618004FF00009CDF81880CDF81C800892ADF80D
:1086280026A0ADF828308DF83600ADF82490CDF8A6
:108638002A90CDF82E90CDF832900DF1180CBCE8A8
:108648000F00DFF810E384F85190AEE80F009CE8C3
:108658000F00AEE807002EF8023B71464FF0010C00
:108668001B0C4FF0FE0E1F20C82201F81E3984F89B
:108678004EE084F8522084F853C084F84F0094F8F0
:10868800D60284F8500080F0F10383EA0313DAB2CB
:10869800130983F0E70343EA022383EAC2031BB208
:1086A80083EA0312D2B2C3F3072383EA121343EA1D
:1086B800022383EAC2031BB283F0C80282EA0212D1
:1086C800D2B2C3F3072383EA121343EA022383EAED
:1086D800C2031BB283EA0C0E8EEA0E1E5FFA8EFEF0
:1086E800C3F3072282EA1E1242EA0E22604482EA9B
:1086F800CE0E84F8D602A4F84CE001F11F0011F860
:10870800013B83EA0E0383EA0313DBB21A0982EA08
:108718001E2242EA032282EAC3031BB21FFA83FE27
:108728008142A4F84CE0EAD183F07C0383EA031386
:10873800DBB21A0982EA1E2E8EEA032E8EEAC30ED7
:108748000FFA8EFE1FFA8EF34FEA132A5FFA8EFE97
:10875800A4F84C30DFF8009284F874A004F16E039A
:1087680084F873E004F14E0C0193DCF80C30DCF86B
:108778000000DCF80410DCF80820C846A8E80F0060
:10878800019B0CF1100C9C45C146EED1DCF80000B1
:10879800C8F80000DFF8C4819CF8043089F8043078
:1087A80008F1270984F825E384F826A318F8011F9F
:1087B800386806F017FBC145F8D194F8C722002A9B
:1087C80041F0478060492B6808780A2184F8C7126D
:1087D800002801F03781DFF888C10128BCF80010B3
:1087E800059141F25085BCF802100291022801F06F
:1087F8001F84BCF804100391032801F08F85BCF88E
:1088080006100191042801F06F850528BCF80810AE
:1088180001F065850628BCF80AA001F05C850728E8
:10882800BCF80CE001F02485BCF80E9094F8D62230
:108838000693104680F0300383EA0313DBB20490FA
:10884800424A9DF810C0128884F850C0180980F078
:108858007A0040EA032080EAC3033D48C2EB0222C3
:1088680080FB02C01044D217C2EB602205988DF835
:108878002D204FF0000860F30F0803984FF0000C0C
:1088880060F30F0C00201BB261F30F0000216EF3A0
:108898000F0183EA031EC3F307230393029B63F3C9
:1088A8001F48019BCDF81C8063F31F4C039BCDF838
:1088B80020C05FFA8EFE6AF31F4069F31F4183EA06
:1088C8001E134FF0000A09900A918DF82CA043EA74
:1088D8000E2C0DF11809B9E80F008CEACE0E0FFA2C
:1088E8008EFE8EF0C808DFF86CC084F851A088EAC4
:1088F80008185FFA88F8CEF3072EACE80F008EEA66
:10890800181E4EEA082399E8030083EAC8080FFAFC
:1089180088F383F023024CF8040B82EA0210C0B2F9
:10892800C3F3072282EA1012049B2CF8141942EAB6
:108938000022591C82EAC0004FF02308162211E0D9
:10894800185C002058690020F86300205069002056
:1089580003082080F81E0020A4210020A321002065
:10896800B46900204FF0FE0EC82384F8D612A4F88C
:108978004C000CEB020184F8538084F84EE084F834
:108988004F2084F852301CF8013B434083EA03131C
:10899800DBB21A0982EA102242EA032282EAC303FE
:1089A8001BB298B28C45A4F84C00ECD183F0F403C8
:1089B80083EA0313DBB24FEA131E8EEA102E8EEA07
:1089C800032E8EEAC30EA0460FFA8EFE1FFA8EF90A
:1089D80058F84E0FDFF81CC4A4F84C904FEA192A37
:1089E8005FFA8EFE84F86AE084F86BA0D8F8041069
:1089F800D8F80820D8F80C30ACE80F00D8F81000E8
:108A0800D8F81410D8F8182004F21D39ACE807007B
:108A180004F2FF2884F81DA384F81CE318F8011F4A
:108A2800386806F0DFF9C145F8D194F8CEE2BEF116
:108A3800000F40F01787E84B94F8D6C2B3F900103E
:108A4800B3F90220B3F904309FEDE46A84F851E0E9
:108A580007EE103A2B6806938CF06A0383EA031337
:108A680006EE901AD9B20B0983F0D50343EA012325
:108A780083EAC1031BB283EA03115242C9B207EE6B
:108A8800902AC3F3072383EA111343EA0123F8EE7C
:108A9800E77AF8EEE66AB8EEC77A83EAC1031BB252
:108AA80067EE867A66EE866A27EE067A002083F0FD
:108AB800C805CDED087ACDED076A8DED097A0A90E3
:108AC8000B900C9085EA05150DF11809EDB2C3F36A
:108AD8000728B9E80F0088EA151848EA052888EA3F
:108AE800C505DFF814832DB2A8E80F0085F01E0E27
:108AF80099E807008EEA0E13DBB2C5F3072E8EEA5B
:108B0800131E4EEA032E88E807008EEAC30EA8F16A
:108B180010051C20C8214FF005091E234FF0FE0840
:108B28000CF1010284F8521084F8CE9284F8533084
:108B380084F84E8084F84F00291884F850C0A4F8AF
:108B48004CE084F8D62215F8013B83EA0E0383EA49
:108B58000313DBB21A0982EA1E2242EA032282EADE
:108B6800C3031BB21FFA83FE8D42A4F84CE0EAD17E
:108B780083F0270383EA0313DBB21A0982EA1E2E65
:108B88008EEA032E8EEAC30E0FFA8EFE1FFA8EF3BC
:108B98004FEA13295FFA8EFEDFF85882A4F84C30AA
:108BA80084F8719084F870E004F14E0C04F16E0AB8
:108BB800DCF80000DCF80410DCF80820DCF80C30E5
:108BC80045460FC50CF1100CD445A846F0D1844D8C
:108BD800BCF80030A8F8003005F1240884F822E336
:108BE80084F8239315F8011F386806F0FBF845450B
:108BF800F8D194F8CF320193002B40F02F8694F8E7
:108C0800D682754B774AB3F90410B2F90620DFF81B
:108C1800ECC1754DDFF8E09184F8508088F02203AC
:108C280083EA0313DBB2180980F05900B2F5FA6F32
:108C380040EA032080EAC303A8BF4FF4FA621BB2DC
:108C4800B2F57A7F83EA0310B8BF4FF47A72C0B2E4
:108C58004FF0640EA2F57A72C3F307230EFB02F2FB
:108C680083EA101385FB02E543EA00238CFB01CE5F
:108C7800D217C9174FF0000AC2EBA512C1EBAE011B
:108C880083EAC0031DB2CDF818A00DF1180CADF899
:108C98002A20ADF82810CDF81CA0CDF820A0CDF8DA
:108CA80024A085F0C80ECDF808C0BCE80F008EEAF5
:108CB8000E1E5FFA8EFEC5F3072585EA1E1545EAE6
:108CC8000E25A9E80F0085EACE0212B282F04A0307
:108CD80083EA0313DBB2C2F3072181EA1311DCF83C
:108CE800002049F8102941EA0321052081EAC3033D
:108CF800142508F101029DF8041084F8CF024FF002
:108D08004A0C4FF0FE0EC82084F8511084F8D62281
:108D180009EB050184F84F50A4F84C304A4684F812
:108D280053C084F84EE084F852001D4612F8010B37
:108D3800684080EA0010C0B2030983EA152343EAB9
:108D4800002383EAC00000B285B28A42A4F84C50DE
:108D5800ECD180F0140080EA0010C0B24FEA101E77
:108D68008EEA152E8EEA002E8EEAC00E25460FFAE0
:108D78008EFE1FFA8EF855F84E0FDFF878C0A4F86B
:108D88004C804FEA182A5FFA8EFE84F869A084F8AE
:108D980068E06968EB68AA68ACE80F002869696947
:108DA8002B8BACE8030004F2FF25ACF80030A84692
:108DB80084F81BA384F81AE304F21B3A18F8011F7D
:108DC800386806F00FF8C245F8D1084B084A1B78F6
:108DD8001278013B14E000BFD03B002088C3E43A7E
:108DE800A3210020B4690020D34D6210603A00200E
:108DF80035690020A4210020F81E002067666666F9
:108E080012F00100DBB214BFC0224022172B04D895
:108E1800CA490B4493F824300193C94B19888B072E
:108E28001ABF002342F01002012311F4027F18BF79
:108E3800022311F0100F18BF062311F0200F18BFDE
:108E48001023002841F05980032194F8D6E20693B4
:108E58008EF0460383EA0313D8B2030983F0920322
:108E680043EA002383EAC0031BB283EA0310C0B2BB
:108E7800C3F3072888EA101848EA002888EAC008D7
:108E88000FFA88F888F0C80C9DF804008DF81C00CB
:108E98008CEA0C1C00235FFA8CFC8DF81E20032042
:108EA800029A8DF81D30C8F307288DF81F108DF829
:108EB800200088EA1C1807CA48EA0C2888EACC0C63
:108EC8000FFA8CFC8CEA0C18A9E803005FFA88F802
:108ED800CCF3072181EA181141EA082181EAC80880
:108EE80094F854C089F800200FFA88F28CEA020C32
:108EF8008CEA0C1C5FFA8CFCC2F3072282EA1C1273
:108F080042EA0C2294F8550094F8561094F85790B9
:108F180094F8588084F8533082EACC0212B2504058
:108F280080EA0010C0B2C2F3072282EA101242EAB5
:108F3800002282EAC00212B2514081EA0111C9B28C
:108F4800C2F3072282EA111242EA012282EAC1022E
:108F580012B289EA020989EA09195FFA89F9C2F3A2
:108F6800072282EA191242EA092282EAC90212B2E7
:108F780088EA020888EA08185FFA88F8C2F3072224
:108F880082EA181242EA082294F859C094F85A0062
:108F980094F85B1094F85C9084F8513082EAC80227
:108FA80012B28CEA020C8CEA0C1C5FFA8CFCC2F33D
:108FB800072282EA1C1242EA0C2282EACC0212B28E
:108FC800504080EA0010C0B2C2F3072282EA1012B1
:108FD80042EA002282EAC00212B2514081EA01113B
:108FE800C9B2C2F3072282EA111242EA012282EAD6
:108FF800C10213B289EA030282EA0212D2B2C3F3AF
:10900800072383EA121343EA022383EAC2031BB24B
:1090180083F0320282EA0212D2B2C3F3072383EA50
:10902800121343EA022383EAC2031BB29AB24FF037
:10903800FE0CDFF8208184F850E00920C8210EF1E9
:10904800010EDBB284F84EC04FEA122C84F84F00B0
:1090580084F8521084F8D6E2A4F84C2084F85EC054
:1090680084F85D30D8F80000D8F80410D8F8082043
:10907800B8F80CA008F2B22EAEE8070008F2C22831
:109088008EF80290AEF800A084F810C384F80F336D
:1090980015F8011F386805F0A5FEA845F8D1009B12
:1090A800C4F8C032FFF705B9DFF8ACA0DFF8AC8030
:1090B800412015F073FEBAF9023088FB0320DB1754
:1090C800C3EBA00080B215F04FFEBAF9003088FB60
:1090D8000320DB17C3EBA00080B215F045FEBAF9F8
:1090E800043088FB0320DB17C3EBA00080B215F027
:1090F8003BFE144B3868197805F074FE94F8BC32BE
:1091080013F0010800F0FD830F4AC4F8B892013348
:10911800DBB2A2FB0312D20802EB8202A3EB4203EA
:1091280084F8BC32FFF7A7B8084B0949186805F05E
:1091380029FE00232370FFF711B900BF44D20208AB
:10914800DC690020507C0020CDCCCCCCD050002055
:1091580010500020F21E0020D03B00206766666693
:1091680094F81434BA4AC4F8106402EB8302D26B40
:1091780042B30EAD04F21B43B64E45F8203D002124
:1091880004F22D433180079380211523A52784F805
:109198001A34284684F8191484F818749047284615
:1091A800318802F09BF9069DAB4804F583616D1A7E
:1091B800152DA8BF15252A4621F0F2FAA74A94F8DA
:1091C80014341570A64A013382FB0312A2EBE37232
:1091D80002EB42029B1A84F81434FFF77AB8A14BC9
:1091E800A14AD4F868112868128893F80BE09F4BBD
:1091F800401A4FF47A71D7B201FB0EF1120A9F7729
:109208001F7588424FF00007DA775A759F701F71F3
:1092180080F02E83964A974811689268C4F8646172
:1092280080FB01E7C91780FB02E0C1EBA701D21759
:10923800C2EBA00208124FEA222C4FF0F40E197765
:109248000127587783F8202030207521782283F869
:1092580021C083F81AE0DF7683F8220083F8231010
:1092680083F82420FEF784BF834F386803685B695E
:10927800984700283FF40BA83868036801219B69C8
:1092880098470222002388F800202370FEF7FFBFCA
:1092980094F8801194F8813138684A1C013384F8B5
:1092A800802184F8813105F09DFDFEF7C3BF734C22
:1092B800DFF8D0914FF0000A0BE01B2B00F043823F
:1092C8000D2B00F00C824FF0010389F80130D8F81B
:1092D800000005F083FD002837D0D8F8000005F01D
:1092E80075FD83B27E2B2A6828D099F80120002AC0
:1092F800EDD194F882110029DFD07D2B00F0038294
:1093080094F886E1BEF1000F04D080F02003DBB2B0
:1093180084F886214A1CD2B2092A635484F882212F
:1093280000F0E581082AD2D8B4F88421134403EB6D
:10933800132303F0FF03A4F88431C8E784F882A15B
:1093480084F883A189F801A0C1E794F887312BB18B
:10935800637884F88701302B00F04B8594F88321DB
:109368003B4BDFF82491DFF824C1DFF824A14FF04C
:10937800010E002A3EF46FAF2968C91B012900F2CB
:10938800A98194F89C82B8F1000F40F0F38194F819
:10939800B41233F8110010B984F8B4E2E9E70131E6
:1093A800B0F5826F84F8B41200F018811ED9B0F5B8
:1093B800E26F00F0BC8033D9B0F5046F00F0C580CF
:1093C800B0F5116F00F0CD80B0F5E46FD1D12C4A23
:1093D800D76B118A642303FB07F393FBF1F115F0B4
:1093E80011FD002384F88331FEF735BFB0F5007F07
:1093F80000F0D1804ED8B0F5807F00F04281B0F502
:10940800887FB6D1D9F800104907B2D500214FF4AA
:10941800887015F0F7FC002384F88331FEF71BBF32
:10942800B0F5C06F00F0CA80B0F5E06FA1D1144A62
:10943800506B118A642303FB00F34FF4E06093FB45
:10944800F1F115F0DFFC002384F88331FEF703BF48
:1094580044D20208804F0020B8620020CD6200206C
:10946800565555559C4F0020844F002078500020B9
:10947800884F00206766666628280020A41E002002
:10948800E037002008000020185C00205869002000
:10949800CD4F0020B0F5047F00F00281B0F5806F59
:1094A8007FF467AF94F8B5320133DBB2032B00F2D7
:1094B8002F8142F2107184F8B53201FB03F1BD4BE4
:1094C8001B88002B40F02A810131BB4B1B78D80741
:1094D800BA4B1B8848BF0431DA0748BF0A319807DE
:1094E80048BF14311A0648BF2831D80548BF28316B
:1094F8005A0748BF6431180748BFC8319A0548BFA2
:1095080001F5C871980648BF01F57A71DA0648BFB7
:1095180001F5FA61580648BF01F57A614FF4806099
:1095280015F070FC002384F88331FEF794BEA44A3A
:10953800976B118A642303FB07F393FBF1F115F092
:1095480061FC84F88381FEF786BE9E4BB3F9041054
:1095580001EB8101490015F055FC84F88381FEF781
:109568007ABE9CF8041000293FF403AF9AF8001063
:1095780000293FF4FEAE944B1B8803EB83035B008A
:109588004FF4116093FBF1F115F03CFC002384F8D3
:109598008331FEF760BE9CF8051000293FF4E9AE60
:1095A8008A4B8B491B6881FB0321DB17C3EBA101A5
:1095B80015F028FC84F88381FEF74DBE9CF8051051
:1095C80000293FF4D6AE814B4FF4C060996815F07E
:1095D80019FC002384F88331FEF73DBED9F800104A
:1095E80011F020087FF4C5AEDBF80010090600F181
:1095F800EA837849097B00293FF4BBAE94F8B61298
:10960800032900F2D985DFE801F032281902724BEC
:109618001B6859799A79DB7901F1407101EB0221D4
:1096280001EB0341002384F8B6324FF4826015F051
:10963800E9FB002384F88331FEF70DBE674B1A68F7
:10964800137A507992781B0403EB002313444A1CC5
:1096580084F8B62203EB0161E7E7604B1A68D37917
:10966800107952781B0403EB00231344EFE75B4B9C
:109678001A689379D07812781B0403EB00231344FB
:10968800E5E7D9F8001048077FF573AE00214FF4DD
:10969800807015F0B7FB002384F88331FEF7DBBD3B
:1096A8009CF8041000293FF464AE9AF800000028E2
:1096B8003FF45FAE474B5B7B002B00F00684424BC8
:1096C800198891FBF0F101EB810149004FF4047016
:1096D80015F098FB002384F88331FEF7BCBD4FF0EA
:1096E800010284F882212370A4F88411EFE5B4F80C
:1096F8008421C2F1FF0293427FF4E5AD4FF00103EC
:1097080084F88731DFE54FF0010384F88631DEE520
:10971800012384F8B53242F21071D0E60231D4E662
:1097280005F00CF92E4B1A6840F6B833801A9842A7
:1097380000F27E812B4F3B793A2B00F0E182002327
:109748002370FEF7A4BDD8F8000005F047FB0028F9
:109758007FF4B9AD4FF0010384F88331B7E5C4F85D
:10976800743184F86C31204F15F096FB94F87831F9
:10977800FEF745BDD4F88C32DFF8709094F8B22229
:109788004B4500F01884511C94F8B3E2D4F890C209
:1097980084F8B21202F00F028DF818200DF11902A8
:1097A800ACEB0301002940F3128506A902910DF1E3
:1097B8001E0720E08869002035690020DC69002048
:1097C800E0370020D03B0020844F0020884F002045
:1097D800676666669C4F0020406E0020A82800201F
:1097E8009827002080270020E04F0020302000200C
:1097F800002840F31A810133C4F88C3213F8011C95
:1098080002F8011BBA42ACEB030081EA0E0EEFD35B
:1098180084F8B3E200F0CA84501CB84282F800E031
:1098280005D20EAB9A1A1B3A002123F03AFA029994
:10983800322015F0CBFA4FF00008002384F89C8200
:1098480084F88331FEF707BD013B84F8C632FEF782
:10985800B4BF013A84F8C722FFF7E7B8013B84F8A0
:10986800CF321CE40EF1FF3E84F8CEE2FFF7C1B917
:10987800C04A29681278C4F86811013A012A3FF6EB
:10988800C9AC1021022299701A71C3E4BA4ABB4BC1
:1098980012680793A3F1240800202121D50003F8BA
:1098A800240C88F8021040F10483B5490327B54B0E
:1098B8001B88580500F1FA82DA0700F1C18303F02A
:1098C8000203B14A002B1CBF03271146AF4D3A468D
:1098D800284620F065FF7B190EA80133A91E40F821
:1098E800203D00225B1A7A5588F8013015F05CFBA0
:1098F800FEF74BBD15F0C2FAA54B01221A70FEF710
:1099080052BCA04B1B88DA0515D4D80600F18D830C
:10991800990600F137845A0600F18784180700F188
:10992800A384D90700F18D8413F0020F0CBF4FF008
:1099380004084FF00C08974B974A1B78D27803F02D
:1099480001030AB143F002035320009315F026FAED
:10995800924A128802EB820202EB8202900080B2E5
:1099680015F002FA002015F0FFF98D4A8D4912888A
:109978003868C2EBC212520081FB023111444FEA2F
:10998800E27ACAEB612A5FFA8AFA514605F02AFAA6
:10999800854B38681A78009B48EA0308824B8AEAA4
:1099A800020A002183F800A005F01CFA4146386835
:1099B80005F018FA7C4B7C4A1B78386888EA030360
:1099C800DBB21946137005F00DFA94F8BC32002B7F
:1099D8007FF49AAB4F2015F0E1F91FF09BF91FF0C7
:1099E80099F91FF097F90121386805F0FBF96F4ADA
:1099F8006D4B92F800801B786B4A386808F00108B4
:109A0800414683F00103137005F0ECF9664B3868A2
:109A18001B7888EA0308644B414683F8008005F008
:109A2800E1F994F8BC32FFF76FBB84F8B3E2F3E6D0
:109A38005F4AB2F8BE3200210133A2F8BE3221706B
:109A4800FEF725BC864682460146019003900290A7
:109A580005908146FEF7EABE484B504907930EAF82
:109A6800A3F1210047F8200D4FF0080E4FF0000831
:109A78000A2003F822EC03F8230C03F8248C384658
:109A8800098801F007FD4B4B4B491B6881FB0321FB
:109A9800DB17C3EBA101384689B201F0FBFC474B49
:109AA800B3F806900DF038FF069B5A1C069283F80F
:109AB8000080069B4FEA1922591C06911A70069BD2
:109AC8005A1C069283F80090069B5A1C069218703E
:109AD800384615F069FAFEF755BCDFF8E8809FEDC7
:109AE800388AB8F90230254A079207EE903AF8EE1C
:109AF800E77A0EAF67EE887AA2F12403FDEEE77AE3
:109B0800A2F12101002047F8201D02F8240C0822A8
:109B1800CDED007A5A701E229A70BDF800103846B2
:109B280001F0B8FCB8F9003007EE903AF8EEE77AA1
:109B3800384667EE887AFDEEE77ACDED007ABDF813
:109B4800001001F0A7FCB8F9043007EE903AF8EEDF
:109B5800E77A384667EE887AFDEEE77ACDED007A47
:109B6800BDF8001001F096FC384615F01DFAFEF716
:109B780006BC00BF53690020F039002010500020B7
:109B880018F40208DC69002030F40208EF4F0020C6
:109B9800080000203569002064690020844F0020F7
:109BA8005069002003082080507C0020F0640020C9
:109BB800A41E0020884F002067666666586900204A
:109BC80058A08B41D03B0020022015F0DDF9D64B80
:109BD800D64AB3F9443082FB03124FEAE379C9EB62
:109BE800A2090FFA89F95FFA89F015F0A9F9C9F302
:109BF800072015F0A5F9032015F0C6F9CC4B1B7802
:109C0800D90740F182811DF0B5FCCA4B9FEDCA7A95
:109C1800D3ED037A67EE877AFCEEE77ACDED007A2A
:109C2800BDF80030002800F0A682DFB24FEA132901
:109C3800384615F085F9484615F082F9DFF824937F
:109C480099F80430002B40F0FE810DF118094946BF
:109C5800BA4815F039F9132015F096F9BDF91870BE
:109C6800F8B215F06DF9C7F3072015F069F91B2054
:109C780015F08AF9BDF91A70F8B215F061F9C7F351
:109C8800072015F05DF9232015F07EF94E2015F018
:109C980057F9002015F054F94946A84815F014F969
:109CA800122015F071F9BDF91870F8B215F048F9DD
:109CB800C7F3072015F044F91A2015F065F9BDF926
:109CC8001A70F8B215F03CF9C7F3072015F038F907
:109CD800222015F059F9452015F032F9002015F029
:109CE8002FF95E21D8F8000005F07CF894F860316F
:109CF800FEF70FBCC4F8706183F80080FEF753BA12
:109D0800BB78DBB103F1FF3C5FFA8CFC0CF1010C72
:109D1800BC44BE4600221EF8013B534083EA0313AD
:109D2800DBB2120AD90042EA0322F44581EA13138E
:109D380082EA0302EFD1002A7FF401AD804B814A09
:109D4800DFF824E21968804B1288DFF82082D1F806
:109D580030C0CEF818201A68B8F8BE829B68CEF8D2
:109D680028200022CEF86800CEF84830CEF83820F7
:109D7800CEF85880BCF1000F00F06782DCF80430A0
:109D8800086C83423BBFCA681B1A1B1A9B18002B1E
:109D98007EF476AA0B68DFF8D8819B690846022111
:109DA80098470423F87888F800300AF08FF90323DD
:109DB8002370FEF767BA0221386805F003F894F8B3
:109DC8007831FEF71CBA10230422184606A98DF82C
:109DD8001A808DF81B808DF81C808DF81D808DF8F9
:109DE80018308DF8192014F0F1FF84F88381FEF7FC
:109DF80032BAA3785A09012A40F0AB8103F00F0C5C
:109E080013F0100300F0C281DFF86881E37894F85A
:109E180004E0A4F8AA0208EB03018EEA030084F820
:109E280088214346C4F8A082C4F8A412A8F1070206
:109E380084F8B002A4F8A8E294F8B002DFF83881F8
:109E480086460CE012F8011BC4F8A002424581EADC
:109E58000E0E197007D2D4F8A412D4F8A032994281
:109E680003F10100EED1424584F8B0E200F01C8213
:109E7800127894F8B0329A4200F0AF81334BC4F8AC
:109E88008C3200220133B4F8A812C4F8903284F856
:109E9800882101234FF6F672A4F8941284F88C31C5
:109EA80084F89C32A4F89622FFF758BA0327284969
:109EB8000CE5DBF80030274A274903F48003834286
:109EC8000ABF114603270427F1E41E4B1988FFF740
:109ED800FABB102015F058F8484615F031F84846F6
:109EE80015F02EF8212015F04FF8484615F028F8FF
:109EF800484615F025F8FEF7E2BA1849C97800294E
:109F08000CBF04210521FEF7A0BFDFF85890144BC1
:109F1800B9F80670A3FB0737BF08F8B215F010F8B8
:109F2800380A15F00DF88BE6E4530020676666667C
:109F380035690020D04F0020CDCC4C3E809698004B
:109F480028280020844F0020884F0020302000203F
:109F580024F402081CF4020818F4020864690020BA
:109F6800CDCCCCCC586900200C000020A41E0020C9
:109F78007D000020B01E0020AC1E002001223868A1
:109F88001A7004F023FF8046386804F01FFF18F0A9
:109F98007F0F7EF408A98E287EF405A994F86C3109
:109FA800002B7EF41CA9D34BC4F874312D2384F8FC
:109FB8007831FEF7FFB8B4F99612D4F890C294F845
:109FC80094E2501C02F00F0242F010020029B8BFC0
:109FD80042F020028DF81820ACEB090282EA0E0E3E
:109FE8005FFA8EFE8DF8192084F8B20284F8B3E285
:109FF8000DF11A02FFF7D4BBBF495A790B8803EB5E
:10A00800830303EB83034FEA830A1FFA8AFA002AC1
:10A0180000F04E81B94B1B681BB202930DF07CFC1B
:10A02800029B019A40B2FEF7F3BA4FF0340882E47B
:10A03800964692461146019203929146FEF7F6BB68
:10A04800AF49042742E4DFF8D0A29AF80020002A9A
:10A058003FF4FBADB4F86271A74B00921B883F0137
:10A068006421BFB201FB03235100B3FBF1F347EABC
:10A078000327BFB2C3F303231F43062014F084FF52
:10A08800F8B214F05DFF380A14F05AFFB4F86231E0
:10A09800994A9C491788009A01339BB293FBF2F0C6
:10A0A80002FB1033487AA4F86231012800F00981D4
:10A0B8004B7B6E2202FB07F7152297FBF2F7002B6A
:10A0C80040F0F9803A2014F05FFFBFB24FF0640A05
:10A0D800B7FBFAF293B2D8B20192009314F030FFB2
:10A0E800009B180A14F02CFF3B2014F04DFF019A36
:10A0F8000AFB127080B20A23053090FBF3F0C0B25D
:10A1080014F01EFF002014F01BFFDFF8F0A1282038
:10A1180014F03AFF0A23DAF8007097FBF3F7F8B265
:10A1280014F00EFFC7F3072014F00AFF042014F000
:10A138002BFFB9F80630002B7BD1DAF8087087F3CB
:10A148001007F8B214F0FCFEC7F3072014F0F8FE6D
:10A158007BE56D4B6D4AC4F88C32591C012384F899
:10A16800880184F88C01C4F89012C4F8942284F809
:10A178009C32FFF7F3B8DBF80020D2067FF555AD27
:10A18800814655E54FF02408FFF7D5BB94F88821A0
:10A19800002A3FF4E3A894F8B122013202F00F023A
:10A1A80062455BD084F88831FFF7D8B8029932202D
:10A1B80014F00CFEFFF741BB4B1CDBB2042B84F8F8
:10A1C800B6324FEA01617FF430AAFFF72BBA06AB2B
:10A1D80002930DF11E07FFF71FBB4D4BD4F8A022C9
:10A1E800C4F8A4224FF0000E03F52072114603F5BF
:10A1F800C079C4F8902203F525707246C4F8A032DD
:10A20800C4F894E2C4F88C9284F888E1F5F7B8FFB2
:10A21800013030D0D4F88C32C4F890320123C4F81D
:10A228008C9284F89C32FFF799B84FF01008FFF72A
:10A2380082BB0DF071FB14F083FE002014F080FE49
:10A2480003E54FF00808FFF776BBC8690B6A984228
:10A258003BBFCA681218C31AD31A98E5D4F8A412D7
:10A26800D4F8A0322B4AE7E54FF02008FFF763BB8C
:10A278009146FEF7DBBAD4F88C320222591CC4F896
:10A288008C121A70C6E796469246114601920392BE
:10A2980002929146FEF7CABA184B9246B3F90030BB
:10A2A80064200A46FEF7B4B984F8B1C2FFF756B87D
:10A2B8004FF0FF33B0E6BFB29AF8003097FBF3F7E0
:10A2C80000E7392014F060FEF8B214F039FE380ABD
:10A2D80014F036FE19E796469146FEF7A7BA964659
:10A2E80092469146FEF7A2BA964692461146914684
:10A2F800FEF79CBA78500020844F0020884F002039
:10A3080028F402089C4F0020302000200000F6FFAF
:10A31800B01E0020A71E0020CD4F00209646924672
:10A32800114601929146FEF781BA00BF2D23437072
:10A338002E2303712F23C37170472DE9F041446820
:10A3480014B12568A4882C8541F08001046840F286
:10A35800E93501E0002D51D02689013D16F0020FA4
:10A36800ADB2F7D0217304F10C0640F2E93101E0F7
:10A3780000294DD02589013915F0010F89B2F7D090
:10A3880031780468A1894FF0000C4FF47A714FF6C8
:10A39800FF764FF0FF0E624502D127E0B1421CD094
:10A3A80025890139AF0789B2F8D584F80CE004F1A2
:10A3B8000C084FF47A7102E0B9B2B1420DD0258988
:10A3C800ED0701F1FF37F7D598F80050EDB20BB162
:10A3D8001D7001330CF1010CDDE7134B9C4205D1D4
:10A3E800124A538B01339BB25383538B436813B187
:10A3F8001A689B8893610120BDE8F0810A498C4264
:10A40800C0D10A4D698B013189B26983698BB9E77B
:10A4180005498C42B5D1054C618B013189B2618304
:10A42800618B0468AEE700BF003800405853002035
:10A4380030B4436813B11C689B882385036840F2D5
:10A44800E93401E0002C3FD01D89013C15F0020FD2
:10A45800A4B2F7D0197303F10C0540F2E93101E019
:10A4680000293BD01C89013914F0010F89B2F7D0BB
:10A478002B78036840F2E93100E0D9B11C89013931
:10A4880014F0020F89B2F8D01A7303F10C0440F2E9
:10A49800E93200E072B11989013A11F0010F92B264
:10A4A800F8D02378436813B11A689B889361012018
:10A4B80030BC70470F4A9342F4D10F4A538B013393
:10A4C8009BB25383538BEDE70A498B42D2D10A4C96
:10A4D800618B013189B26183618BCBE705498B427E
:10A4E800C7D105494B8B01339BB24B834B8B036818
:10A4F800C0E700BF0038004058530020002870B55E
:10A508001EDB0928044620DD012303EB83035B00DF
:10A51800B0FBF3F2092AF8D87BB10E4EB4FBF3F086
:10A528000928CCBF57223022A6FB03E5024403FBCF
:10A538001044EB0801F8012BF0D100230B7070BD1B
:10A548002D230B7040420131DBE7303001F8010B5D
:10A55800F3E700BFCDCCCCCC884230B44FF0010437
:10A568002ED301FB04F4B0FBF4F58D42F9D284B18B
:10A57800AAB901E0B0FBF4F5092DCCBF572230226F
:10A588002A4404FB150003F8012BB4FBF1F4002C5A
:10A59800F0D100221A7030BC7047B0FBF4F5092DD9
:10A5A800CCBF372230222A4404FB150003F8012BC4
:10A5B800B4FBF1F4002CF0D100221A7030BC7047C3
:10A5C8000546002AEBD1D7E703685A1C02601970C8
:10A5D80070472DE9F047089C2578002B804689466E
:10A5E8000CBF4FF0200A4FF0300A661C35B3002A22
:10A5F80029DD334601E0024698B113F8011B501ECD
:10A608000029F8D1971E60B13D46013D51464046AC
:10A61800C8476B1C002BF8DC257827EAE770013067
:10A6280055B1041B29464046C847301916F8015B46
:10A63800002DF7D1BDE8F087BDE8F087002A04DCDB
:10A648002846BDE8F0870020EBE7571EDCE70A4400
:10A65800914251D030B441F2210411F8013B80EA13
:10A668000320430010F4004F84EA03059BB2ADB207
:10A6780008BF1D466B0015F4004F84EA03009BB227
:10A6880080B208BF1846430010F4004F84EA03055F
:10A698009BB2ADB208BF1D466B0015F4004F84EAAB
:10A6A80003009BB280B208BF1846430010F4004F65
:10A6B80084EA03059BB2ADB208BF1D466B0015F4D2
:10A6C800004F84EA03009BB280B208BF18464300DB
:10A6D80010F4004F84EA03059BB2ADB208BF1D46D3
:10A6E8006B0084EA030015F4004F85B298B218BFD6
:10A6F80028468A42B1D130BC704783684268D0EDA1
:10A70800037A00EB83010133934281ED040A8360ED
:10A7180004BF0023836000EB830393ED047A03688E
:10A7280070EE277A9A42C0ED037A77EEC77AC0EDC9
:10A73800037A0CDA013307EE103AF8EEC76AB7EE7F
:10A74800007A87EEA60A036030EE070A704707EE24
:10A75800102AB8EEC77A87EE870A704790ED097A13
:10A7680090ED004AD0ED0A6AD0ED014AD0ED047AA6
:10A7780090ED035AD0ED025AA4EE007AB0EE406A8A
:10A78800B0EE470AB0EE667AA6EE247A67EEC07A93
:10A79800A0EE457AE6EE257A80ED097AC0ED0A7AD0
:10A7A8007047D0ED057A90ED013AD0ED003AD0ED42
:10A7B800064A90ED024A90ED077A90ED035A90ED23
:10A7C800086AD0ED045AC0ED067AF0EE406A27EE2A
:10A7D800830AC0ED056AA3EEA60A80ED087AA4EE06
:10A7E800240AA5EE470AA5EEC60A80ED070A7047B7
:10A7F800D0ED007A90ED017A30EE670AE7EE007A44
:10A80800B0EE670AC0ED007A704770474FF4805386
:10A818000382704750F8043C012280F83520143830
:10A8280003B11847704790F8493013B1002280F8F7
:10A8380049201846704770B5044682B00830256A2A
:10A848006B4606223B21A847A8B19DF804009DF855
:10A8580000609DF801109DF802509DF803209DF8B6
:10A86800053041EA062143EA002342EA05226182D3
:10A87800A282E382012002B070BD30B490E81200D9
:10A88800057B43690222AA404A602268586A996A8D
:10A898004FF6FE752A408842226004D1012283F8CF
:10A8A800442030BC70479C695A6B0C44D4600DD866
:10A8B80018690024411A51609C621168002041F017
:10A8C800010183F8440030BC11607047411A51609F
:10A8D8009862F2E770B40468037B2268022101FAE7
:10A8E80003F31A4213D042690A49582000FB0212A6
:10A8F8004FF6FE7650685289C5680068296831406D
:10A908002960C168D24392B20A40C260636070BCD9
:10A91800704700BF4844002030B4094B1C7864B12C
:10A92800084B002503EBC4041A6899885562D0685F
:10A9380008330143A342D160F6D130BC704700BF51
:10A94800684800206C48002010B40268047B116835
:10A958000223A340194209D00649406800240C701C
:10A9680001684FF6FE742140016053605DF8044BA6
:10A97800704700BF926900202DE9F341056906463A
:10A988000F467DBBD0F80080C8F30A0323B3002329
:10A99800D6F80080019311F0F9FD042819D1224C52
:10A9A800236943F001032361BBB2A8F8003011F01A
:10A9B800EDFD04282ED108F102030193019B3F0C01
:10A9C8001F8011F0E3FD2369042823F001032361AC
:10A9D80025D06FF0010505E011F0D8FD042805D059
:10A9E8004FF0FF35284602B0BDE8F0810E4C2369D0
:10A9F80043F002032361C4F81480236943F0400341
:10AA0800236111F0C3FD2369042823F002032361A5
:10AA1800BDD0E5E7236923F001032361D9E7336853
:10AA280004333360DEE700BF00200240F8B5044677
:10AA38000D468E180027B54201D12069F8BDE3689C
:10AA4800591CE160234415F8012B1A720429F2D12C
:10AA5800A1682046FFF790FFE7602061EBE7024B13
:10AA6800186804F0BFB900BF587C0020F0B5044650
:10AA780090F84D0083B0002840F0C580784E3778B4
:10AA8800002F52D004F11805A06915F0B7FF94F80B
:10AA980046201A212846FFF7CBFC012003F09AFF35
:10AAA800A269266D138823F040031B041B0C138036
:10AAB800138823F038031B041B0C138013889BB2E4
:10AAC80043F040031380284694F85C106B46062236
:10AAD800B047D0B19DF802609DF803309DF8005052
:10AAE8009DF801109DF804009DF8052043EA06230F
:10AAF8001BB2E3845BB241EA052142EA002201333A
:10AB0800A184228506D003B0F0BDB4F926305BB22B
:10AB18000133F8D194F924300133F4D106201BF025
:10AB28007DFB504B504ADA60EDE7254655F8180F83
:10AB380015F064FF80226B212846FFF779FC9620E8
:10AB480003F0A2FF032268212846FFF771FC962034
:10AB580003F09AFF03226B212846FFF769FC0F20B8
:10AB680003F038FF10226A212846FFF761FC0F2006
:10AB780003F030FF3A466C212846FFF759FC0F20B6
:10AB880003F028FF94F8482019212846FFF750FCC5
:10AB98000F2003F01FFF18221B212846FFF748FC4F
:10ABA8000F2003F017FF10221C212846FFF740FC56
:10ABB8000F2003F00FFF102237212846FFF738FC3B
:10ABC8000F2003F007FF012238212846FFF730FC49
:10ABD8000F2003F0FFFEA269138823F040031B0433
:10ABE8001B0C1380138823F038031B041B0C1380E1
:10ABF80013889BB243F040031380012003F0EAFE60
:10AC08000123337040E704F0FFF80546D8B120234C
:10AC180000218371C17104F08DFB2146134B41F86B
:10AC2800143F284615F070FFAB88B3FA83F3C3F1DD
:10AC38001F035A1C3FF422AF01229A400C490B68AB
:10AC480013430B601AE7014604F074FB2146074BD7
:10AC580041F8143F284615F057FF0122EEE700BFE0
:10AC6800D822002000ED00E00400FA051DA8000825
:10AC78000004014070B582B004466946183015F0EA
:10AC8800A9FFA8B19DF805009DF801609DF8021084
:10AC98009DF803509DF804209DF8063041EA0621EE
:10ACA80043EA002342EA0522A184E28423850120A5
:10ACB80002B070BDF0B5064683B00D4600240127EA
:10ACC80014E003290CBF03220122C3F3011E6946C5
:10ACD800C3F3810330468DF805208DF806E08DF822
:10ACE80007301AF0D7F80134102C0FD02B8807FA48
:10ACF80004F21342F7D0AB78E9780092022903F006
:10AD080003028DF80420DCD10A46DEE703B0F0BD6B
:10AD18002DE9F0410B4E346873691C400FD0DFF801
:10AD280028800127B4FA84F3C3F11F0307FA03F557
:10AD380058F8230003689847AC437561F2D1BDE821
:10AD4800F08100BF00040140105300202DE9F041BC
:10AD58000B4E346873691C400FD0DFF82880012738
:10AD6800B4FA84F3C3F11F0307FA03F558F8230074
:10AD780003689847AC437561F2D1BDE8F08100BF24
:10AD88000004014010530020084A094808B5936997
:10AD980043F0010393610021402221F082FF054B1B
:10ADA8004FF0FF321A60C3F8032008BD00100240BC
:10ADB80010530020505300202DE9F0410446184656
:10ADC8000D46164698461EF039FF2768E672284455
:10ADD800A07229467D69434632462046AC46BDE806
:10ADE800F0416047036810B504461B68984723681C
:10ADF80020469B689847A37B0133A37310BD30B4EA
:10AE0800436813B11A689B88138541F08001026872
:10AE180040F2E93301E0002B42D01489013B14F0E1
:10AE2800020F9BB2F7D0117302F10C0440F2E93320
:10AE380001E0002B3ED01189013B11F0010F9BB2BC
:10AE4800F7D023780268938940F2E93300E0EBB148
:10AE58001189013B11F0020F9BB2F8D0FF23137345
:10AE680002F10C0440F2E93300E07BB11189013BA7
:10AE780011F0010F9BB2F8D02578EDB2436813B1F9
:10AE88001A689B889361284630BC70470F4B9A42DA
:10AE9800F4D10F4A538B01339BB25383538BEDE7A5
:10AEA8000A4B9A42CFD10A494B8B01339BB24B8351
:10AEB8004B8BC8E7054B9A42C4D1054A538B0133E3
:10AEC8009BB25383538B0268BDE700BF0038004034
:10AED80058530020427A02B9704710B504460368F7
:10AEE800406804F10A0198470023637210BD437A51
:10AEF8005A1C0344D2B242729972037A934200D820
:10AF080002B9704710B504460368406804F10A01A5
:10AF180098470023637210BD10B40B49002301E069
:10AF2800272B0CD011F8132082424FEA430403F177
:10AF38000103F5D121445DF8044B4878704700209F
:10AF48005DF8044B704700BF90D2020870B5448882
:10AF580006460D46C4F30B0422460021284621F07C
:10AF6800A0FE3369094A934209D3094A934206D29B
:10AF7800224628461946BDE870401FF011BC23B18F
:10AF880021462846BDE87040184770BDD8230308FD
:10AF980078240308064B07498B4202D3002318463E
:10AFA80070471A88C2F30B029042F8D01433F3E7C3
:10AFB800F01F0308D8230308024A136823EA000095
:10AFC80010607047FC290020F8B51A4D2B789F2B8C
:10AFD8002ED16B78BE2B2BD105221749A81C21F046
:10AFE800ABFE28BB072229464FF6FF70FFF72FFB61
:10AFF800124FEC1D22884AB1A618BE4218D2052A63
:10B0080016D92146FFF723FB3446F3E721460222EF
:10B01800FFF71DFB0222A118FFF719FB0634084BA6
:10B02800641B1C8041F60F53C31A58425841F8BD9F
:10B038000020F8BD00F0030834F4020800000408FA
:10B04800142400202DE9F04FDFF86091504F8DB0A7
:10B058000326A7EB090718220DEB0200002121F0B7
:10B0680020FE4C4BCDF8189007971A69120604D5A4
:10B07800494A5A6002F188325A6001228DF82C2020
:10B088003422DA60454B464C18689A8804909B79BC
:10B09800ADF8142004A9072206A88DF81630FFF78A
:10B0A800C5FC072204A94FF6FF70FFF7D0FADFF8B6
:10B0B80000B180464FF0000A5C4536D30CAC002541
:10B0C80024F82C5D0222214606A8FFF7AFFC0222D5
:10B0D80021464046FFF7BBFA40BAC043ADF8080026
:10B0E800022202A906A8FFF7A1FC099860B108ABE3
:10B0F800C0F104022946184421F0D3FD089906A896
:10B10800FFF73AFC09950A909DF82C300A9A23B16A
:10B1180020490B6943F080030B61013E2DD0002AC2
:10B1280099D1FFF751FF50B32FE065888DF80DA036
:10B13800C5F30B05AA1DADF808202288C2F30B0140
:10B14800120BADF80A108DF80C2002A9062206A8E9
:10B15800FFF76CFC062202A94046FFF778FA6168FF
:10B1680080462A4606A8FFF761FC616840462A46E1
:10B17800FFF76DFA143480469EE7002AD1D00520E7
:10B188001BF04CF8074B084ADA600DB0BDE8F08FA9
:10B19800000004080020024023016745DED20208AF
:10B1A800F01F030800ED00E00400FA0500F00308B2
:10B1B800D82303080378202B024600F10100F9D0B8
:10B1C800092BF7D02D2B2CD02B2B03BF5378B7EEA0
:10B1D800000A0246B7EE000AA3F13001C8B20928F6
:10B1E8009FED467A10D8F2EE046A07EE901AF8EE50
:10B1F800E77A12F8013FE7EE267AA3F13001C8B2E8
:10B208000928B0EE677AF0D92E2B4CD003F0DF0373
:10B21800452B0BD0F7EE007A67EE276A20EE260A58
:10B2280070475378BFEE000A0246D5E710B451784C
:10B238002D2959D02B290ABF9178501C901C002425
:10B24800A1F13003092B53D8002303EB830301EB4F
:10B25800430310F8011FA1F13002092AA3F13003BA
:10B26800F3D9B3F59A7F28BF4FF49A73072B42D9C5
:10B27800DFED236A1A46F7EE007A083A072A67EEE6
:10B28800A67AFAD803F007032BB1F2EE046A013B61
:10B2980067EEA67AFBD124B3C7EE276A5DF8044BA4
:10B2A80020EE260A70475378A3F13001C8B2092866
:10B2B80002F10102AAD8F2EE046AF0EE665A07EE2D
:10B2C800901AF8EEE77A12F8013F87EEA66AA3F122
:10B2D8003001C8B2092866EEA56A37EE067AEED9BB
:10B2E80094E767EE276AD9E7901C91780124A7E7CD
:10B2F800F7EE007ACFE7F7EE007AC5E70000000026
:10B3080020BCBE4CB5EEC00ADFED317AF1EE10FA82
:10B31800CCBF30EE270A30EE670ADFED2E7A20EE3A
:10B32800270A30B5FDEEC07A87B017EE904A054679
:10B3380084EAE470002303A9A0EBE470019300936E
:10B3480002931DF093FA002CACBF20232D2303A8F1
:10B358008DF800301EF072FC012803A924D00228C1
:10B368002DD0032805BF3023684668468DF8013084
:10B3780021F0BDFC68461EF061FC0338C4B22246C9
:10B388006946284621F011FD00232B5528461EF05A
:10B3980055FC2E22431C2A540DEB0401E81821F019
:10B3A800C3FC284607B030BD302368468DF801300D
:10B3B8008DF802308DF8033021F099FCDAE730235C
:10B3C80068468DF801308DF8023021F090FCD1E705
:10B3D8006F12033A00007A442DE9F04106461546FB
:10B3E8000846B6FBF2F43CB905FB1464124B1B5D2E
:10B3F80000F8013BBDE8F081B4FBF2F767B90E4BEA
:10B4080005FB174705FB1464DA5D00F8012B1B5D8B
:10B4180000F8013BBDE8F081B7FBF2F8B8F1000F86
:10B4280002D04046FFF7D8FF05FB1878024B13F807
:10B43800082000F8012BE3E73CF4020830B4026866
:10B448001146531C036011F8024B0160D31C51785C
:10B4580003609378151D05601B0443EA0123D07827
:10B46800234343EA006030BC70470368591C1A46FE
:10B47800016012F8021B0260587841EA0020704708
:10B4880038B50446006815461FF08AF922682A4430
:10B49800226038BD036810B40A0A5C1C04601A7084
:10B4A80003685A1C026019705DF8044B7047036802
:10B4B8005A1C026010B4197003680A0A5C1C046004
:10B4C8001A7003680A0C5C1C04601A700368090E81
:10B4D8005A1C026019705DF8044B704703685A1CC7
:10B4E800026019700368090A5A1C026019707047D3
:10B4F8002DE9F047002488B080460F461E46A14635
:10B5080005AD531C0393117839B3252933D1931C06
:10B51800CDF810900393507830284ED04FF0000AA1
:10B52800A0F13003DBB2092B42D96C2819D064286A
:10B5380000F0938024D825281CD063D9582876D0C9
:10B5480063281BD131784046B847039A531C0393AC
:10B558001178043601340029D7D1204608B0BDE857
:10B56800F087039B5A1C03921B78642B7CD02AD843
:10B57800252B54D1252140460134B847039AC0E70A
:10B58800732833D044D975284FD106F1040E30689A
:10B598002B4600220A217646FEF7DEFF049A009524
:10B5A800534639464046FFF714F8039A0444A8E77F
:10B5B80004AA03A911F0D0F9B7E7D31C0393907834
:10B5C8004FF0010AACE7732B10D05BD9752B3AD03A
:10B5D800782B96D1A3F15802B2FA82F23068520958
:10B5E8002B4610210436FEF7B7FFD7E73368049AD5
:10B5F8000093394600234046FEF7EBFF0436044427
:10B60800039A7EE70028B9D1204608B0BDE8F08744
:10B618006E28B3D1039A336804361C6071E72AD9BF
:10B62800582BD7D0632B8DD06BE77828A6D1A0F103
:10B638005802B2FA82F2306852092B461021FEF7FE
:10B648008BFF0436AAE706F1040E30682B46002269
:10B658000A217646FEF780FFA0E7331D30682946A9
:10B668001E46FEF74BFF99E7331D306829461E46F4
:10B67800FEF744FF92E7002B7FF443AF204608B063
:10B68800BDE8F0876E2BC6D03BE70EB400B584B09A
:10B6980005AB019053F8042B0649039301A8FFF763
:10B6A80027FF019B00221A7004B05DF804EB03B079
:10B6B800704700BFD1A500080FB430B583B006AB02
:10B6C8000B490C4853F8042B096800680193FFF7ED
:10B6D8000FFF094C0546206803685B6998470028F6
:10B6E800F9D0284603B0BDE8304004B0704700BF29
:10B6F800483700204C370020587C0020DFED2B7A9B
:10B70800B4EEE70AF1EE10FA4ADDDFED296A9FEDA3
:10B71800297A01E0B0EE670AB4EEC70AF1EE10FA32
:10B7280070EE667AF6DC9FED247AF4EEC77AF1EED5
:10B7380010FA38D5DFED1E6A9FED207A01E0F0EEB1
:10B74800407AF4EEC77AF1EE10FA37EEA60AF6D48C
:10B75800DFED1B7AB4EEE70AF1EE10FA14DDDFED47
:10B76800137A37EEC00A60EE006A9FED166A9FED05
:10B77800167ADFED167AA6EE867A20EE266AE6EECF
:10B78800877AA6EE270A7047DFED117AB4EEE70A4A
:10B79800F1EE10FA44BFDFED087A37EEC00AE2E7AF
:10B7A800F0EE407ABFE7B0EE670AD1E7DB0F494019
:10B7B800DB0FC940E4CB1641DB0F49C0E4CB16C10F
:10B7C800DB0FC93F92E741B99730083C15A82ABE5C
:10B7D800DB0FC9BF41404A0011F0800F82F0D5034A
:10B7E800D2B2DBB208BF1346590013F0800F81F0C4
:10B7F800D502C9B2D2B208BF0A46510012F0800F72
:10B8080081F0D503C9B2DBB208BF0B46590013F06B
:10B81800800F81F0D502C9B2D2B208BF0A465100E2
:10B8280012F0800F81F0D503C9B2DBB208BF0B4616
:10B83800590013F0800F81F0D502C9B2D2B208BF07
:10B848000A46510012F0800F81F0D503C9B2DBB26D
:10B8580008BF0B465A0082F0D50013F0800FD2B211
:10B86800C0B208BF1046704709B909E0194690FBF5
:10B87800F1F301FB13030846002BF7D10846704784
:10B888000146FBE710B507EE901A2DED028BB8EED6
:10B89800678ADFED227A28EE008A044628EE278A96
:10B8A800B0EE480A1FF03CF9F0EE408AB0EE480AC4
:10B8B8001FF098F8F7EE007A9FED197AF0EE675AC4
:10B8C800E8EE875A0023A361B0EE676AC7EEA56A5F
:10B8D80063612362E361A3626362A8EEC76ABDEC99
:10B8E800028B77EEC07AB6EE007AF8EE005A27EEB1
:10B8F800877A20EE250A27EE267A26EE266A67EE54
:10B90800A67A20EE260A84ED046AC4ED017A84ED55
:10B91800007A84ED027A84ED030A10BD27D4D2366A
:10B92800F304353F10B44C09012250F8243001F0DB
:10B938001F0102FA01F10B4340F824305DF8044B73
:10B9480070474B0901F01F0150F82320012303FA27
:10B9580001F1114214BF184600207047F8B5154B85
:10B96800154A16481946012405274FF4FA4640F2AD
:10B978001945DF741C721C751680958217F0FAFC45
:10B988000F4B104AB42450216420252623252D2747
:10B998009C710F241F7219705E701E719D705D710D
:10B9A800D8701070507051719171D1719470547237
:10B9B800F8BD00BF1C4900201C44002064F40208A4
:10B9C800B62800205E2E0020F0B5574B574A97B096
:10B9D8001968914200AF00F09C805549554A0023F0
:10B9E8004FF47000C1F888003B607B60136843F433
:10B9F8008033136003E03B68B3F5A04F09D01368A8
:10BA080003F400337B603B6801333B607B68002BA9
:10BA1800F1D0484B1B6813F4003318BF01237B6037
:10BA28007B68012B4BD0424D424B434AEA60434A64
:10BA3800596A11605A6A424E42F080725A625A69D3
:10BA480007F1580442F4FC0241F6FF715A6124F8E8
:10BA5800501D032321464FF09040BB72FFF72AF98F
:10BA68004FF6FF73214637483B81FFF723F92146FC
:10BA78003548FFF71FF921463448FFF71BF92146DF
:10BA88003348FFF717F921463248FFF713F92046E4
:10BA980018F0B4FFBB683049304AA1FB03133049A2
:10BAA8009B0CF02400204FF0070E5C370B605660AB
:10BAB80085F823409060C2F800E0BD46F0BD294AF1
:10BAC8001C4B122111605A685A605A685A605A68A9
:10BAD80042F480625A605A6822F47C125A605A68AA
:10BAE80042F4E8125A601A6842F080721A601A68C2
:10BAF8009201FCD559680F4A21F003015960596831
:10BB080041F002015960536803F00C03082BFAD185
:10BB180089E700221A6062B6134B1B6883F3088812
:10BB2800124B1B689847FEE7FC9F0020EFBEADDE76
:10BB380000ED00E0001002400005FA054849002029
:10BB48003F1901000004004800080048000C0048A4
:10BB5800001000480014004883DE1B4310E000E09A
:10BB6800C45300200020024000D8FF1F04D8FF1F44
:10BB780070B50F4C0F4DC0EBC00004EB8004686932
:10BB880026693043686182B09209667BA16000250E
:10BB9800012101A863618DF804608DF805208DF8F6
:10BBA80006508DF8071014F043FE02B070BD00BFB8
:10BBB800E018002000100240074BC0EBC00030B472
:10BBC80003EB8000054C056963692B4363610176CB
:10BBD800427630BC704700BFE018002000100240D9
:10BBE8002DE9F04F5E4C54F8204083B0002C71D002
:10BBF800666D984691465B4B72682265A16023602A
:10BC080004F15A014FF4807304F5AD726161A261C9
:10BC1800E36023610746307E14F06CFCF068A8B13D
:10BC2800514B00215A68904203F11C0300F09280A6
:10BC380001310C29F6D100207A1CD2B20C21FFF771
:10BC4800BBFF236DF26822632433E364B068D8B184
:10BC5800454B00215A68904203F11C0378D001310A
:10BC68000C29F7D100257A1CD2B20B212846FFF700
:10BC7800A3FF2346F27E3D492846FFF779FF236D4F
:10BC8800B26862632833A36494F8590003F0BCF8DF
:10BC9800054694F8580003F0B7F818F0080F8246E4
:10BCA80096F819B01AD0CDB118F0110F4FF00B0358
:10BCB80007F1010714BF4E213E21EF715A46AB71BF
:10BCC800284603F065F918F0010F45D0236B5BB3E4
:10BCD800636B4BB3204603B0BDE8F08F18F0010F3B
:10BCE8000CBF4FF02E084FF04E0819F0020F09D084
:10BCF80045B10B227B1CAA71EB7128465A46414676
:10BD080003F046F919F0010FE0D0BAF1000FDDD0C9
:10BD180001370C238AF807705A4641468AF80630DC
:10BD2800504603F035F9D1E7337FB27E8DF8042011
:10BD38009B090021012201A88DF805308DF8061015
:10BD48008DF8072014F074FD204603B0BDE8F08F8D
:10BD5800CDB288E7C8B26FE7284603F0A7FCB5E77D
:10BD680054370020E8D20208E018002083A8000811
:10BD78000348D0F83C3113B100F59A701847704762
:10BD8800E01800200348D0F8203113B100F58C707A
:10BD980018477047E01800200348D0F804310BB169
:10BDA800FC301847704700BFE01800200348D0F85F
:10BDB800E8300BB1E0301847704700BFE0180020AA
:10BDC8000348D0F8CC300BB1C4301847704700BFD7
:10BDD800E01800200348D0F8B0300BB1A83018475D
:10BDE800704700BFE01800200348D0F894300BB12A
:10BDF8008C301847704700BFE01800200248836F56
:10BE08000BB1703018477047E01800200248C36D26
:10BE18000BB1543018477047E01800200248036CF3
:10BE28000BB1383018477047E01800200248436AC1
:10BE38000BB11C3018477047E0180020024883688F
:10BE480003B11847704700BFE01800201749184B86
:10BE5800184A194810B4D1F8884044F47004C1F85D
:10BE680088401C6844F001041C605C6822405A60E9
:10BE78001A6822F0847222F480321A601A6822F456
:10BE880080221A605A6822F4FE025A60DA6A22F0A6
:10BE98000F02DA621A6B002410404FF00062186338
:10BEA8009C608A605DF8044B704700BF00ED00E0BD
:10BEB800001002400CC07FF8CCFC00FF2DE9F04FC9
:10BEC8002DED028B9B4A9C49137897B004460B9042
:10BED80000F59C4020300E900860002B00F07E8515
:10BEE800964909688C4240F29780954905910968FE
:10BEF8009448954D954C0491013B137001F480537F
:10BF080003900A93002B40F09580039B5B7D002BE8
:10BF180040F00285049B180400F1E987049BD905C9
:10BF28000BD50B9A8A4BDFF858B29A429BF802203D
:10BF380001F2AD81002A41F0AE81864B0693864E10
:10BF4800049B13F4805840F00885039BB4F90670ED
:10BF58005B8B9F42B4BF00270127804B1B6813F0FF
:10BF6800805374D0069A127812F0010276D00399A1
:10BF7800DFF81092898C99ED037A07EE901AF8EEA3
:10BF8800E77AB4EEE77AF1EE10FA81F27680002FC4
:10BF98006BD195F8A410002967D1714871490068E0
:10BFA80090F830004FF0000EC1F800E0C1F804E04E
:10BFB800C1F808E06C49002858D10870002A59D007
:10BFC800049AD00656D5694A1278D10652D4B8F1E7
:10BFD800000F4FD1002B4DD1049B5A024AD496F83A
:10BFE80000E0BEF1000F01F08787614B9B78002FBE
:10BFF80041F0AE873BB15F4A5F4B12681B689B1AE2
:10C00800002BC1F2CF87102012F016FA012385F811
:10C01800A53096F800E02FE0494B05931B68049380
:10C02800484A494D039203F48053484C0A93002B25
:10C038003FF46BAF00214948FFF783FC00287FF4E9
:10C0480064AF13F02DFD059B1B6804935DE7049A0C
:10C05800520287D4069A127802F00102002185F86C
:10C06800A410DFF82091002F97D03F4901200870D5
:10C07800002AA5D196F800E0039AB4F90080518B04
:10C08800928BB4F9020095F8A6B08845CCBF4FF062
:10C09800800C4FF0000C4CF040039045A8BF63465D
:10C0A8009B0843F0800C8842C8BF634643F0400CAD
:10C0B8009042B8BF63469B08B4F904C0B4F90600BF
:10C0C80043F080088C45C8BF434643F04008944578
:10C0D800B8BF43469B0843F0800C8842C8BF6346FC
:10C0E80043F0400C9042B8BF63469B4500F0108671
:10C0F8004FF0000885F8A63085F8A780BEF1000F3C
:10C1080000F06787059B1B6803F00403002B40F0D1
:10C118007D850DF1500A194E0023CAF8043006F146
:10C12800500B14934FF0190840F6330340F283374D
:10C138002DE000BF1C650020046400201865002065
:10C148004C4900201C49002014230020B469002019
:10C15800404B4C0035690020861A0020F039002039
:10C16800A8280020C8370020501E0020F0640020B6
:10C178003C3A0020C0530020E4520020643A0020DA
:10C1880064690020D04F002004365E4524D0B17881
:10C19800F278914218FB0170F6D296F801E00EF1A0
:10C1A800040E18FB027134F91E209A42A8BF1A46E1
:10C1B800B2F5617FB8BF4FF461729042E4DA914200
:10C1C800E2DB31782329DFD8504604360493FFF7A1
:10C1D800A9FB5E45049BDAD15C4B9AE803001F7803
:10C1E8005B4B83E80300002F00F09B84594B0493BA
:10C1F80057480121FFF7A5FB002840F05E82059B08
:10C208001B68DE0500F15482534B0793534D2B886E
:10C218001EB226F001061FFA86FA5345A5F800A0BB
:10C2280000F0E4854E4E4FF002080F2014274FF01F
:10C23800FF0B86F80080777086F802B012F0FCF8E1
:10C2480041464348B5F800A0FFF77BFB002841F0C2
:10C25800B3812AF002039BB253452B800BD0404B8D
:10C268001421FF2202260F201E7059709A7012F0B6
:10C27800E3F8B5F800A03B4B3B4A1978506809939E
:10C288001AF0030F08BF81F00201C1F340010892C0
:10C2980003F018FA079B1B6813F00A0F1AD006213F
:10C2A8002B48FFF74EFB002800F07F862B885806A6
:10C2B80041F1EE8007212648FFF743FB50B12B4B95
:10C2C8002B4AB3F904302B4982FB0302DB17C3EB7B
:10C2D800A2030B800C211E48FFF733FB2A88002895
:10C2E80000F04F8242F480739A422B8009D01C4B95
:10C2F80002261421FF220F201E7059709A7012F026
:10C308009BF81D4B1B78082B00F047820E2B00F082
:10C318004482059B1B68590561D5184B1B79002B76
:10C3280000F0188114210A48FFF70BFB002840F0A1
:10C33800168112F07BFE012011F0D0FF00284ED0AC
:10C34800DFF83CA000264FF0CC0B1EE0DE69002091
:10C35800F0390020406E0020185C0020DC690020C5
:10C368005C260020885300208C530020D03B0020FE
:10C3780067666666E2520020603A00209C4F002003
:10C38800A0770020DEB2022E29D80BFB06F8731C1A
:10C398005AF80870002FF5D1C378D84A90F90200EE
:10C3A80052F8233001970322009201213A4611F0F6
:10C3B80077FB034606EB460000EB0010079353B1EA
:10C3C80039460AEB8000CC2220F06BFC079B4AF828
:10C3D80008300136F6B21AF04DFC0028D3D1069B7E
:10C3E8001E7816F0010600F01182C54B01221A7062
:10C3F800049BB4F906101B68C2485A890127914268
:10C40800077080F2E981C04B4FF07E521A60BF4A34
:10C41800039BB4F900C01F8B92F9043092F801E035
:10C428001078002BACEB070314BF01224FF0FF324A
:10C43800002B40F3C581B3F5FA7FC0F2C7814FF4F2
:10C44800FA731B1A07EE903AF8EEE77A6745C9EDDA
:10C45800007A03DDF1EE677AC9ED007AB4F902C01B
:10C46800ACEB0703002B40F38081B3F5FA7FC0F2F1
:10C4780082814FF4FA731B1A07EE903AF8EEE77AC6
:10C488006745C9ED017A03DDF1EE677AC9ED017AF6
:10C49800B4F90400C31B002BD8BF3B1AB3F5FA7FCD
:10C4A80080F25E817345D8BF4FF0000E00F35A81C9
:10C4B80002FB0EF207EE902A059BF8EEE77AB842E7
:10C4C8001A68C9ED027ABCBFF1EE677AC9ED027A43
:10C4D80012F4805200F00B82B1F5FA6FA8BF4FF446
:10C4E800FA61B1F57A7FB8BF4FF47A71A1F57A7124
:10C4F800874C884884FB013ECB17C3EB6E1303F1CE
:10C50800010E6FF0630C30F91EE030F913000CFBDC
:10C518000313AEEB000103FB01F384FB0314DB17E9
:10C52800C3EB641303441BB207EE903AB8EEE78AF4
:10C5380089ED038A002A40F08C832B885B0624D47B
:10C54800002E40F0A8801BF042FA17B0BDEC028B19
:10C55800BDE8F08F069B1B78DA077FF5EAAE3C2032
:10C568001CF07CFB00283FF43AAF1CF07BF83C2021
:10C578001CF016FB00283FF432AF1CF073F83C2087
:10C588001CF00EFB0028F0D129E7634B634AB3F98E
:10C5980004306349DFED636A09889FED637A82FBA3
:10C5A8000302DB17C3EBA2035B1A1BB207EE903A38
:10C5B800F8EEE77A67EEA67A77EE876ABDEEE66A66
:10C5C80016EE103A2033402B40F26D87BDEEE77A25
:10C5D800DFED626A17EE103A2033402B00F2B08785
:10C5E8009FED527AF4EEC77AF1EE10FA41F32C83FC
:10C5F800DFED4F5A9FED4F6A01E0F0EE477AF4EE17
:10C60800C67AF1EE10FA37EEE57AF6DCDFED4A7A13
:10C61800B4EEE77AF1EE10FA41F11283DFED445AF5
:10C628009FED466A01E0B0EE677AB4EEC67AF1EEA5
:10C6380010FA77EE257AF6D49FED3B7AF4EEC77AB6
:10C64800F1EE10FA40F330859FED387A77EE677A8D
:10C6580067EEA75A9FED3A5A9FED3A6A9FED3A7AEC
:10C66800A5EE856A27EEA55AA5EE867AE5EE077A45
:10C6780099ED016AD9ED005A27EEC67A65EEA77AD8
:10C68800A5EEA67AE6EE267A89ED007AC9ED017A5A
:10C69800002E3FF458AF099B1978089B01F001015F
:10C6A800186803F00FF817B0BDEC028BBDE8F08FE7
:10C6B800264BDB78002B3FF4A7AD254B07931B686F
:10C6C8009D077FF5A3AD234DB5F800A01AF0010F23
:10C6D8007FF4BFAD4AF001039A452B803FF4B9AD12
:10C6E8001D4B022214211A700F20FF2259709A70D4
:10C6F80011F0A2FEB5F800A0ABE500BF60E90208A2
:10C7080036690020881D00202C1E0020103A0020C9
:10C718001F85EB51446E0020D03B0020676666669B
:10C72800E252002035FA8E3CDB0FC93FDB0F49404F
:10C73800DB0FC940E4CB1641DB0F49C0E4CB16C17F
:10C7480092E741B99730083C15A82ABE64690020D1
:10C75800185C0020DC6900205C2600200000000036
:10C768004FF4FA73A3EB0E0EA2E6A7EB0C03B3F596
:10C77800FA7FBFF67EAE9842FFF67DAE5FED097A8E
:10C788007EE622F480739BB29A422B807FF4AFAD91
:10C798007E4B1B78082B7FF4B9AD2A8822F0400322
:10C7A8009BB29A422B803FF4B4AD794B02261421F8
:10C7B800FF220F201E7059709A7011F03DFEA8E5F7
:10C7C800A7EB0C03B3F5FA7FBFF639AE9842FFF634
:10C7D80038AEDFED707A39E6B1F5FA6F80F228836A
:10C7E800187A8B1A03FB00F3C2F5FA6293FBF2F393
:10C7F800C3F1640307EE903AF8EEE77A9FED667AA4
:10C80800664B67EE877AC3ED007A00E6644B1B78C7
:10C818000793002B7FF4ECADDFF8B8B1DFF8B8A1CF
:10C828001BF8030C9AF800805946ABF103071AF07D
:10C838004BFE002800F00283079BB8F1000F53D18C
:10C8480007F1080178791AF03FFE002841F06A8262
:10C858005449B87A1AF038FE002800F00383B8F17A
:10C86800020F41F062825049F87B1AF02DFE002831
:10C8780041F05E824D49387D1AF026FE002800F00E
:10C888000383B8F1040F41F056824949787E1AF0C3
:10C898001BFE002841F052824649B87F1AF014FE68
:10C8A800002800F00383B8F1060F41F038824249AE
:10C8B80097F823001AF008FE002840F084873F49C3
:10C8C80097F828001AF000FE002800F00383B8F15A
:10C8D800080F40F067873A4997F82D001AF0F4FDE1
:10C8E80000283FF485AD09231A4600F05DBF039B7D
:10C8F800588B8142C0F29A82B1F5FA6FD4BFC0EB6F
:10C908000101C0F5FA614FF47A7303FB01F1C0F538
:10C91800FA60B1FBF0F1EBE5039A013BD27D34F903
:10C928001330002A40F06E83A3F57A73B3F57A7F4B
:10C93800A8BF4FF47A7323EAE37307EE903A9FEDAA
:10C94800217AF8EEE77A67EE877A1F4AFCEEE77AF3
:10C9580017EE903A1380FFF7E1BA1D211B48FEF746
:10C96800F0FF00287FF4F1AA194A039BD2881B8B99
:10C97800B4F90670991A8F4240F3C48613449F4253
:10C98800B4BF00270127FFF7E8BA00BF603A0020CC
:10C998005C260020000000000AD7233C2C1E002043
:10C9A80036690020372600203C260020412600203A
:10C9B800462600204B260020502600205526002021
:10C9C8005A260020AAF1823F50690020F039002041
:10C9D800D84100202D2600200A000020B34DB44B7A
:10C9E8002E780393DFF8CC82002E00F02183B6B1B5
:10C9F800DFF80893DFF808B3AE4FCA460024072CC7
:10CA08003846E1B2D8F8043041F35282984700B270
:10CA18000134A6422BF8020F0AF1040AEFD1A64B03
:10CA280005931A460B99A54B12680492A3FB013E85
:10CA380042F2010313404FEA9E1E099300F0E78279
:10CA48009F48A04AA04B0078A049079012781A7016
:10CA5800079B087023B19C4B1B7883F00103079355
:10CA68009B4A039912780D920D9A0C8D994BB1F847
:10CA7800269091F822C010940C8B13941146A3FBB6
:10CA880001135B0803EB4303D31ADBB295F8294083
:10CA98000F93049B98F800002E7808900F222046E8
:10CAA8000CF1040C03F480538B4F8C4CDFF854A228
:10CAB800CDF818905FFA8CFCB34685F828201192BF
:10CAC8000A93002181460C95CDF8488036B9089B19
:10CAD8009C458DBF9B46E34666465E46B14280F262
:10CAE8006383079B002B00F00D837D4B069833F979
:10CAF80011201FFA82F880454FEA410303D31098AA
:10CB0800804540F24C835AF82120964580F00483F2
:10CB1800E25E0998002840F01B83E2520131063793
:10CB2800D4E7DFF8E4B1DFF8E4810BF15A064FF0FF
:10CB3800010A59461BF8010C1AF0C6FCF8B19BF81B
:10CB480004009BF802309BF803E000EB400105EB82
:10CB58008101013BD1F8B42003EB430343449342E2
:10CB68000DD095F8E02081F8B0E00AFA00F022EA4A
:10CB78000000C1F8B430C1F8B87085F8E0000BF1D6
:10CB8800060B5E45D5D1574B574A049319464F4B70
:10CB9800D2F800B009681B78544E0891DA4607931A
:10CBA8000027AB46736853B31D7845B3B168AAEB49
:10CBB800010100290ADB9BF8E0100120B84021EAB6
:10CBC80000010AF5FA708BF8E010B060079AB2B16C
:10CBD800317858780431C9B2002840F05382039A5A
:10CBE80034F91110108B00F1C80E714540F35E85C1
:10CBF8009BF8E0109B783941C90740F1BE850137A1
:10CC0800042F06F10C06CDD1FFF7F2BA95F8AB3038
:10CC180053B1069B1B78D80706D5039BB4F90620A9
:10CC28005B8B9A4200F39B8511213148FEF789FE00
:10CC3800002800F0098295F8AE302BB995F8A93094
:10CC480013B93223A5F8AC30012385F8AE30FFF7CD
:10CC580060BA1D212648FEF774FE00283FF46DAC2B
:10CC6800244BDB78002B7FF468ACDFED237A134983
:10CC780038EE678AC7F5FA63FDEEC87A1BB2CDEDC8
:10CC8800037ABDF90C20120381FB0201D217C2EB13
:10CC9800A11203FB02F343F30F333B4407EE903A30
:10CCA800F8EEE77AC9ED037A47E400BF14230020C1
:10CCB8001C490020F86300204C490020D34D621025
:10CCC800D4630020381A0020391A0020496900204E
:10CCD800D9270020ABAAAAAA40230020B4690020C3
:10CCE80018230020406E0020C0530020C4230020D9
:10CCF800F03900206469002000007A4444280020AC
:10CD080016230020DC2700204525002010D3020828
:10CD180095F8A780B8F1F90F00F2A88108F1010889
:10CD28005FFA88F885F8A78085F8A630BEF1000F6D
:10CD380000F05081B8F1140F7FF4E4A95F2B40F0A4
:10CD48005C81069F3B7813F0010300F0818712F0A5
:10CD5800A7FE3B7803F00103002B7FF4D3A995F8D5
:10CD6800A620572A00F00087059B1B6813F00403D0
:10CD780002D05A2A00F02A855D2A00F05D875B2AD6
:10CD880000F07F875E2A00F0FE84562A00F0E187D3
:10CD980033782BB16F2A00F0D487CA4B0021196071
:10CDA800972A00F0E587A72A00F0CE840021BB2A45
:10CDB800149101F00B80B72A00F0EA87BE2A01F02F
:10CDC8000880BD2A01F047809E2A01F031809D2A03
:10CDD80001F02680AE2A01F01B80AD2A7FF492A9CB
:10CDE800FF21002018F0AFF8FFF78CB90221B648F0
:10CDF800FEF7A7FD00283FF42CAA2E801AF0020F98
:10CE08007FF439AA4AF0020353452B803FF433AA32
:10CE1800AE4B022214211A700F20FF2259709A700B
:10CE280011F00AFBB5F800A0FFF725BA11466EE528
:10CE38001B7AC3F1640307EE903ADDE40BF10501B8
:10CE480078791AF041FB00283FF402ADB8F1010FE0
:10CE580040F0688707F10D01B87A1AF035FB002811
:10CE680040F063879A49F87B1AF02EFB00283FF4BC
:10CE780001ADB8F1030F40F05B879649387D1AF091
:10CE880023FB002840F057879349787E1AF01CFB53
:10CE980000283FF401ADB8F1050F40F04F878F49E6
:10CEA800B87F1AF011FB002840F039878C4997F8B1
:10CEB80023001AF009FB00283FF401ADB8F1070F71
:10CEC80040F08184874997F828001AF0FDFA002875
:10CED80040F06884844997F82D001AF0F5FA002884
:10CEE8003FF486AAB8F1090F3FF482AAFBE4D5F80B
:10CEF8008C300B9AD31A002BFFF610A87B4A95F8B2
:10CF08009030517C7A4A039E32F811200E98B17DF8
:10CF1800C5F88C00013303F00F0385F890302B44DB
:10CF280092B292FBF1F283F8942095F8940095F868
:10CF3800951095F8962095F8973001440A4495F88D
:10CF4800980095F899101344184495F89A2095F884
:10CF58009B3001440A4495F89C0095F89D101344B1
:10CF6800184495F89E2095F89F3001440A4495F896
:10CF7800A00095F8A1101344184495F8A23095F82C
:10CF8800A32001440B441A4442F30B12642AF17D96
:10CF9800A8BF642213B209B1C2F1640307EE903A44
:10CFA8009FED547AF8EEE77ACDE42A8822F0400320
:10CFB8009BB29A422B803FF47DA9444B0226142150
:10CFC800FF220F201E7059709A7011F035FAFFF782
:10CFD80071B9F04600213C48FEF7B3FCD8B10023F4
:10CFE80085F8A83013F010F995F8A730142B7FF4C2
:10CFF80089A83378002B40F0D187069B1B7803F073
:10D008000103A9E6C3F53B6308331BB28CE43A4B32
:10D018001B7807931EE5069B2A4A1B781060DB07DE
:10D0280000F17C85B8F1140F3FF499AEFFF76AB8A8
:10D0380093F8223098F800600433DBB2B3428EBF15
:10D048002E702B701E46D2E495F8A930002B3FF4C1
:10D0580060A8069B1B7813F001037FF45AA80122ED
:10D0680085F8A93085F8AA20FFF753B885F8A6B047
:10D07800BEF1000FAED0FFF745B8012185F8A41026
:10D08800FEF7F3BF012800F083859BF8E010012329
:10D09800BB4001370B43042F8BF8E03006F10C0638
:10D0A8007FF480ADFFF7A4B89FED147AF4EEC77A49
:10D0B800F1EE10FA44BF9FED127A77EE677AFFF728
:10D0C800C7BA00BFE8520020F03900205C260020D3
:10D0D8003C26002041260020462600204B26002022
:10D0E80050260020552600205A260020EC52002009
:10D0F8000853002014AE234149690020DB0FC9BF43
:10D10800DB0F49C0069B002B47D05AF821209645D3
:10D118004FEA4103FFF4FCACBE4ABE48D25C00EBC8
:10D128000308002A00F01082022A40F0A58198F82E
:10D13800012002EB820202EB820202F2EE2292B29C
:10D14800032940F39B80099812B200283FF4E5AC0C
:10D158000F9803EB010880440C9800EB4808A8F8E6
:10D168002C20B9F1000F03D10D9802287FF6D5AC19
:10D17800B7F800907A88B7F804804A449044A64AE1
:10D188000FFA88F882FB0802A448A2EBE87220F89C
:10D19800038012B24FF00109BFE41A464B000EF5A6
:10D1A80096784AF82180B4E411990C9D9C4BDDF8DF
:10D1B800488085F800B00F294A460CBF012200229A
:10D1C80085F8299085F828101A7006D11B219548F2
:10D1D800FEF7B7FB002800F018859348934B826848
:10D1E8001968934BC1608A1A012119704368914FDD
:10D1F8009A42039A397088BF002392F8227088BF38
:10D2080080F821300A9B98F80000B2F818C0B2F8EC
:10D2180026800437FFB2002B00F0A38187427D4AA5
:10D2280040F22082844F964600210EB98346064676
:10D23800B1421ADA12F8113093B1022B0ED19EF8CE
:10D24800013003EB830303EB830303F2EE239BB26A
:10D2580027F8023B01310EF1020EE6E73B88F7E7BB
:10D26800CBB2032BFAD86346F2E785F800B00D9BE2
:10D27800724A013313700A9BFEF744BE012000FA7C
:10D2880001F8119820EA080012B2119041E412B98D
:10D2980001228BF802206A4B06931E789BF8219096
:10D2A80006F001031B2004931AF038F9B9F1010FB5
:10D2B800089000F02A8206F0020307939BF82020CA
:10D2C800604EDFF888A1604FDFF86081052A00F220
:10D2D8009880DFE802F0887C032E3E52B9F1010FF6
:10D2E80004BF05238BF82030049B002B00F0D88066
:10D2F800039BD8F80000B3F91810BAF802300022DE
:10D3080061F30F0263F31F42002361F30F0361F31C
:10D318001F43DBF8141062608842236040F2738177
:10D328000323079347F230520323CBF81C208BF8D2
:10D3380020303B8843F002033B8012F0B1FBD8F861
:10D348000020DBF81C3013440422CBF818308BF88B
:10D358002020B9F1010F40F06684D8F80030DBF8DE
:10D3680018209A424DD2307818B91AF0D7F8002808
:10D3780047D13B8823F002033B80D8F80020BAF855
:10D388000630642101FB03234FF4806000228BF8F0
:10D3980020208BF80320CBF8103011F043F99BF8CC
:10D3A800202093E71AF0E6F8012800F0AD84089BE6
:10D3B800002B40F0AD81B9F1010F22D0D8F8003030
:10D3C800DBF810209A4259D301238BF82030B9F1A9
:10D3D800010FD2D09AF80830012B4FD00DF020FF62
:10D3E8009BF8202072E7049B002BDBD1089B4FF4AD
:10D3F8008060002B00F0F28011F02CF90022CBF8AD
:10D408001020079B002B40F0FA80059B1B680493B3
:10D41800FEF797BD782800205655555588230020DB
:10D42800F1640020F039002064690020C053002016
:10D43800381A0020391A0020B4690020D9270020A2
:10D4480035690020861A002088690020EC410020F8
:10D45800E4CB1641DB0F49C0DB0FC940E4CB16C152
:10D46800DB0FC93FDB0F494092E741B99730083CD1
:10D4780015A82ABE00000000E25A61E60DF0D0FEB1
:10D48800032240F6B8338BF82020CBF81C3050E745
:10D4980043F0400293422A807FF48FADFEF70ABF23
:10D4A800D8F800303EE7F4EEC77AF1EE10FA40F310
:10D4B80023845FED175A1FED1A6A01E0F0EE476A00
:10D4C800F4EEC66AF1EE10FA36EEE57AF6DC5FEDB8
:10D4D8001F6AB4EEE67AF1EE10FA40F111845FEDBE
:10D4E800225A1FED226A01E0B0EE667AB4EEC67ADF
:10D4F800F1EE10FA77EE256AF6D41FED277AF4EEEE
:10D50800C76AF1EE10FA6CDD1FED2A7A77EE666ACB
:10D5180066EEA65A1FED2C5A1FED2C6A1FED2C7AC9
:10D52800A5EE856A26EEA55AA5EE867AE5EE076A87
:10D53800BDEEE77A17EE103A2033402B7FF650A85D
:10D548005FED347AFFF794B8CAB2022A40F2E38258
:10D55800032A91D1139A0A98069D002808BF2A46E3
:10D56800EEE587421946B64A55D8B64896460EB9EA
:10D57800BB463E468E427FF778AE12F8113093B123
:10D58800022B0ED19EF8013003EB830303EB8303D8
:10D5980003F2EE239BB220F8023B01310EF1020E9A
:10D5A800E5E70388F7E7CBB2022B03D9032BF8D1C1
:10D5B8004346F0E76346EEE72AF0010292B252458D
:10D5C8002A803FF41BAC0F2086F80080777086F81D
:10D5D80002B010F031FFB5F800A00FE411F022F806
:10D5E8000CE79FED997AF4EEC76AF1EE10FA44BFA2
:10D5F8009FED967A77EE666A8AE703230793079882
:10D6080010F01AFF01E7B9F1010FF6D103239BF8D7
:10D61800202007935AE68B4F96460EB98346064656
:10D62800B142BFF622AE12F8113093B1022B0ED1DF
:10D638009EF8013003EB830303EB830303F2EE232D
:10D648009BB227F8023B01310EF1020EE5E73B8859
:10D65800F7E7CBB2022B03D9032BF8D14346F0E707
:10D668006346EEE77748964600210EB9BB463E462C
:10D67800B142BFF6FAAD12F8113093B1022B0ED1B8
:10D688009EF8013003EB830303EB830303F2EE23DD
:10D698009BB220F8023B01310EF1020EE5E7038848
:10D6A800F7E7CBB2032BFAD86346F2E7C8388142D2
:10D6B8003DDA9BF8E0109B783941CA073FF59FAAED
:10D6C800C3F10008012010F095FF691E162900F229
:10D6D8000B81DFE811F0F8010C02E101BC015401F3
:10D6E8002F010C01A3018E01790164010901BC011C
:10D6F800CD012F010C01A301B601B901CF00F9003A
:10D70800E300A1000127FEF728BC00230793D5E515
:10D718009AF80430002B3FF44EAE0DF081FD032241
:10D728004FF47A738BF82020CBF81C3001E69BF875
:10D73800E0300121B94023EA01030AF5FA718BF8B8
:10D74800E030B160FFF75BBA4149059B0A781B6876
:10D7580042F004020A7003F00403FEF7D7BC00216C
:10D768003C48FEF7EEF800287FF45EAA322385F8DD
:10D77800AB00A5F8AC30FFF757BA9846002B0CBFA2
:10D78800012002209FE7344B022203203349344E04
:10D798000B60327010F02EFF059B1B6803F004032A
:10D7A800FEF7B4BC08231A4602EB820217448AF833
:10D7B8000030B978787818F06DFB069B1E7806F073
:10D7C8000106FEF715BE07231A46EDE795F8A920CE
:10D7D800002A40F0438395F8AB1081F0010185F8E9
:10D7E800AB10002940F099831E4A126812F40032E7
:10D7F80004D01D4A1279002A40F0C583114610460C
:10D808001A4A565C0D2E01F10C0100F0E682013037
:10D818001528F6D1FEF77ABCDBF8E400144B90F833
:10D828003A109D7841446429A8BF642121EAE17136
:10D8380080F83A10002D40F0BC8316F0A1FC24E4D7
:10D8480078280020B4690020DB0FC9BFDB0F49C06E
:10D85800F0640020F03900204A290020A828002080
:10D868008C2E00203C2500205869002030D6020864
:10D878000D2F0020DBF8E4008178B74B4144C8291C
:10D88800A8BFC82121EAE17181709B78002BD4D010
:10D89800142019F0A1FEDBF8E400CEE7DBF8E40081
:10D8A800AD4B90F83B109D784144FE29A8BFFE215E
:10D8B80021EAE17180F83B10002DBED0162019F046
:10D8C8008BFEDBF8E400B8E7089AA34B5178414493
:10D8D800B1F5967FA8BF4FF4967121EAE1715170B6
:10D8E8009B78002B40F02283DBF8E400A5E7DBF807
:10D8F800E400994B01799B784144C829A8BFC82105
:10D9080021EAE1710171002B40F04283102D94D07F
:10D918004178914B4144C829A8BFC82121EAE17147
:10D9280041709B78002B88D0132019F055FEDBF846
:10D93800E40082E7DBF8E400874BC1789B78414438
:10D94800C829A8BFC82121EAE171C170002B40F0A5
:10D95800F9820F2D3FF471AF01787F4B4144C829FC
:10D96800A8BFC82121EAE17101709B78002B3FF420
:10D9780064AF122019F030FEDBF8E4005DE7089A86
:10D98800754BD1799878414481F30801D171002809
:10D99800AAD0052019F020FEDBF8E4004DE7DBF8FB
:10D9A800E4006D4B017A9D784144C829A8BFC8217D
:10D9B80021EAE1710172002D3FF43FAF0B2019F00D
:10D9C8000BFEDBF8E40038E7DBF8E400624BC179D2
:10D9D8009D784144C829A8BFC82121EAE171C171D5
:10D9E800002D3FF42AAF0A2019F0F6FDDBF8E40019
:10D9F80023E7DBF8E400584B81799D784144C82936
:10DA0800A8BFC82121EAE1718171002D3FF415AF4B
:10DA1800092019F0E1FDDBF8E4000EE7DBF8E4008B
:10DA28004D4B41799B784144C829A8BFC82121EAB8
:10DA3800E1714171002B40F07F82112D7FF41CAF02
:10DA4800FBE6DBF8E40087E7DBF8E40060E7089A28
:10DA5800414B9179987841446429A8BF642121EA0F
:10DA6800E1719171002840F08A820D2D3FF43CAF9E
:10DA7800089A394B5179987841446429A8BF6421A0
:10DA880021EAE171517100283FF42EAF0E2019F000
:10DA9800A3FDDBF8E400D0E6089A15794544642D27
:10DAA800A8BF642525EAE575157119F0AFFD2A4B65
:10DAB8009B78002B3FF418AF0320294619F08CFD02
:10DAC800DBF8E400B9E6089A234B11784144FA29B7
:10DAD800A8BFFA2121EAE17111709B78002B3FF46D
:10DAE80003AF012019F078FDDBF8E400A5E6089AF9
:10DAF800194B917841446429A8BF642121EAE17156
:10DB080091709B78002B3FF4EFAE022019F064FD72
:10DB1800DBF8E40091E6139AFFF712BB0F4B1B7872
:10DB2800002B3EF4EFAA0E4BDB78002B7EF4EAAA1A
:10DB380095F8A8300133DBB2032B85F8A8307EF6C0
:10DB4800E1AA084B5B7813B9002F7EF4DBAA11F029
:10DB5800A7FFFFF749BA00BF0D2F00204969002031
:10DB6800646900203C3A0020C04BC1491A684FF450
:10DB78007A73B3FBF2F3C3EB431203EB8202059B08
:10DB88001B68D200A1F8A82003F00403FEF7BEBA70
:10DB980034F911109878B1F5617F4FF4966393FBCF
:10DBA800F0F372DB40F633008142A8BF01460C2D2A
:10DBB800A1F5617191FBF3F100F00D81182D7FF44F
:10DBC80064AAC9B2C8290B46A8BFC823DBF8E40079
:10DBD800C57D5FFA83FEAE453FF457AA5B1BA54A95
:10DBE80080F817E048BF0733DB1092785D1CEDB270
:10DBF8003AB9002D3FF449AA284610F0FBFCFFF77C
:10DC080044BA182019F0E8FCF3E79B499B4BCA6813
:10DC18001B688B609B1AC82B7FF629AB012381F800
:10DC28002130FFF724BBD8F80010DBF81C200A4489
:10DC3800CBF81820FFF7E5BB914B00220120A5E5A2
:10DC4800F0EE477AFEF7F8BCB0EE677AFEF7DEBC76
:10DC58008C4A1268970304D58B4A1279002A40F03F
:10DC6800EE808A4A18461946175C0B2F00F10C0003
:10DC780023D001311529F7D1002285F8A720FFF715
:10DC88006BB8834B0122022080E50C2D7AD1002548
:10DC98002946804B09915B78AB423FF4F6A92846A8
:10DCA80009F0CCFA734B09999B781BB1C9B20C20C7
:10DCB80019F092FC0135EDB29BE7774FD7F800C019
:10DCC8004800BCF1000F09D000EB010E02EB8E0EEC
:10DCD8009CF801C09EF801E0E645CDD200EB010EAC
:10DCE8006E486F4902EB8E024FF0000E3A60A0F8C2
:10DCF80000E0C1F800E0BFE7B0EE667AFFF7E7BBE7
:10DD0800F0EE476AFFF7F9BBD8F80020BAF80630FA
:10DD1800642101FB0323CBF81030FFF748BB06232F
:10DD28001A4641E501231A463EE502231A463BE519
:10DD380003231A4638E504231A4635E505231A460F
:10DD480032E512F061FA059B1B6803F00403FEF745
:10DD5800DDB915F045FBFDF775F915F029FB02F063
:10DD68001BF9012010F046FC95F8A620FFF710B823
:10DD7800059B4C4A1B684FF4C871118003F00403DB
:10DD8800FEF7C4B9182D7FF480A900210B461DE7C2
:10DD98000B464FF6FE71444A908956890144334434
:10DDA8005381918115F01CFBFDF74CF915F000FB30
:10DDB80002F0F2F8012010F01DFC059B1B68002200
:10DDC80003F0040385F8A720FEF7A0B90B4602214B
:10DDD800E1E70223DFE7CDB25BE72F4FD7F800E09A
:10DDE8004100BEF1000F08D00E1802EB86069EF81F
:10DDF80001E076787645BEF489A90144274E284883
:10DE080002EB810200213A6031800160FEF77EB9A1
:10DE18000121002017F097F895F8A620FEF7DDBF3E
:10DE28000021FF2017F08FF895F8A620FEF7D2BF43
:10DE3800012017F088F895F8A620FEF7C8BF1B4AFE
:10DE48001278002A7FF40DAF10F0DAFA069B1B78DF
:10DE580003F0010310E74FF6FE739CE7002101224F
:10DE680085F8A91085F8AA20FEF750B9085C0020AB
:10DE7800E45300200D2F002064690020C0530020C7
:10DE8800B62800203C2500205869002030D602081A
:10DE9800002900208C2E0020241E0020961E002021
:10DEA800981E00205C6E0020183A0020CD4F0020FC
:10DEB800039A115D9847032C1BDC40F2EE2240F6D2
:10DEC800CA0C00283EF4A4AD39F824E0BAF80210D0
:10DED8004FF47A73A0EB0E0003FB00F0A1EB0E01E8
:10DEE80090FBF1F018449042B8BF10466045A8BFB7
:10DEF800604600B2FEF78CBD002F3EF484A895F86A
:10DF0800A5E0BEF1000F3EF4B7A810F079FA96F834
:10DF180000E085F8A580FEF7AFB80C2010F08CFA69
:10DF2800059B1B6803F00403FEF7F0B8152019F0F1
:10DF380053FBDBF8E40080E4112019F04DFBDBF81B
:10DF4800E4007AE50F2019F047FBDBF8E40000E570
:10DF58003BB11E491E4A09684FF47A7000FB03134F
:10DF6800136095F8A530002B3EF486A810F048FA07
:10DF7800002385F8A53096F800E0FEF77DB80D205F
:10DF880019F02AFB71E5134A1278B2B1084637E452
:10DF9800102019F021FBDBF8E400B7E495F8A6306F
:10DFA800FEF7CCBE11F07CFD002385F8A530FEF706
:10DFB80061B8172019F010FB96E410F021FA059BC0
:10DFC8001B6803F00403FEF7A1B800BFC05300208C
:10DFD800E4520020CD4F0020436A826970B4D154C6
:10DFE800436A0469426B0133A34228BF002343629A
:10DFF800DAB1116811F0010101D070BC7047856A6F
:10E0080086699D422E44D6600BD3641B546081629E
:10E018001368002143F0010380F8441070BC1360BA
:10E0280070475D1B55608362F2E7026D136843F029
:10E0380080031360E1E700BF026B10B462B1036CA8
:10E04800C2684469D11A013B615C5DF8044B08BFA2
:10E0580013460364C8B27047016A4369C4685B5CCD
:10E068000131A14228BF114601625DF8044BD8B2C4
:10E07800704700BF436B13B190F844007047836A40
:10E08800406A181AB0FA80F040097047416A836AFA
:10E0980099420AD3CB1A416B026961B14968501E93
:10E0A8000B4483420AD2C01A704702691144CB1A42
:10E0B800416B0029F2D1501EC01A704700207047EA
:10E0C800036B43B1026C5B6893422FBF981AC06818
:10E0D8009B1AC0187047C269036A9A422FBFD01AA8
:10E0E800C0688018C01A70470A4B30B503F1140491
:10E0F80093F900205D78072AC8BF143A81180433C1
:10E108000D7313F8025C855413F8012C0A76A342A8
:10E11800EED130BD58D3020803682DE9F041DF691C
:10E128001FB13B46BDE8F0411847002A164611DDED
:10E1380004460D460E4400E023689B682046984735
:10E148000028F9D0236815F8011B1B68204698475A
:10E15800AE42F1D1BDE8F0810023292125220170CA
:10E1680042708370C370704730B50446006D6171AA
:10E178000368A26823F00103036087B0A3790092C3
:10E1880013F004023DD04FF4805213F002030192C1
:10E1980044D102934FF480630022039311F00103EA
:10E1A800059237D1049308238D07694648BF049325
:10E1B80016F014FE6079236DA17900F00202002A9E
:10E1C80015BF4FF440324FF480324FF4003400242E
:10E1D80010F0010F586808BF2246CC074CBF024315
:10E1E80020EA02025A609A6809074CBF42F0080206
:10E1F80022F008029A601A6842F001021A6007B019
:10E2080030BD13F0020301920BD04FF400551346B2
:10E218000295C1E7042304930C23C5E74FF4005388
:10E22800B7E70293B8E700BF10B50446006DA160D8
:10E23800036823F001030360A37986B013F0040296
:10E24800009141D04FF4805213F00203019244D15F
:10E2580002934FF4806362790393D1074FF0000370
:10E268000493059345BF0423049308230C236946AC
:10E27800920748BF049316F0B1FD6079236DA17928
:10E2880000F00202002A15BF4FF440324FF48032EA
:10E298004FF40034002410F0010F586808BF2246DC
:10E2A800CC074CBF024320EA02025A609A68090769
:10E2B8004CBF42F0080222F008029A601A6842F045
:10E2C80001021A6006B010BD13F00203019207D0D4
:10E2D8004FF4005113460291BDE74FF40053B7E7DE
:10E2E8000293B8E72DE9F0470569C3681D4028D0B7
:10E2F8000F4606464FF000484FF00009B5FA85F37F
:10E3080028FA03F2D2431B3B32611540042B16D87E
:10E31800DFE803F03129211903007B6A002B32D092
:10E3280003F1FF3A1FFA8AFAC7F824903C6A34B11D
:10E3380023682046514698476468002CF8D1002D80
:10E34800DCD1BDE8F0873868716B036889B29847FB
:10E35800002DD3D1F5E77868B16B036889B2984787
:10E36800002DCBD1EDE7B868F16B036889B2984707
:10E37800002DC3D1E5E7F868316C036889B2984786
:10E38800002DBBD1DDE7F36A1FFA83FACEE700BFA1
:10E398002DE9F04104684A4DA30AAB4272D009D86E
:10E3A800B3F5801F6AD04A3DAB425AD14FF0700E88
:10E3B800022608E0434DAB4268D00135AB4252D14A
:10E3C8004FF0C00E042647794FEA970C002961D018
:10E3D800B000634685190227D4F80C809F400CEBE7
:10E3E8004503BFB2384D03F1040C47EA080745F866
:10E3F800231045F82C20E760EFF31181502282F3B7
:10E408001288821905EBC202136973B313620433CD
:10E41800821905EBC202576917B11F6053690433AB
:10E42800821905EBC202976917B11F60936904331B
:10E43800821905EBC202D76917B11F60D36904338B
:10E448000027CAB21F6082F31188304405EBC00070
:10E45800036A6BB9E3684FF6FE721340E360BDE8E8
:10E46800F081BDE8F081BDE8F08105EB0E03CFE750
:10E47800E36843F00103E360BDE8F0814FF0480E24
:10E488000126A0E74FF0200E00269CE74FF0980EDB
:10E49800032698E7BF08022306FA03F0BB40DB43D4
:10E4A800E768094D9BB23B4087190CEB470CE360CA
:10E4B8000CF1040345F82C1045F823209CE700BF15
:10E4C8004B00100051001000046A002030B50368AA
:10E4D8005C4D18885C4CB4FBF2F20139013AAB424E
:10E4E80094B283B089B282B266D05848834263D06E
:10E4F800B3F1804F60D0A0F5983083425CD000F52E
:10E508008060834258D0524883425BD000F58060D7
:10E5180083427CD022F4407200F58C3092B2834260
:10E528001A80D9621C850ED0484A93420BD002F556
:10E538004062934207D002F58062934203D002F50D
:10E548008062934201D100221A8601225A611A88F8
:10E558003C4992B242F001028B421A8061D0B3F179
:10E56800804F60D03B4A93425FD002F5806293426D
:10E578005DD002F5006293425BD002F5806293425F
:10E5880059D002F59032934257D002F54062934237
:10E5980055D002F5806293421ED002F58062934204
:10E5A80008BF092219D002A84FF0012340F8043D02
:10E5B80012F03EF903B030BD254822F070028342C4
:10E5C80092B2A3D101201A80D9621C8558611A8899
:10E5D80092B202431A80C5E708221F4B03EBC2031D
:10E5E80001A85C798DF80440012300228DF80530DC
:10E5F8008DF807308DF8062012F01AF91B2CD9D1A6
:10E60800164B019301A812F013F903B030BD012095
:10E618001A80D9621C8558611A8892B202431A80FE
:10E628009DE70022D9E70122D7E70222D5E7032296
:10E63800D3E70422D1E70522CFE70622CDE7072258
:10E64800CBE700BF002C014000A24A04003401407F
:10E65800001000400004004088D30208190100019E
:10E668001F4B98422CD0B0F1804F2BD0A3F5943398
:10E67800984229D003F58063984227D003F50063B8
:10E68800984225D003F58063984223D003F5903350
:10E69800984221D003F5406398421FD003F5806368
:10E6A800984207D003F58063984208BF092202D038
:10E6B8000020704708220B4B03EBC2031879704700
:10E6C8000022F8E70122F6E70222F4E70322F2E744
:10E6D8000422F0E70522EEE70622ECE70722EAE744
:10E6E800002C014088D302082DE9F04F013085B095
:10E6F800C3B203930B4602918B4C8C4E002B00F057
:10E7080099808B4D8B4FDFF8309217F0F3FB4FF465
:10E71800FA7A4FF0100C4FF47A70D9F80430C3F33A
:10E728000803002B40F0DE80EFF31183002B40F04C
:10E73800D9802968A26800BF2B689942F9D1D7F817
:10E7480000E000FB0EF39B1AB3FBFEF300FB013164
:10E758004FF0010E0191D9F80430C3F30803002BE0
:10E7680040F08780EFF31183002B40F082802B6804
:10E77800A16800BF2A689342F9D1D7F800B000FB1E
:10E788000BF2521AB2FBFBF200FB0323019A9B1A0D
:10E79800B3F57A7FDFD3BAF1010ABED1039B002B10
:10E7A80040F0BD804FF47A7ADFF88C9150464FF0F4
:10E7B800100CD9F80430C3F30803002B75D1EFF31C
:10E7C8001183002B71D12968A26800BF2B68994278
:10E7D800F9D1D7F800E000FB0EF39B1AB3FBFEF368
:10E7E80000FB01314FF0010E0191D9F80430C3F359
:10E7F800080313BBEFF31183FBB92B68A16800BFB3
:10E808002A689342F9D1D7F800B000FB0BF2521AEC
:10E81800B2FBFBF200FB0323019A9B1AB3F57A7F44
:10E82800E3D3BAF1010AC4D1029B013B0293002B46
:10E838007FF467AF05B0BDE8F08FEFF311888CF374
:10E848001288A1682368DB0344BFC6F800E0A1680A
:10E858002B6832685FFA88F888F31188D7F8008047
:10E868001A4400FB08F35B1AB3FBF8F300FB02330E
:10E87800D2E7EFF311888CF31288A1682368DB03D1
:10E8880044BFC6F800E0A1682B6832685FFA88F8D0
:10E8980088F31188D7F800801A4400FB08F35B1A44
:10E8A800B3FBF8F300FB023370E7EFF311828CF34C
:10E8B8001288D4F808E02368D90303D5012333600C
:10E8C800D4F808E02B683168D2B282F311883A682C
:10E8D800194400FB02F3A3EB0E03B3FBF2F300FBB6
:10E8E80001317FE7EFF311828CF31288D4F808E046
:10E8F8002368D90303D501233360D4F808E02B68D3
:10E908003168D2B282F311883A68194400FB02F3E5
:10E91800A3EB0E03B3FBF2F300FB013118E7184633
:10E9280012F0A6F93EE700BF10E000E0BC5300205B
:10E93800C0530020C453002000ED00E0204B5B686A
:10E94800C3F3080330B4BBB9EFF31183A3B91D4B6C
:10E958001D4C1868A16800BF1A689042F9D11B4B7A
:10E968001C684FF47A7202FB04F3591AB1FBF4F1F4
:10E9780030BC02FB00107047EFF31182102383F3C1
:10E98800128811498C680B6813F4803F104B02D031
:10E99800012018608C680B49D2B20D68186882F3A0
:10E9A80011880A4B19684FF47A72284402FB01F364
:10E9B8001B1B30BCB3FBF1F302FB0030704700BFF8
:10E9C80000ED00E0C053002010E000E0C453002038
:10E9D800BC5300202DE9F84F8046FFF7AFFF254EC6
:10E9E8002549DFF8A0E0254A254D844610274FF435
:10E9F8007A740120DEF80430C3F30803D3B9EFF3C7
:10EA08001183BBB90B68D2F808A000BFD1F80090F9
:10EA18004B45F7D1D6F800B004FB0BF9A9EB0A096E
:10EA2800B9FBFBF904FB0393A3EB0C034345E1D3C8
:10EA3800BDE8F88FEFF3118A87F31288D2F808B08F
:10EA48001368DB0344BF2860D2F808B00B68D5F818
:10EA580000905FFA8AFA8AF31188D6F800A09944E0
:10EA680004FB0AF3A3EB0B03B3FBFAF304FB093330
:10EA7800DAE700BFC4530020C053002010E000E0D4
:10EA8800BC53002000ED00E02DE9F04FDFF830C165
:10EA9800474A4849484E494D8046102718F1FF38E3
:10EAA800C0F08480DCF80430C3F30803002B5CD189
:10EAB800EFF31183002B58D10B68946800BF0868E6
:10EAC8008342F9D1D6F800904FF47A7000FB09FE22
:10EAD800AEEB040EBEFBF9FE00FB03EEDCF80430DF
:10EAE800C3F308034FF47A740120FBB9EFF31183E1
:10EAF800E3B90B68D2F808A000BFD1F800904B45E5
:10EB0800F7D1D6F800B004FB0BF9A9EB0A09B9FB59
:10EB1800FBF904FB0393A3EB0E03B3F57A7FBDD295
:10EB2800DCF80430C3F30803002BDFD0EFF3118ABD
:10EB380087F31288D2F808B01368DB0344BF286053
:10EB4800D2F808B00B68D5F800905FFA8AFA8AF311
:10EB58001188D6F800A0994404FB0AF3A3EB0B0331
:10EB6800B3FBFAF304FB0933D5E7EFF3118487F31A
:10EB78001288D2F808901368D80303D501232B60B4
:10EB8800D2F808900B682868E4B284F31188D6F8A4
:10EB980000A04FF47A7400EB030E04FB0AF3A3EB16
:10EBA8000903B3FBFAF304FB0E3E97E7BDE8F08FC9
:10EBB80010E000E0C0530020C4530020BC530020E4
:10EBC80000ED00E030B4EFF31183102282F31288D5
:10EBD8000649074C0A680748013200250A60256083
:10EBE800DBB2026883F3118830BC7047C053002041
:10EBF800BC53002010E000E01D4B70B59C68236DED
:10EC0800226BDD69C2B1636B2BB12B0702D5236D73
:10EC180008221A6270BD2A06F7D5A26A616A8A427A
:10EC28001FD0511CA069A162825C2069266D8142B7
:10EC38003285EAD3A362E8E7A906E4D5E26A1AB105
:10EC4800988C80B29047DEE7E1699B8C6069DBB203
:10EC58004E1CE6614354E169E368994228BFE261CA
:10EC6800D1E7226D136823F080031360CDE700BF5E
:10EC7800543700201D4B70B55C68236D226BDD692D
:10EC8800C2B1636B2BB12B0702D5236D08221A6220
:10EC980070BD2A06F7D5A26A616A8A421FD0511C44
:10ECA800A069A162825C2069266D81423285EAD31F
:10ECB800A362E8E7A906E4D5E26A1AB1988C80B2A3
:10ECC8009047DEE7E1699B8C6069DBB24E1CE66128
:10ECD8004354E169E368994228BFE261D1E7226DB4
:10ECE800136823F080031360CDE700BF543700207A
:10ECF8001D4B70B51C68236D226BDD69C2B1636B57
:10ED08002BB12B0702D5236D08221A6270BD2A0683
:10ED1800F7D5A26A616A8A421FD0511CA069A16214
:10ED2800825C2069266D81423285EAD3A362E8E7D6
:10ED3800A906E4D5E26A1AB1988C80B29047DEE75A
:10ED4800E1699B8C6069DBB24E1CE6614354E16962
:10ED5800E368994228BFE261D1E7226D136823F086
:10ED680080031360CDE700BF5437002003685B6A57
:10ED780003B11847704700BF03681B6A03B11847FF
:10ED8800704700BF03682DE9F041DF691FB13B46BA
:10ED9800BDE8F0411847002A164611DD04460D4625
:10EDA8000E4400E023689B68204698470028F9D065
:10EDB800236815F8011B1B6820469847AE42F1D11D
:10EDC800BDE8F08103689B69184700BF0368DB68EA
:10EDD800184700BF03689B68184700BF03685B6853
:10EDE800184700BF03681B68184700BF054B53F856
:10EDF800203033B11A689B88918A0B4218BF1B04D4
:10EE0800936170478C53002010B50409013C052C10
:10EE180017D80D4B33F8142000F00F0042FA00F316
:10EE280013F001030DD0012303FA00F0013810405C
:10EE38001BF0AEFB054A064B125D104403EBC00005
:10EE480010BD002010BD00BFC8E70208D4E70208C3
:10EE5800EC4200202DE9F04F4A484B4B4B4C4FF009
:10EE680090414FF0010A4FF002094FF004084FF0AB
:10EE7800080C4FF0100E20274026802530F8022B72
:10EE880012F0010F03D01960A3F804A0083312F0A0
:10EE9800020F03D01960A3F80490083312F0040F8E
:10EEA80003D01960A3F80480083312F0080F03D0C8
:10EEB8001960A3F804C0083312F0100F03D01960CA
:10EEC800A3F804E0083312F0200F02D019609F80E5
:10EED800083312F0400F02D019609E80083312F0F8
:10EEE800800F02D019609D80083312F4807F05D00E
:10EEF8004FF4807B1960A3F804B0083312F4007F44
:10EF080005D04FF4007B1960A3F804B0083312F45D
:10EF1800806F05D04FF4806B1960A3F804B00833F4
:10EF280012F4006F05D04FF4006B1960A3F804B019
:10EF3800083312F4805F05D04FF4805B1960A3F8A2
:10EF480004B0083312F4005F05D04FF4005B196079
:10EF5800A3F804B0083312F4804F05D04FF4804B67
:10EF68001960A3F804B00833D20B04D04FF4004260
:10EF780019609A80083301F58061A1427FF47EAF61
:10EF8800BDE8F08FC8E70208EC42002000180048EE
:10EF9800002867D003682DE9F04F03F138445C4E30
:10EFA800A40A0125345D04F01F066409022C05FA41
:10EFB80006F558D0032C00F0A580012C58D0808885
:10EFC800B0FA80F4C4F11F04A4B2E50803EB850588
:10EFD80004F007042E6AA4000F27A74026EA0706B4
:10EFE8002E622E6A01F00307A2407C1E3243012CD8
:10EFF800C1F3810CC1F300182A62C1F341113CD955
:10F00800C60700F18980850700F19580440700F163
:10F01800A380020700F1B180C60600F1BF80850613
:10F0280000F1CD80440600F1DB80020600F1E980A2
:10F03800C60500F1F780850500F10581440500F15A
:10F048001381020500F12181C60400F12F81850496
:10F0580000F13D81440400F14B81020400F1598123
:10F06800BDE8F08F70472B4CA6693543A561A6E72C
:10F07800284C666935436561A1E7002422464FF0B4
:10F08800010E4FF0030904E00132102A04F10204D2
:10F09800E6D00EFA02F636EA0005F5D1D3F808A054
:10F0A80009FA04F5ED430AEA050AC3F808A0D3F8FB
:10F0B80008B00CFA04FA4AEA0B0AC3F808A0B3F835
:10F0C80004A01FFA8AFA2AEA06069E80B3F804A06A
:10F0D80008FA02F646EA0A06B6B29E801E682E4074
:10F0E8001E60D3F800A007FA04F646EA0A061E6076
:10F0F800D3F80CA001FA04F605EA0A0A46EA0A055A
:10F10800DD60C1E7034CE6693543E56157E700BFB9
:10F11800DCE70208001002401A6822F003021A60B5
:10F128001A683A431A60DA6822F003020A4385072C
:10F13800DA607FF56BAF1A6822F00C021A601A6861
:10F1480042EA87021A60DA6822F00C0242EA810277
:10F158004407DA607FF55DAF1A6822F030021A6062
:10F168001A6842EA07121A60DA6822F0300242EAA4
:10F178000112DA6002077FF54FAF1A6822F0C00269
:10F188001A601A6842EA87121A60DA6822F0C00226
:10F1980042EA8112C606DA607FF541AF1A6822F4A6
:10F1A80040721A601A6842EA07221A60DA6822F482
:10F1B800407242EA01228506DA607FF533AF1A68A9
:10F1C80022F440621A601A6842EA87221A60DA68F2
:10F1D80022F4406242EA81224406DA607FF525AFD4
:10F1E8001A6822F440521A601A6842EA07321A6012
:10F1F800DA6822F4405242EA0132DA6002067FF508
:10F2080017AF1A6822F440421A601A6842EA873235
:10F218001A60DA6822F4404242EA8132C605DA60AE
:10F228007FF509AF1A6822F440321A601A6842EA78
:10F2380007421A60DA6822F4403242EA0142850540
:10F24800DA607FF5FBAE1A6822F440221A601A6869
:10F2580042EA87421A60DA6822F4402242EA81428E
:10F268004405DA607FF5EDAE1A6822F440121A60A0
:10F278001A6842EA07521A60DA6822F4401242EA2F
:10F288000152DA6002057FF5DFAE1A6822F4400207
:10F298001A601A6842EA87521A60DA6822F4400251
:10F2A80042EA8152C604DA607FF5D1AE1A6822F0CC
:10F2B80040721A601A6842EA07621A60DA6822F035
:10F2C800407242EA01628504DA607FF5C3AE1A68CB
:10F2D80022F040621A601A6842EA87621A60DA68A5
:10F2E80022F0406242EA81624404DA607FF5B5AEFA
:10F2F8001A6822F040521A601A6842EA07721A60C5
:10F30800DA6822F0405242EA0172DA6002047FF5BC
:10F31800A7AE1A6822F040421A601A6842EA877754
:10F328001F60DA6822F0404242EA8171D960BDE884
:10F33800F08F00BF002852D0036803F138422DE94E
:10F34800F04F920A504DAA5C02F01F0552090124A1
:10F35800022A04FA05F443D0032A00F09080012A17
:10F3680043D001F003077A1E012AC1F3810CC1F3CF
:10F3780000188088C1F341113CD9C60700F1888084
:10F38800850700F19480440700F1A280020700F18C
:10F39800B080C60600F1BE80850600F1CC80440628
:10F3A80000F1DA80020600F1E880C60500F1F68077
:10F3B800850500F10481440500F11281020500F180
:10F3C8002081C60400F12E81850400F13C814404AB
:10F3D80000F14A81020400F15881BDE8F08F7047BE
:10F3E8002A4A95692C439461BBE7284A55692C43FE
:10F3F8005461B6E7002422464FF0010E4FF003098E
:10F4080004E00132102A04F10204E6D00EFA02F6F2
:10F4180036EA0005F5D1D3F808A009FA04F5ED435A
:10F428000AEA050AC3F808A0D3F808B00CFA04FAE7
:10F438004AEA0B0AC3F808A0B3F804A01FFA8AFA2C
:10F448002AEA06069E80B3F804A008FA02F646EAFD
:10F458000A06B6B29E801E682E401E60D3F800A031
:10F4680007FA04F646EA0A061E60D3F80CA001FA69
:10F4780004F605EA0A0A46EA0A05DD60C1E7034A16
:10F48800D5692C43D4616CE7DCE702080010024020
:10F498001A6822F003021A601A683A431A60DA6896
:10F4A80022F003020A438507DA607FF56CAF1A6819
:10F4B80022F00C021A601A6842EA87021A60DA68B7
:10F4C80022F00C0242EA81024407DA607FF55EAF5F
:10F4D8001A6822F030021A601A6842EA07121A60A3
:10F4E800DA6822F0300242EA0112DA6002077FF598
:10F4F80050AF1A6822F0C0021A601A6842EA8712EE
:10F508001A60DA6822F0C00242EA8112C606DA609E
:10F518007FF542AF1A6822F440721A601A6842EA0C
:10F5280007221A60DA6822F4407242EA012285064C
:10F53800DA607FF534AF1A6822F440621A601A68FC
:10F5480042EA87221A60DA6822F4406242EA81229B
:10F558004406DA607FF526AF1A6822F440521A6032
:10F568001A6842EA07321A60DA6822F4405242EA1C
:10F578000132DA6002067FF518AF1A6822F44042B9
:10F588001A601A6842EA87321A60DA6822F440423E
:10F5980042EA8132C605DA607FF50AAF1A6822F4BA
:10F5A80040321A601A6842EA07421A60DA6822F49E
:10F5B800403242EA01428505DA607FF5FCAE1A68FE
:10F5C80022F440221A601A6842EA87421A60DA680E
:10F5D80022F4402242EA81424405DA607FF5EEAE29
:10F5E8001A6822F440121A601A6842EA07521A602E
:10F5F800DA6822F4401242EA0152DA6002057FF525
:10F60800E0AE1A6822F440021A601A6842EA875289
:10F618001A60DA6822F4400242EA8152C604DA60CB
:10F628007FF5D2AE1A6822F040721A601A6842EA70
:10F6380007621A60DA6822F0407242EA01628504C1
:10F64800DA607FF5C4AE1A6822F040621A601A6860
:10F6580042EA87621A60DA6822F0406242EA81620E
:10F668004404DA607FF5B6AE1A6822F040521A6098
:10F678001A6842EA07721A60DA6822F0405242EACF
:10F688000172DA6002047FF5A8AE1A6822F04042DF
:10F698001A601A6842EA87771F60DA6822F04042E7
:10F6A80042EA8171D960BDE8F08F00BF10B10368EC
:10F6B80082881A85704700BF10B1036882889A61F2
:10F6C800704700BF38B100298388026814BF002141
:10F6D80010218B40936170470E4B1B8801463BB944
:10F6E8000D4B0E4A1B7810680BB981F00101E9E750
:10F6F8000B4B5A691AB118B91A68106058747047D8
:10F70800084A18681188084A92FBF1F20121026040
:10F7180059747047985300209A5300209C53002036
:10F72800A0530020B853002020A1070010B40A4BB2
:10F738000A4A1C7801238340234052F8200029B943
:10F74800B3FA83F149095DF8044BBBE7191C18BFEC
:10F7580001215DF8044BB5E7885300208C53002045
:10F7680030B1036882881B8A1A4214BF0120002026
:10F77800704700BF2DE9F0410B4E346873691C4097
:10F788000FD0DFF828800127B4FA84F3C3F11F03F0
:10F7980007FA03F558F8230003689847AC437561E6
:10F7A800F2D1BDE8F08100BF0004014010530020F1
:10F7B8002DE9F0410B4E346873691C400FD0DFF817
:10F7C80028800127B4FA84F3C3F11F0307FA03F56D
:10F7D80058F8230003689847AC437561F2D1BDE837
:10F7E800F08100BF00040140105300202DE9F041D2
:10F7F8000B4E346873691C400FD0DFF8288001274E
:10F80800B4FA84F3C3F11F0307FA03F558F8230089
:10F8180003689847AC437561F2D1BDE8F08100BF39
:10F8280000040140105300202DE9F0410B4E3468CC
:10F8380073691C400FD0DFF828800127B4FA84F3DD
:10F84800C3F11F0307FA03F558F823000368984724
:10F85800AC437561F2D1BDE8F08100BF00040140FE
:10F86800105300202DE9F0410B4E346873691C4099
:10F878000FD0DFF828800127B4FA84F3C3F11F03FF
:10F8880007FA03F558F8230003689847AC437561F5
:10F89800F2D1BDE8F08100BF000401401053002000
:10F8A80003680A7A591C01601A70704738B50B4C06
:10F8B80023688BB15A68821A002A054604DA0CE0DC
:10F8C8005A68AA1A002A07DB9A68226018461A683A
:10F8D80090472368002BF3D138BD38BDA8640020B9
:10F8E8000B4B002210B4027203F1A004042102E0C1
:10F8F800072A09DC9979890702D5197981540132D7
:10F908009C4203F11403F3D15DF8044B704700BF28
:10F91800B0E9020810B40D4C04232146002200E08F
:10F928008B7913F0010301F1140106D10132092A80
:10F93800F6D103705DF8044B704702EB820204EBCA
:10F9480082025DF8044B137903707047B0E902082E
:10F9580001231521222241704271037003717047FF
:10F968002DE9F0410B78057BDB43DFB200F1130290
:10F9780000F11D0302F8015F9342FBD1DFF890E02C
:10F9880000F12701002203F8012F9942FBD114212D
:10F998000524002647FA04F303F00103002B1E4454
:10F9A80014BF4FF019084FF00A0814F0010FF6B20F
:10F9B80014BFAC464FF0000C0023CA1810FA82F2AC
:10F9C8000133434582F814C0F7D15A1E92B201326E
:10F9D800013C8B18621C9BB201D01946DAE716F07D
:10F9E800010F14BF19240A240022991810FA81F172
:10F9F8000132A2420D75F8D113449BB25A1C03443C
:10FA0800002192B21975AEF800200261BDE8F081BC
:10FA1800FC2300202DE9F04FDFF890A0BAF802305F
:10FA28000B3383B01FFA83F901F1060B4FF001087D
:10FA38004FF0000C002711F801EB3E464C4601221E
:10FA4800A4F10B039BB2019105E001339BB2017B4A
:10FA580029759C4208D0C518002AF6D1C51801336B
:10FA68009BB29C422A75F6D103190136092F0199D8
:10FA780083F814C0F6B20CD0092E15D008FA07F393
:10FA880013EA0E0F14BF012200220C34A4B201376E
:10FA9800D6E709F1780959451FFA89F9CAD1AAF8B0
:10FAA80002C003B0BDE8F08F0022EEE7FC2300207F
:10FAB8002DE9F047DFF85C80B8F8043004331FFA0A
:10FAC80083FC01F109094FF0010E11F8017B64462E
:10FAD8000026231F0EFA06F29BB23A40C2B1B0F8D4
:10FAE8000CA0C51801339BB29C4285F814A0F5D12F
:10FAF80001360434082EA4B2EBD10CF1200C494590
:10FB08001FFA8CFCE1D10023A8F80430BDE8F08787
:10FB18009246E6E7FC23002010B40268047B1168D3
:10FB28000223A340194209D00649406800240C70FA
:10FB380001684FF6FE742140016053605DF8044B84
:10FB4800704700BFCC6A002070B54E680546304645
:10FB58001AF074F831460446024628681AF020FE66
:10FB68002A68131901333B212B60115570BD00BF62
:10FB780008B50AF0C7FD024B024ADA60FEE700BF8B
:10FB880000ED00E00400FA05024A034B12781978E8
:10FB980005F0D0B96C1C00206D1C0020F0B5434B5B
:10FBA8001A6883B001235102414900935CBF03F1F5
:10FBB800805300930968D7005CBF43F0100300939B
:10FBC8008E073C4948BF43F0C603097848BF0093F5
:10FBD800D40548BF43F0006301F0EF0048BF00932D
:10FBE80008286D4655D00E2953D0D0033248009BC3
:10FBF80000784CBF43F4204343F40053D7044CBF70
:10FC080043F0C84343F0884300280CBF07200F2067
:10FC1800960648BF43F48073540748BF43F4003343
:10FC280043F400245205009402D5244A1279A2BB59
:10FC3800182936D001900027012639462846FCB2FB
:10FC4800FBF77FFE60B11E4B002203F5D87103E07D
:10FC58008B420FD013F80C2C944203F10C03F7D10C
:10FC68000137242FE9D195E80300164B83E80300F8
:10FC780003B0F0BD7A0904F01F0455F8223006FAE3
:10FC880004F4013723EA0404242F45F82240D4D190
:10FC9800E9E743F480530093A7E743F4C0130093C4
:10FCA800C6E7009B43F060730093C3E74C4900200C
:10FCB800185C0020603A0020444400209C4F00203B
:10FCC8005CCE0208641C00202DE9F84F4E014FF06D
:10FCD800000B174D8146904606F120075C465946B1
:10FCE80028465FFA8BFAFBF72CFEC0B1A64215D85E
:10FCF800A74213D900200F4A014604E00131242904
:10FD080014D012F80C0C504502F10C02F6D10A4B33
:10FD180001EB410103EB81014846C04701340BF177
:10FD2800010BBBF1240FDAD1BDE8F88F0021F3E70E
:10FD3800641C00205CCE020850CE020800210A4A4A
:10FD48000B4604E00133242B0BD012F80C1C88421C
:10FD580002F10C02F6D1054803EB430300EB8300E4
:10FD680070470020704700BF64CE020850CE0208DA
:10FD780000210A4A0B4604E00133242B0BD012F869
:10FD88000C1C884202F10C02F6D1054803EB430330
:10FD980000EB830070470020704700BF5CCE02086C
:10FDA80050CE02081C4C08B501210220FFF7BEFC0A
:10FDB800237803F00502052A2AD003F00903092B4A
:10FDC80008D000210120FFF7B1FC00210846FFF709
:10FDD800ADFCFEE7114A124B11681A680B68114C0A
:10FDE8004FF6FE7003400B601388206823F0010370
:10FDF8001B041B0C138018B1292200238271C371C4
:10FE080002224E21FFF7C4F82068FFF74FFCD8E71D
:10FE18000AF028FD2378D0E750370020786E0020BC
:10FE28007C6E0020E06E0020022828BF022010B45B
:10FE3800084C094B207000EBC00200EB8202074916
:10FE48005DF8044B013003EB4203C0B20B600EF0C7
:10FE5800D1BB00BF8C2E0020B6280020A828002087
:10FE680008B513F0BDFAFBF7EDF8BDE8084013F04C
:10FE78009FBA00BF38B5414B5A899989914224BF2E
:10FE880000225A81198ADA89914224BF0022DA8134
:10FE9800DA788AB1072A0FD0394C3A48A27801217A
:10FEA8000025062A01709970DD7150D92379DFED9C
:10FEB800366A002B3AD138BDDA79002A4CD09A78C4
:10FEC8003048DFED316A0178042A38BF042207EE92
:10FED800902AB8EEE77A07EE901A27EE267AF8EE1F
:10FEE800E77A9A7067EE877A254CA278062A2BD88B
:10FEF800264B03EB8203D3ED006AF4EEE76AF1EEDA
:10FF080010FA10DDC6EE877AFDEEE77A17EE903A22
:10FF1800102BA8BF1023012BB8BF0123DBB28B42E3
:10FF280028BF0B4603702379002BC4D0013A032A5B
:10FF3800C1D8B7EE000A80EE260A1AF0A5FD23887C
:10FF4800984238BF208038BDDFED0F6AD5E7DFED76
:10FF5800107AB0EE677ACBE79B780A48DFED0D6A36
:10FF6800017807EE103A07EE901AB8EEC77AF8EE65
:10FF7800E77A27EE267A67EE877AB5E7D05300202E
:10FF88001C4400200C3A00206F1203386CD302087E
:10FF98006F12833A6F1203392DE9F047A84FA94E23
:10FFA80013F01EFABE421ED2DFF82083DFF820933A
:10FFB8004446258862197DB14A450DD2052D0BD9D5
:10FFC80033886188C3F30B03994200F0D880144644
:10FFD80025886219002DEFD1716830461436FAF77A
:10FFE800B5FFBE42E4D3984A5378022B40F2EC8026
:08FFF8000023964953701378B1
:020000040801F1
:100000009548022B016000F2DF8003EBC301934AA5
:1000100003EB810302EB4303914C1846236013F07A
:100020006DFF904A1378A3F1170102290FD98E4969
:1000300011F83300002840F0D180D80001444978FD
:1000400029B18A4911F83330002B00F0F580884B34
:100050009A78042A00F0E78032B91A88B2F5F07F66
:1000600084BF4FF4F0721A80824D834A2B681A4085
:10007000002A00F0E480DE0700F1D080580400F18F
:10008000C880190700F1C0809A0100F1B7809B0475
:1000900000F1AD8023689A8CD98C914224BF002254
:1000A0009A84FFF7EBFE0BF0EFFF10B973480DF0E9
:1000B000A9FC17F0AFFA0021302271481CF0F5FDC1
:1000C000704B266803F1500102E00433994279D065
:1000D0001A78002AF9D19C78D8788442F5D26A49F6
:1000E0006A4B91F800E06A486A4D1C6B6A4B2860C5
:1000F000C827642111FB0E71DFF8E0E15960674FFA
:1001000030F8041C664DAEF8001000219960D960EB
:10011000196159619961D96183F8201083F8211020
:100120003A702E600CB113F09BF85E4B9FED5E5A57
:100130001B885E4A9FED5E6A557B5E4C5E495F4858
:10014000086006EE903AF8EEE66A1389C5EE265A84
:1001500007EE103A5389127BC4ED005A07EE903A2D
:10016000B8EEC77A564BF8EEE77A1D725A7227EE50
:10017000067A67EE867ABDE8F04783ED017AC3ED33
:10018000007A13F019B963799B077FF424AF716883
:1001900094F804A03046FAF7DDFE3388BAEB133F3B
:1001A0000BD173887068AA1FC3F30B039A4204F142
:1001B0000601A8BF1A461AF0F7FA1436BE42FFF439
:1001C000FBAE14E701228AE700231370234B23E7D9
:1001D000204903EB430301EB830110E7D8000D181E
:1001E0006D68002D7FF42AAF1725157026E7354876
:1001F000FAF7E6FE4020FAF7E3FE4BE746F2090085
:10020000FAF7DEFE2B6842E72F48FAF7D9FE2B6893
:100210003AE72E48FAF7D4FE2B6832E72C48FAF773
:10022000CFFE2B682AE71A8BB2F57A7FBFF41CAF9A
:100230004FF47A721A8317E71823137007E743F015
:1002400008032B6017E700BFD8230308F01F03083B
:100250008C2E00205E2E0020406E0020B62800204C
:10026000A8280020603A002014EE0208F0EB0208F3
:100270001C440020FC29002009600002CC6D0020F5
:10028000C4230020643A0020EC410020E037002025
:100290001C3A0020A87C002064690020861A0020F7
:1002A000F8230020801D0020C0C9FB48FC2300204B
:1002B00017B7D138841D0020E43B00203661023D91
:1002C000B83B002009400002016000020920000242
:1002D0000860000207F0030800000408086400201A
:1002E00008B513F081F8FAF7B1FE13F065F8FFF7DF
:1002F00057FE0120BDE808400EF080B938B5114C1A
:10030000114DAC4206D2616820461434FAF722FE41
:10031000AC42F8D30D4B1B78012B0FD00C4B0D4C7E
:100320000D4818600025257013F0E8FD0B4B0C4AB2
:1003300065701A60BDE8384015F01ABCFBF712FB77
:10034000ECE700BFF01F0308D8230308803B002020
:10035000A82800208C2E0020B6280020406E002007
:100360005E2E002008B5FFF7C9FF13F03DF8FAF73D
:100370006DFEBDE8084013F01FB800BFF0B50C29B2
:100380002BD8DFE801F06F2A2A2A4C2A2A2A2B2AA6
:100390002A2A0700046AB2F80CE097881668674DAD
:1003A00024F480540462036A4468C16923F400534E
:1003B00043EA0E3321F4E641A84243EA073341EA17
:1003C000062100F0B58005F50065A84200F0B08078
:1003D00092684460C16102640362F0BD046A968958
:1003E0009588D2F800E0554F24F480740462036AC3
:1003F0004468C16923F4007343EA062321F07301C2
:10040000B84243EA052341EA0E017ED04C4DA84292
:100410007BD092684460C161C2630362F0BD046A2C
:1004200096899588D2F800E0444F24F010040462C5
:10043000036A4468816923F0200321F0807143EA54
:10044000061321F4E641B84243EA051341EA0E21BE
:1004500048D03B4DA84245D0926844608161826398
:100460000362F0BD046A9389B2F804E01768334E62
:1004700024F001040462056A4468816943EA0E03BA
:1004800021F4803125F002059BB221F07301B042C6
:1004900043EA050341EA070114D0294DA84211D0CF
:1004A00005F54065A8420DD005F58065A84209D044
:1004B00005F58065A84205D0926844608161426379
:1004C0000362F0BDD689158A578A23F008033343A7
:1004D0003D43D68824F4407423F00403ADB2334383
:1004E0002C43E9E7D589178AD68823F0800343EAAD
:1004F000051324F44064558A23F0400344EA87043A
:1005000043EA061344EA8504A6E7D589178AD68804
:1005100023F4006343EA052324F44054558A23F46A
:10052000806344EA071443EA062344EA051470E7AB
:10053000158A24F4804444EA851449E7002C0140DC
:10054000003401402DE9F84FC82200218E488F4C1D
:10055000DFF860928E4D8F4E8F4FDFF85C821CF07B
:10056000A4FB8E488E49DFF854E2DFF854C2002223
:100570001359834200F0F880B3F1804F00F0F68009
:10058000AB4200F0F580B34200F0F480BB4200F0D3
:10059000F380734500F0F280634500F0F18043453D
:1005A00000F0F080DFF81CA2534500F0A7800AF5A8
:1005B000806A534508BF092300F0A1801432B42A91
:1005C000D6D1DFF8C881774F774D08F1B4064FF0E8
:1005D000030A4FF0020998F804301C09013C052C6D
:1005E00003F00F0300F2838037F8140040FA03F29F
:1005F000D2077CD54FF0010B0BFA03F3013B1840F7
:1006000019F0CAFF694B1B5D184415EBC0046ED08E
:1006100055F83030664898F8081003F13842920ACD
:10062000825C02F01F005209022A0BFA00FB00F064
:100630009480032A00F08A80012A05D1584A58483C
:1006400052694BEA02024261B4F804E0BEFA8EF24B
:10065000C2F11F0292B2D00803EB800002F0070241
:10066000046A92004FF00F0C0CFA02FC24EA0C040E
:100670000462046A01FA02F22243002402624FF08B
:10068000010C224603E0102A04F102042FD00CFAD8
:1006900002F030EA0E0102F10102F4D1D3F808B001
:1006A0000AFA04F1C9430BEA010BC3F808B0D3F806
:1006B00008B0C3F808B0B3F804B01FFA8BFB2BEAFC
:1006C00000009880988880B2988018680840186068
:1006D000D3F800B009FA04F040EA0B001860D868BB
:1006E000102A01EA0001D96004F10204CFD108F117
:1006F000140846457FF46FAFBDE8F88F082309EB77
:10070000C3034FF0010B93F820A00AF01F034FEA38
:100710005A1ABAF1020F0BFA03F30BD0BAF1030F16
:100720000ED0DA457FF44AAFD1F814A043EA0A03A9
:100730004B6143E7D1F818A043EA0A038B613DE718
:10074000D1F81CA043EA0A03CB6137E7144A1448E6
:10075000D2694BEA0202C26176E7114A10489269F7
:100760004BEA020282616FE70023C8E70123C6E774
:100770000223C4E70323C2E70423C0E70523BEE73F
:100780000623BCE70723BAE7046A0020B0E90208A1
:10079000000400400008004000100040002C014010
:1007A00000100240C8E70208EC420020D4E702082B
:1007B000DCE702086CD3020800400140001400404E
:1007C000003401400044014001490248FDF78EBD5C
:1007D000A46A00200048014001490248FDF786BD97
:1007E000546A00200004004002494FF08040FDF7A9
:1007F0007DBD00BF2C6A002010B5064C064821467E
:10080000FDF774FD04F178010448BDE81040FDF7E0
:100810006DBD00BF046A0020002C0140004401406F
:1008200001490248FDF762BD046A0020002C014026
:100830002DE9F74F824619F005FA484D04462F6816
:10084000E8B94748474EDFF8408116F0F4FA012531
:1008500005FA04F33B4206D00C2303FB0463404635
:10086000996816F0E8FA0134132CF1D117B93E4813
:1008700016F000FB03B0BDE8F04F16F068BB02466F
:100880003A49DFF8E09050461CF05AFA064668B93B
:100890003748384D16F0EEFA09EB060328469968FA
:1008A0000C3616F0C8FAFC2EF6D1E3E79AF80030C1
:1008B0002D2B03BF0AF1010A04F1FF344FF0010BA5
:1008C0004FF0000B4FF000080C2303FB089250463A
:1008D00096680193224631461CF032FA019B90BB88
:1008E000BBF1000F1AD0B8F1130F0BD1224B2B60C4
:1008F000224816F0BFFA1F48314603B0BDE8F04F5A
:1009000016F03CBBB8F1140F02D16B682B60EFE717
:10091000012303FA08F31F432F60E9E7B8F1130F2F
:1009200005D1C5F800B0164816F0A4FAE3E7B8F10F
:10093000140F01D16F60F6E7012303FA08F327EAE9
:1009400003072F60EFE708F10108B8F1150FBCD1DC
:100950000C4803B0BDE8F04F16F028BD3C25002040
:100960006DF4020830D6020877F4020883F4020816
:1009700088F402087FF40208FFFF0700A0F40208D1
:10098000A9F4020893F402087EF402082DE9F84F56
:10099000054619F057F9384F0446D7F80090B0B91A
:1009A0003648374D374F16F065FA012655F82410B2
:1009B00049B106FA04F313EA090F02D0384616F0DB
:1009C0003AFA0134F2E7BDE8F84F16F0C0BA024631
:1009D0002D4928461CF0B4F978B92C482C4C2D4DE3
:1009E00016F048FA54F8041F0029ECD00B78002BBD
:1009F000F8D0284616F01FFAF4E72B78DFF880B01D
:100A00002D2B03BF013504F1FF344FF0010A4FF0E5
:100A1000000A00265BF82680B8F1000F04D11E48BA
:100A2000BDE8F84F16F0C2BC2246414628461CF0ED
:100A300087F9F8B90120B040020604D51748BDE88F
:100A4000F84F16F0B3BC8305F8D4BAF1000F0AD002
:100A5000FAF7B6FA124816F00DFA41460D48BDE80D
:100A6000F84F16F08BBA40EA090038600D4816F0CE
:100A700001FAF2E70136CDE7FC290020B1F40208C3
:100A8000B4D50208BBF4020883F4020888F4020813
:100A9000B0D502087FF4020893F40208BFF40208FC
:100AA000A0F40208A9F4020870B5054619F0CAF8C6
:100AB000044690B1112200210F481CF0F6F822469E
:100AC0000E4928461CF063F938B1102C22462946FD
:100AD00028BF102208481CF06CF9094B13F8042FAA
:100AE000002A064A06BF012113460021054A0120BB
:100AF000BDE8704016F020BB902E0020931703082D
:100B00008C2E0020CBF402082DE9F04188B08046FD
:100B100016F036F9054608B33B4CDFF8F4800025A3
:100B200019274FF46176237917FB03630493E37865
:100B300017FB03630393A37802936378019314F87C
:100B4000053B009342462B4600210120013516F05B
:100B5000F3FA0A2DE7D108B0BDE8F081404619F05C
:100B6000FBFD0928064648DC8400271808F101002F
:100B70008DF81F5016F00CF9234D804648B119F03E
:100B8000EBFD0D2805D89DF81F30E85501338DF891
:100B90001F30404616F0FCF8804660B119F0DCFDCD
:100BA000431E042B07D8A3192B4458709DF81F30FF
:100BB00001338DF81F30404616F0EAF8804660B1E8
:100BC00019F0CAFD431E072B07D89DF81F30344487
:100BD0002C440133A0708DF81F30F91C0DF11F0259
:100BE0002944404616F0E1F89DF81F30052BB2D09D
:100BF000EA190023EB511371ADE709222946034896
:100C000016F0C9F9A7E700BF2A260020E9F4020878
:100C1000D3F402082DE9F04F85B0044616F0B0F881
:100C2000064620B116F0C8FB05B0BDE8F08F20469F
:100C300003AA4549DFF83C91DFF83CA1DFF83CB15D
:100C400019F0E6FD34460546B0464FF0FF37B5B91A
:100C500039463E48FAF734FD3D4B78B20C2606FB88
:100C600005F2D118D256824256D00135062DF6D162
:100C7000B8F1000F33D13748FAF722FDD4E7012E3F
:100C80000ED0022E11D01EB9284619F065FD074678
:100C900003AA2D49002019F0BBFD01360546D6E711
:100CA000284619F059FD8046F2E7494628461CF0CF
:100CB00095F820B9284928461CF090F808B144F06E
:100CC0000104514628461CF089F828B9594628469F
:100CD0001CF084F80028DBD044F00204D8E7002C94
:100CE00008BF03240022E4B2019200944346114657
:100CF0000CF0DAFE054618B91848FAF7E1FC93E75C
:100D000041461748FAF7DCFC1648FAF7D9FC164BAF
:100D10002946186818F01CF84D68002DA8D0134813
:100D2000FAF7CEFC54B169798C4207D022461048BC
:100D3000FAF7C6FCE1B22846FEF748F8EB6A002B4A
:100D4000E2D00023EB62DFE7DEF50208FBF40208E5
:100D5000B048002004F50208F2F402081CF502086D
:100D600033F5020876F502082824002048F5020829
:100D700058F50208EFF40208F5F40208F8F4020846
:100D80002DE9F743054615F0FBFF044638B1354918
:100D90000022012003B0BDE8F04316F0DFB9009057
:100DA0000190284619F0D8FC2E4B6E1C40B203EB84
:100DB000C40595F90220824250D00134062CF6D1A8
:100DC00000252C46304615F0E3FF074628B119F000
:100DD000C3FC0134ADF80000E4B2DFF88C800026DB
:100DE000384615F0D5FF0746C8B119F0B5FC814665
:100DF0000DF0AEFA58F82030994510D1022E1AD0D5
:100E0000032E1DD0431E012EDBB20FD00B2B03D8B7
:100E10008DF803000134E4B20136042EE0D1052C34
:100E200015D803B0BDE8F04316F0C6BA042BF3D8CA
:100E30008DF80400EEE70528EED88DF80600E9E706
:100E4000831EDBB20D2BE7D88DF80500E2E76B4679
:100E500003CB2860696003B0BDE8F0838DF8020021
:100E60000124AFE7CC6D002060E902082DE9F04FC6
:100E700082468FB091460E46154600273378089378
:100E800073780993F3780A9396F904300B9396F9E3
:100E9000028096F905300C93B3790D93B8F1000FE9
:100EA00004D10FB0BDE8F04F16F051B8B9F1000F02
:100EB0004ED02B78089C6A7895F90210E87895F95D
:100EC00004E095F905C095F806B09C423ED1099C16
:100ED00094423BD1884539D10A9C844236D10B9C3F
:100EE000744533D10C9C644530D10D9C5C4514BFD6
:100EF000002401240390029101920093CDF818B0D0
:100F0000CDF814C0CDF810E03B46124A21465046B9
:100F100016F0FCF80D9B06930C9B05930B9B04931A
:100F20000A9B0393099B0193089B0093CDF80880CB
:100F30003B46084A21465046013716F0FDF8102F6F
:100F400006F1070605F1070598D1AAE70024D1E7C5
:100F50004C46DFE799F502082DE9F0478AB00546CF
:100F600018F070FE024630B987490120FFF77EFF76
:100F70000AB0BDE8F0870522844928461BF0E0FE50
:100F8000044660B9702201467F481BF08EFE804BFC
:100F900020462246C2500C306028FBD1E8E70422EC
:100FA0007C4928461BF0CCFE044620BB284615F0A1
:100FB000EFFE06460028DBD018F044FEDFF8F8818B
:100FC000074658F824501DB9734816F0EFF9CFE7DB
:100FD0003A46294630461BF0B3FE50B9204612F07F
:100FE000CFFE29466D4815F0C9FF6D48FFF7B4FFE5
:100FF000BEE70134E5E707226A4928461BF0A0FE58
:101000000446002875D1202128461BF083FE0646A1
:1010100018F018FE054680BB634815F00CFF2C46FF
:10102000624D21462846013415F005FF0E2CF8D1FB
:1010300015F08DFFDFF88491554FDFF8848100248F
:101040002146484615F0F7FE0C26DFF878A100256A
:1010500006FB0476326856480123AB40134214BFA6
:1010600041465146013515F0E6FE0E2DF2D1013410
:1010700015F06DFF082CE3D17AE7304601AA4D49FF
:101080004C4E19F0C5FB02AD00283DD0022C15D105
:10109000029A072A2AD803990D2927D80378722B98
:1010A00017D06E2B22D10C2353433948012202FA68
:1010B00001F1C25822EA0102C25013E019F04CFBC0
:1010C00001AA45F824003146002019F0A1FB0134A3
:1010D000DAE70C232E4C5343012000FA01F1E058CB
:1010E0000843E0502F48FFF737FF41E716F064F957
:1010F000F8E7284601AA2F492E4E19F089FB002453
:1011000002AD78B1082C02D116F056F930E719F08B
:1011100023FB01AA45F824003146002019F078FB92
:101120000134EEE7082CEFD1029B0F2BECD8DDF851
:101130000CC0BCF1070FE7D8049F0D2FE4D8059E23
:1011400006F16402C82ADFD8069DFF2DDCD8079877
:101150006428D9D808996429D6D88842D4DA099C59
:10116000032CD1D8DFF820E0C3EBC3020EEB02035F
:101170000EF802C018715F709E70DD7059719C711D
:101180000748FFF7E9FEF3E690660020B8F502088D
:1011900050680020BEF5020893F40208C3F5020867
:1011A00047F50208CDF5020881F40208D5F50208DA
:1011B000DAF50208DEF5020848D50208F919030835
:1011C0000BF60208B6F502082DE9F04FDFF820B162
:1011D00089B08046894616460D4614464FF0000AEF
:1011E000002E71D06A6863689A426BD1AF68A368B9
:1011F000FB1A5F425F4194F90B30049394F90A3073
:101200000393B4F908300293B4F906300193B4F9AA
:10121000043000935A4653463946404615F076FF4F
:1012200095F90B30049395F90A300393B5F908301A
:101230000293B5F906300193B5F9043000935A468C
:101240005346394640460AF1010A15F075FFBAF1D6
:10125000080F05F10C0504F10C04C1D10024DFF8DE
:1012600094A0254696B30027012303FA07FB3259C1
:1012700059F8043053403BEA030314BF0123002311
:1012800012EA0B0F079306D000972B465246079998
:10129000404615F03BFF59F804301BEA030F06D017
:1012A00000972B4652460799404615F045FF0137F7
:1012B0000E2FD9D10135082D04F10C04D2D109B07B
:1012C000BDE8F08F002796E73746A9E737460123A8
:1012D00059F80420BB40134206D000972B465246D3
:1012E0000121404615F028FF01370E2FEFD1E1E72D
:1012F000E0F50208F8F50208F0B585B0054615F0EE
:101300003FFD002838D104462B78002B3BD1062C1A
:1013100041D1BDF904309AB2072A3CD8BDF9061074
:10132000A1F2EE2292B240F2DC54A24233D8BDF9CF
:101330000820A2F2EE2080B2A0422CD8BDF90A000B
:10134000814228DC824226DB914224DCBDF90C502C
:1013500005F16404A4B2C82C1DD8BDF90E40112CAF
:1013600019DC1A4E0C2707FB03639980DA80188179
:101370009D72DC7205B0F0BD14490022012005B059
:10138000BDE8F04020E72D2B03D0A3F13002092A5D
:1013900016D8052C04DD05B0BDE8F04016F00CB8F9
:1013A000284619F0D9F904AB661C03EB440424F871
:1013B0000C0C15F8013F303B092BFAD93446A3E752
:1013C000202BE8D101352646F8E700BF5068002001
:1013D0002DE9F04FDFF8E8A085B0054688461446B1
:1013E000002706237B4303930026039B334408EB2B
:1013F000030292F8C0B0002C5ED02344524693F80A
:10140000C0300193ABEB0300D0F1000949EB0009B8
:1014100000963B464946284615F078FE8DE8400880
:101420003B46524649462846013615F085FE062EB3
:10143000DBD10137062FD4D1DFF884B008F1E40AFC
:1014400000261AF8019B002C38D0A3195A4693F8AD
:10145000E4300193A9EB03014F424F41009606236C
:101460003946284615F052FE8DE840020623144AFC
:1014700039462846013615F05FFE0B2EE1D198F86B
:10148000F0606CB194F8F0300193F21A5442544178
:10149000002300930A4A07232146284615F036FE0A
:1014A0000023009301960723054A2146284615F09C
:1014B00043FE05B0BDE8F08FA146AFE72746D3E76E
:1014C0000DF602087FB5054615F05AFC044630B10A
:1014D000002218490120FFF77BFF04B070BD2846A9
:1014E0006A461549144E19F093F901AD78B1032CF1
:1014F00002D115F061FFF0E719F02EF96A4645F8C0
:1015000024003146002019F083F90134EEE7032C62
:10151000EFD101AC70CC32462946E0B20EF09AF819
:101520000028E6D033462A462146044815F026FD19
:10153000D3E700BFE0500020DEF502080DF60208F8
:101540002DE9FF47DFF86CA0814690460E46154610
:101550000027B8F1000F2AD02B8832889A4224D174
:1015600074886A88A21A54425441EA780292AA788E
:101570000192009352463B462146484615F0C6FD6F
:10158000F3780293B378019336F8043B0093524604
:101590003B4621464846013715F0CEFD102F05F198
:1015A0000405D6D104B0BDE8F0870024DDE7444649
:1015B000E6E700BF21F6020870B5064615F0E0FB2D
:1015C000044628B100220F490120BDE87040B7E76A
:1015D000304619F0C1F80F2805460BDC304615F0EF
:1015E000D7FB014628460EF05DF850B9BDE87040C3
:1015F00015F0E2BE21460F220348BDE8704015F009
:10160000CABC70BD60510020E9F402082DE9F04F1A
:10161000DFF868808FB007468A46164600240DF131
:1016200024095AF824300293494602A817F048FCCE
:1016300016B356F82430029D0393EB1A5D420DF168
:10164000100B5D41594603A817F03AFCCDF800B0E5
:10165000234642462946384615F058FD2346CDF824
:101660000090424629463846013415F065FD202C8D
:10167000D7D10FB0BDE8F08F3546EFE733F602085B
:1016800070B5064615F07CFB044628B100220F49D0
:101690000120BDE87040B9E7304619F05DF81F2819
:1016A00005460BDC304615F073FB014628460DF06D
:1016B000FBFE50B9BDE8704015F07EBE21461F22EA
:1016C0000348BDE8704015F066BC70BDE0500020D6
:1016D000E9F402082DE9F347DFF868A081460F46D8
:1016E000904602260024B8F1000F28D037F82420B5
:1016F00038F824309A4238F806201ED1BD5BA91A6A
:101700004D424D4101920093524623462946484698
:1017100015F0FCFCBB5B019337F824300093524674
:10172000234629464846013415F006FD042C06F1EF
:101730000406D8D102B0BDE8F0870025E2E74546AF
:10174000E8E700BF3DF60208F8B5054615F018FBBE
:10175000064628B1002227490120BDE8F840B9E734
:10176000254928461BF0A9FA68B9224B4FF47A7133
:101770004FF4FA6219805A809980DA8019815A816F
:101780009981DA81F8BD284618F0E6FF032804465F
:1017900028D8284615F0FCFA064658B118F0DCFFA8
:1017A00001270546304615F0F3FA30B9BDE8F84098
:1017B00015F002BE05460746F4E718F0CDFF002FEE
:1017C000F4D0A5F2EE2240F2DC539A42EED8A0F219
:1017D000EE229A42EAD8074B23F8245003EB840305
:1017E0005880F8BD314603220448BDE8F84015F0A2
:1017F000D2BB00BF44280020B8F502084EF602080C
:101800002DE9F04F2DED088BDFF80C9193B0804659
:1018100092460D461446002695ED008AB5EE408AA4
:10182000F1EE10FA71D0D5ED019A95ED029AD5ED51
:10183000038ABAF1000F3FD094ED000A94ED01BA8B
:10184000D4ED02AA94ED03AAB4EE408AF1EE10FAA8
:1018500060D1F4EE4B9AF1EE10FA5BD1B4EE6A9AD5
:10186000F1EE10FA56D1F4EE4A8AF1EE10FA0CBFFE
:10187000012700270FA8F9F749FDB0EE4B0A834670
:101880000CA8F9F743FDB0EE6A0A059009A8F9F72C
:101890003DFDB0EE4A0A049006A8F9F737FD049A18
:1018A000059B039002920193CDF800B033464A465F
:1018B0003946404615F02AFCB0EE480A0FA8F9F761
:1018C00025FDB0EE690A07460CA8F9F71FFDB0EE3A
:1018D000490A834609A8F9F719FDB0EE680A049091
:1018E00006A8F9F713FD049B039002938DE8800886
:1018F00033464A4600214046013615F01DFC0C2EA9
:1019000005F1100504F1100486D113B0BDEC088B6D
:10191000BDE8F08F0027ADE756F602082DE9F04745
:10192000494E4A4FDFF83C810446204615F028FA1C
:10193000814628B1002246490120BDE8F0475FE713
:101940000522314620461BF0FBF940B940490022F0
:1019500043181030C0281A60FAD1BDE8F08704227D
:10196000394620461BF0ECF90546204615BB15F01C
:101970000FFA8146002864D018F064F92C465FFA0B
:1019800080FA58F8245025B93248BDE8F04715F0E0
:101990000DBD5246294648461BF0D2F940B92046B3
:1019A00017F05EFA29462C482C4C15F0E7FABCE7F4
:1019B0000134E6E718F0D0FE0B2805463AD8204659
:1019C00015F0E6F9064648B3F9F7F8FB204B03EBB0
:1019D000051383ED000A0124304615F0D9F90646B7
:1019E00038B1F9F7EBFB1A4B03EB051383ED010A52
:1019F0000134304615F0CCF9064638B1F9F7DEFB74
:101A0000134B03EB051383ED020A0134304615F046
:101A1000BFF928B9BDE8F04715F0CEBC0446DBE7B6
:101A2000F9F7CCFB0A4B032C03EB051585ED030AF4
:101A3000F0D17FE749460B220948BDE8F04715F091
:101A4000AABABDE8F08700BFB8F50208BEF50208E3
:101A5000047A002093F40208C3F5020847F502084F
:101A6000E9F4020848D502082DE9F04F834687B013
:101A700092460C46154600274FF019094FF461783D
:101A8000BAF1000F4ED023782A7893422B7947D1B0
:101A900060786978884243D1A078A97888423FD19C
:101AA000E078E97888423BD12179994238D166794A
:101AB0006979711A4E424E410593EB780493AB78E5
:101AC00019FB038303936B78019219FB0383029341
:101AD0006B790093144A3B463146584615F016FB85
:101AE00023790593E3780493A3780F4A19FB0383C2
:101AF0000393637819FB038302932378019363793B
:101B0000009331463B465846013715F015FB0F2F21
:101B100004F1060405F10605B2D107B0BDE8F08F67
:101B20000026C9E75646DBE76AF60208F7B507461E
:101B300015F026F9044630B1002236490120FFF79E
:101B400093FF03B0F0BD384618F006FE0E28054698
:101B500059DC06264643781C8DF8074015F018F925
:101B60002C4C074650B118F0F7FD032806D8A319EE
:101B700058719DF8073001338DF80730384615F05D
:101B800007F9074658B118F0E7FD0D2807D80623D6
:101B90006B43E0549DF8073001338DF80730711C1A
:101BA0000DF107022144384615F0FFF815F0F0F862
:101BB000074660B118F0D0FD182808D8062303FBAB
:101BC0000543D8709DF8073001338DF8073038464B
:101BD00015F0DEF860B118F0BFFD0D2808D8062317
:101BE00003FB05459DF80730287101338DF8073058
:101BF0009DF80730062BA4D0A2190023A35193808F
